:100000000C94980C0C94BD0C0C94BD0C0C94BD0C71
:100010000C94BD0C0C94BD0C0C94BD0C0C94BD0C3C
:100020000C94BD0C0C94BD0C0C948B0F0C94BD0C5B
:100030000C94BD0C0C94BD0C0C94BD0C0C94BD0C1C
:100040000C94BD0C0C94BD0C0C94BD0C0C94BD0C0C
:100050000C94BD0C0C94BD0C0C94BD0C0C94BD0CFC
:100060000C94BD0C0C94BD0C0C94BD0C0C94BD0CEC
:100070000C94BD0C0C94BD0C0C94BD0C0C94BD0CDC
:100080000C94BD0C0C94BD0C0C94BE0C0C941B3049
:100090000C94BD0C0C94BD0C0C94BD0C0C94BD0CBC
:1000A0000C94BD0C0C94BD0C0C94BD0C0C94BD0CAC
:1000B0000C94BD0C0C94BD0C0C94BD0C0C94B4278A
:1000C0000C94BD0C0C944A2B0C948D310C94BD0CEB
:1000D0000C94BD0C0C94BD0C0C94BD0C0C94BD0C7C
:1000E0000C94BD0C0C94BD0C0C94BD0C0C94BD0C6C
:1000F0000C94BD0C0C94BD0C0C94BD0C0C94BD0C5C
:100100000C94BD0C0C94BD0C0C94BD0C0C94BD0C4B
:100110000C9466310C94252B0C94BD0C0C94BD0CE6
:100120000C94BD0C0C94BD0C0C94BD0C0C94BD0C2B
:100130000C94BD0C0C94BD0C0C94BD0C0C941C27A1
:100140000C940A0D0C94C80C0C9449300C94BD0C02
:100150000C94BD0C0C949C2A0C94C3310C94BD0CD3
:100160000C94BD0C0C94BD0C0C94BD0C0C94BD0CEB
:100170000C94BD0C0C94BD0C0C94BD0C0C94BD0CDB
:100180000C94BD0C0C94BD0C0C94BD0C0C94BD0CCB
:100190000C94BD0C0C94BD0C0C94BD0C0C94BD0CBB
:1001A0000C94BD0C0C94BD0C0C94BD0C0C94BD0CAB
:1001B0000C94BD0C0C94BD0C0C94BD0C0C94BD0C9B
:1001C0000C94BD0C0C94BD0C0C94BD0C0C94BD0C8B
:1001D0000C94BD0C0C94BD0C0C94BD0C0C94BD0C7B
:1001E0000C94BD0C0C94BD0C0C94BD0C0C94BD0C6B
:1001F0000C94BD0C0C94676D0C94BD0C1E03430055
:10020000680061006D0065006C0065006F006E00A5
:100210002D004D0069006E00690000002A034B00AC
:10022000610073007000650072002000260020004D
:100230004F007300770061006C00640020004700ED
:100240006D006200480000000403090409023E003A
:10025000020100C03209040000010202010005246D
:10026000001001042402060524060001070582038C
:100270000800FF09040100020A000000070504024B
:10028000100005070583021000051201100102008D
:100290000008D016B20401000102DC01351036104E
:1002A0003710381039103A103B103C103F104010F6
:1002B00000000001007528F62815292B3547355117
:1002C000353B1052356339763940000700017528F7
:1002D000F6281529B5344B3551353B105235633965
:1002E0007639C0000700017528F62815293F3547E3
:1002F0003551353B105235633976395000070001CE
:100300007528F62815294335473551353B105235A8
:1003100063397639A4000700017528F6281529B637
:1003200039013A053A3B10063AFD401941400104B3
:1003300000017528F6281529C539013A053A3B1000
:10034000063AFD40194100040400017528F62815FD
:1003500029D439013A053A3B10063AFD40194100CB
:10036000040700017528F6281529E339013A053AF2
:100370003B10063AFD40194100100400017528F6B3
:10038000281529F239013A053A3B10063AFD401981
:100390004100100700017D323C335D33375845582A
:1003A0004A584B584D583F1040100000000100F0D3
:1003B00029782AE62B47504A505750585009533F46
:1003C00010401000000000004F5CD25C055D995D9C
:1003D0009C5D9F5DA05DA15D845E8B5E002008003A
:1003E000054F5CD25C055D381039103A103B103C6B
:1003F000103F10401000000001004F5CD25C055D12
:10040000925E955E985E995E9A5E8B609260002027
:100410000800054F5CD25C055D9960B760C560C699
:1004200060E660D86037622C000800054F5CD25C43
:10043000055D5F637663866387634167D3665E6845
:10044000D000080005004E4F4E450000000000009F
:10045000000000000000000000000000000000009C
:10046000000000000000014D465F554C5452414CC5
:100470004947485400000000000000000000000050
:1004800000000000000000034D465F554C545241EF
:100490004C494748545F4556315F383042000000B0
:1004A0000000000000000000044D465F554C54520F
:1004B000414C494748545F4556315F31363442001C
:1004C000000000000000000000024D465F554C5443
:1004D00052414C494748545F43000000000000006F
:1004E00000000000000000000000054D465F434C86
:1004F00041535349435F4D494E495F344200000028
:100500000000000000000000000000064D465F43B0
:100510004C41535349435F314B0000000000000041
:10052000000000000000000000000000074D465FD2
:10053000434C41535349435F314B5F374200000006
:1005400000000000000000000000000000084D4610
:100550005F434C41535349435F344B00000000005C
:100560000000000000000000000000000000094D35
:10057000465F434C41535349435F344B5F3742001E
:100580000000000000000000000000000000000A61
:1005900049534F3134343433415F534E494646005A
:1005A000000000000000000000000000000000004B
:1005B0000B49534F3134343433415F524541444544
:1005C00052000000000000000000000000000000D9
:1005D000000C564943494E495459000000000000A0
:1005E000000000000000000000000000000000000B
:1005F00000000D49534F31353639335F534E49466C
:1006000046000000000000000000000000000000A4
:100610000000000E534C32533230303200000000E4
:1006200000000000000000000000000000000000CA
:10063000000000000F544954414749545354414E5F
:10064000444152440000000000000000000000008F
:10065000000000000010454D34323333000000002C
:10066000000000000000000000000000000000008A
:100670000000000000000100000100010100000175
:100680000100010000010001010001000001010062
:100690000001000101000001010001000001010052
:1006A0000001000101000100000100010100000142
:1006B0000100010000010001010001000001010032
:1006C0000001000101000100000100010100000122
:1006D0000100010000010100000100010100000112
:1006E0000100010000010001010001000001010002
:1006F00000010001010000010100010000010100F2
:1007000000010001010001000001000101000001E1
:1007100001000100000101000001000101000001D1
:1007200001000100000100010100010000010100C1
:1007300000010001010001000001000101000001B1
:1007400001000100000100010100010000010100A1
:100750000001000101000001010001000001010091
:100760000001000101000100000100010100000181
:10077000010001000001008040C020A060E0109056
:1007800050D030B070F0088848C828A868E8189899
:1007900058D838B878F8048444C424A464E4149481
:1007A00054D434B474F40C8C4CCC2CAC6CEC1C9C39
:1007B0005CDC3CBC7CFC028242C222A262E212925D
:1007C00052D232B272F20A8A4ACA2AAA6AEA1A9A39
:1007D0005ADA3ABA7AFA068646C626A666E6169621
:1007E00056D636B676F60E8E4ECE2EAE6EEE1E9ED9
:1007F0005EDE3EBE7EFE018141C121A161E111911B
:1008000051D131B171F1098949C929A969E9199908
:1008100059D939B979F9058545C525A565E51595F0
:1008200055D535B575F50D8D4DCD2DAD6DED1D9DA8
:100830005DDD3DBD7DFD038343C323A363E31393CC
:1008400053D333B373F30B8B4BCB2BAB6BEB1B9BA8
:100850005BDB3BBB7BFB078747C727A767E7179790
:1008600057D737B777F70F8F4FCF2FAF6FEF1F9F48
:100870005FDF3FBF7FFF004E4F4E4500000000008E
:100880000000000000000000000000000000000068
:1008900000000000000000015549445F52414E44F1
:1008A0004F4D0000000000000000000000000000AC
:1008B0000000000000000000025549445F4C45461E
:1008C000545F494E4352454D454E540000000000D0
:1008D000000000000000000000035549445F524939
:1008E0004748545F494E4352454D454E5400000021
:1008F00000000000000000000000045549445F4C67
:100900004546545F44454352454D454E5400000012
:100910000000000000000000000000055549445F91
:1009200052494748545F44454352454D454E540053
:1009300000000000000000000000000006435943D2
:100940004C455F53455454494E4753000000000046
:1009500000000000000000000000000000075354E9
:100960004F52455F4D454D00000000000000000063
:10097000000000000000000000000000000008521D
:100980004543414C4C5F4D454D00000000000000C8
:10099000000000000000000000000000000000094E
:1009A000544F47474C455F4649454C4400000000C2
:1009B0000000000000000000000000000000000037
:1009C0000A53544F52455F4C4F470000000000004F
:1009D0000000000000000000000000000000000017
:1009E000000B434C4F4E450000000000000000008B
:1009F00000000000000000000000000000000000F7
:100A000000000C434C4F4E455F4D46550000000022
:100A100000000000000000000000000000000000D6
:100A2000000000004F4646000000000000000000EB
:100A300000000000000000000000000000000000B6
:100A400000000000014D454D4F52590000000000CC
:100A50000000000000000000000000000000000096
:100A60000000000000024C49564500000000000054
:100A70000000000000000000000000000000000076
:100A8000000000000000004E4F4E45000000000036
:100A90000000000000000000000000000000000056
:100AA0000000000000000001504F5745524544002F
:100AB0000000000000000000000000000000000036
:100AC0000000000000000000025445524D494E4114
:100AD0004C5F434F4E4E000000000000000000003D
:100AE000000000000000000000035445524D494E34
:100AF000414C5F52585458000000000000000000B4
:100B00000000000000000000000004534554544958
:100B10004E475F4348414E4745000000000000003B
:100B20000000000000000000000000054D454D4F92
:100B300052595F53544F52454400000000000000DA
:100B4000000000000000000000000000064D454DC0
:100B50004F52595F4348414E474544000000000052
:100B60000000000000000000000000000008434FEB
:100B70004445435F525800000000000000000000A0
:100B80000000000000000000000000000000094319
:100B90004F4445435F54580000000000000000002F
:100BA000000000000000000000000000000000073E
:100BB0004649454C445F4445544543544544000030
:100BC0000000000000000000000000000000000025
:100BD0000A4C4F474D454D5F46554C4C00000000B8
:100BE0000000000000000000000000000000000005
:100BF0000025632C25630025356400416E7920694A
:100C00006E74656765722066726F6D203020746F38
:100C10002025752E205265666572656E63652076A7
:100C20006F6C746167652077696C6C206265202841
:100C3000564343202A205448524553484F4C4420A1
:100C40002F203430393529206D562E00257500258A
:100C500035640030203D206E6F2074696D656F75BE
:100C6000740D0A312D363030203D20313030206D6A
:100C700073202D203630303030206D732074696D34
:100C8000656F7574002575206D730025342E3458FA
:100C900000253575206D56002575202866726F6D0C
:100CA000207768696368202575206E6F6E2D766FDA
:100CB0006C6174696C6529002575002575002563D4
:100CC0002C25630052414E444F4D004E4F20554954
:100CD000442E004368616D656C656F6E4D696E6989
:100CE0002052657647202553207573696E67204C26
:100CF00055464120255320636F6D70696C656420F3
:100D000077697468204156522D4743432025532E5E
:100D1000204261736564206F6E20746865206F7077
:100D2000656E2D736F75726365204E464320746F38
:100D30006F6C204368616D656C656F6E4D696E699F
:100D40002E2068747470733A2F2F67697468756207
:100D50002E636F6D2F656D7365632F4368616D65DD
:100D60006C656F6E4D696E6920636F6D6D6974207F
:100D7000255300313931323131003135313131359E
:100D800000342E392E320038363864386236000D81
:100D90000A000D0A000D0A000D0A000D0A000D0AD6
:100DA00000643130303A4F4B00000000000000007A
:100DB0000000000000000000000000000000000033
:100DC0000000653130313A4F4B2057495448205488
:100DD0004558540000000000000000000000000022
:100DE0000000006E3131303A57414954494E472096
:100DF000464F5220584D4F44454D00000000000022
:100E000000000000C83230303A554E4B4E4F574E1E
:100E100020434F4D4D414E440000000000000000B3
:100E20000000000000C93230313A494E56414C4969
:100E30004420434F4D4D414E4420555341474500BA
:100E4000000000000000CA3230323A494E56414C90
:100E5000494420504152414D455445520000000044
:100E600000000000000000783132303A46414C5317
:100E7000450000000000000000000000000000002D
:100E80000000000000000000793132313A54525520
:100E9000450000000000000000000000000000000D
:100EA000000000000000000000CB3230333A54490B
:100EB0004D454F55540000000000000000000000A8
:100EC0000000000000000000000056455253494F4A
:100ED0004E000000000000000000000000000000C4
:100EE0007B1C434F4E4649470000000000000000B5
:100EF000000000000000A31C9D1C55494400000098
:100F00000000000000000000000000000000041DC0
:100F1000C51C524541444F4E4C5900000000000092
:100F2000000000000000691D5D1D55504C4F4144FC
:100F300000000000000000000000961D00000000FE
:100F40000000444F574E4C4F414400000000000049
:100F500000009B1D00000000000052455345540056
:100F600000000000000000000000A01D00000000C4
:100F70000000555047524144450000000000000069
:100F80000000AB1D0000000000004D454D53495AC4
:100F9000450000000000000000000000000000000C
:100FA000B61D55494453495A450000000000000051
:100FB0000000000000000000CE1D52425554544F66
:100FC0004E00000000000000000000000000EB1DCB
:100FD000E41D52425554544F4E5F4C4F4E47000053
:100FE000000000000000071E001E4C425554544FE4
:100FF0004E00000000000000000000000000231E62
:101000001C1E4C425554544F4E5F4C4F4E470000EF
:101010000000000000003F1E381E4C45444752456A
:10102000454E0000000000000000000000005B1EB4
:10103000541E4C454452454400000000000000008E
:10104000000000000000771E701E4C4F474D4F44BB
:101050004500000000000000000000000000911E9C
:101060008C1E4C4F474D454D000000000000000015
:101070000000000000000000A61E4C4F47444F57E0
:101080004E4C4F41440000000000CB1E0000000009
:1010900000004C4F4753544F5245000000000000E1
:1010A0000000D01E0000000000004C4F47434C459C
:1010B00041520000000000000000D31E00000000AC
:1010C000000053455454494E470000000000000002
:1010D000000000000000DB1ED61E434C45415200BC
:1010E00000000000000000000000E31E00000000FF
:1010F000000053544F524500000000000000000063
:101100000000E71E000000000000524543414C4C27
:1011100000000000000000000000EB1E00000000C6
:1011200000004348415247494E470000000000007C
:101130000000000000000000EF1E48454C50000079
:1011400000000000000000000000F71E000000008A
:10115000000052535349000000000000000000004E
:101160000000000000000000331F5359535449434E
:101170004B00000000000000000000000000000024
:10118000661F53454E445F52415700000000000067
:10119000000000000C200000000053454E440000F9
:1011A000000000000000000000000000821F00009E
:1011B000000047455455494400000000000000006D
:1011C0000000DF2000000000000044554D505F4D3E
:1011D00046550000000000000000AB2000000000A9
:1011E0000000434C4F4E455F4D4655000000000047
:1011F0000000C8200000000000004944454E54494A
:1012000046590000000000000000FC200000000023
:10121000000054494D454F555400000000000000A7
:10122000000000000000392119215448524553485C
:101230004F4C440000000000000000000000A62108
:101240008C214155544F43414C4942524154450031
:10125000000035220000000000004649454C4400D3
:101260000000000000000000000000000000FB2162
:101270002522434C4F4E45000000000000000000B6
:1012800000006122000000000000000000000000DB
:10129000000000000000000000000000000000004E
:1012A000000053414B3A09005549443A0900415462
:1012B00051413A0900546865726520697320617470
:1012C000206C65617374206F6E65206D6F72652090
:1012D0006361726420747970652063616E6469640F
:1012E0006174652C2062757420746865726520775E
:1012F0006173206E6F7420656E6F7567682074650A
:10130000726D696E616C20627566666572207370BD
:101310006163652E0D0A000D0A0004000109010039
:1013200000000000000000000000000000000000BD
:10133000004E5850000000000000000000000000B7
:10134000004D4946415245204D696E69000000003C
:10135000000000000000000000000000000000008D
:10136000000000000000000000000000000000007D
:10137000000000000000000000000000000000006D
:10138000000400010801000000000000000000004F
:1013900000000000000000004E5850000000000057
:1013A00000000000000000004D4946415245204326
:1013B0006C617373696320316B00000000000000F2
:1013C000000000000000000000000000000000001D
:1013D000000000000000000000000000000000000D
:1013E00000000000000000000200011801000000E1
:1013F0000000000000000000000000000000004E9F
:101400005850000000000000000000000000004DE7
:10141000494641524520436C617373696320346BC4
:1014200000000000000000000000000000000000BC
:1014300000000000000000000000000000000000AC
:101440000000000000000000000000000000004458
:10145000000100010000000000000000000000008A
:101460000000000000004E58500000000000000086
:101470000000000000004D494641524520556C7463
:1014800072616C6967687400000000000000000071
:10149000000000000000000000000000000000004C
:1014A000000000000000000000000000000000003C
:1014B00000000000000044030120017577810280D4
:1014C000000000000000000000000005004E585021
:1014D000000000000000000000000000004D494630
:1014E00041524520444553466972650000000000A2
:1014F00000000000000000000000000000000000EC
:1015000000000000000000000000000000000000DB
:101510000000000000000000000000000044030183
:1015200020017577810280000000000000000000AB
:10153000000005004E5850000000000000000000B0
:10154000000000004D49464152452044455346693C
:1015500072652045563100000000000000000000C8
:10156000000000000000000000000000000000007B
:10157000000000000000000000000000000000006B
:101580000000000004030128013877B14A434F509E
:10159000333100000000000000090149424D000005
:1015A00000000000000000000000004A434F5033DC
:1015B00031000000000000000000000000000000FA
:1015C000000000000000000000000000000000001B
:1015D000000000000000000000000000000000000B
:1015E0000000000000000000000000480001200191
:1015F0007877B1024A434F50763234310000000010
:101600000C0149424D0000000000000000000000F5
:1016100000004A434F5033312076322E342E3100B1
:1016200000000000000000000000000000000000BA
:1016300000000000000000000000000000000000AA
:10164000000000000000000000000000000000009A
:10165000000048000120013833B14A434F50343173
:10166000563232000000000C0149424D00000000DB
:101670000000000000000000004A434F50343120B9
:1016800076322E3200000000000000000000000052
:10169000000000000000000000000000000000004A
:1016A000000000000000000000000000000000003A
:1016B0000000000000000000000400012801383391
:1016C000B14A434F503431563233310000000D01DE
:1016D00049424D0000000000000000000000000032
:1016E0004A434F5034312076322E332E31000000E1
:1016F00000000000000000000000000000000000EA
:1017000000000000000000000000000000000000D9
:1017100000000000000000000000000000000000C9
:10172000040001880100000000000000000000002B
:1017300000000000000000496E66696E656F6E0073
:10174000000000000000004D494641524520436C16
:10175000617373696320316B0000000000000000BA
:101760000000000000000000000000000000000079
:101770000000000000000000000000000000000069
:1017800000000000000000020001980100000000BD
:10179000000000000000000000000000000047659D
:1017A0006D706C75730000000000000000004D506B
:1017B000434F530000000000000000000000000044
:1017C0000000000000000000000000000000000019
:1017D0000000000000000000000000000000000009
:1017E0000000000000000000000000000000000CED
:1017F00001000000000000000000000000000000E8
:101800000000000000496E6E6F766973696F6E208C
:1018100052265400004A6577656C00000000000005
:1018200000000000000000000000000000000000B8
:1018300000000000000000000000000000000000A8
:101840000000000000000000000000000000000098
:10185000000000000002000138010000000000004C
:101860000000000000000000000000004E6F6B69E7
:101870006100000000000000000000004D494641EA
:10188000524520436C617373696320346B202D20B3
:10189000656D756C61746564202836323132204381
:1018A0006C61737369632900000000000000000090
:1018B00000000000000000000000000008000138E7
:1018C0000100000000000000000000000000000017
:1018D0000000004E6F6B6961000000000000000016
:1018E0000000004D494641524520436C61737369C5
:1018F0006320346B202D20656D756C6174656420E8
:101900002836313331204E464329000000000000C4
:1019100000000000000000000000000000000000C7
:101920000000006364696E6F70737578585B000027
:1019300011241FBECFEFCDBFDFE3DEBF00E00CBF41
:1019400018BE19BE1ABE1BBE14E2A0E0B0E2ECEE57
:10195000FEEE00E00BBF02C007900D92AA38B1075F
:10196000D9F71BBE27E3AAE8B4E201C01D92A73A4B
:10197000B207E1F7D3D10C947477C4C2EF93FF930D
:10198000E0918D2FF0918E2F0995FF91EF91189591
:10199000EF93FF93E0918B2EF0918C2E0995FF91A0
:1019A000EF9118953BB78BBFFB01879196913BBF99
:1019B00008953BB78BBFCB0142E20D94F00F3BB7CC
:1019C0000B0143E20D94F00F3BB78BBFCB0145E217
:1019D0000D94F00F3BB746E208C02091CF0127FDE0
:1019E000FCCF22272093CA0108954093CA0128ED15
:1019F00031E0209334003093CB016091C4017091A9
:101A0000C5018091C60199270895FC014093CA0140
:101A1000849108950F9200240F932F933F934F9337
:101A20005F930FB70F93EF93FF93EAB1FBB151911F
:101A3000442735B124B1569578F400928C08009271
:101A4000000806E10A95F1F700C001E000930008E4
:101A500003E000938C0804C00AE10A95F1F7000046
:101A60002150304019F40E948A2A0CC04F5F477001
:101A700011F4519102C000C000C00AE00A95F1F7CC
:101A800000C0D9CFFF91EF910F910FBF5F914F91A0
:101A90003F912F910F910F901895F190E190D19077
:101AA000C190B190A190919081900B941B942B9434
:101AB0003B944B945B946B947B948B949B94AB94EE
:101AC000BB94CB94DB94EB94FB940895F801D894E9
:101AD000E4DF5894E2DFD894E0CFF801D894DDDF5A
:101AE0005894DBDFF801D894D8CFF801D894D5CF3B
:101AF000F8015894D2CFF80170965894CEDFF801CF
:101B00003896D894CADFF8015894C7CFF801589492
:101B1000C4DFD894C2DFF8015894BFCFFF90EF9094
:101B2000DF90CF90BF90AF909F908F907F906F90FD
:101B30005F904F903F902F90112408952F923F92E5
:101B40004F925F926F927F928F929F92AF92BF92CD
:101B5000CF92DF92EF92FF920F931F93FB01719050
:101B600061905190419031902190119001908A01A3
:101B7000CDDFFC017192619251924192319221929A
:101B8000119201921F910F91C9CF2F923F924F92C4
:101B90005F926F927F928F929F92AF92BF92CF92FD
:101BA000DF92EF92FF920F931F93FC01719061906F
:101BB0005190419031902190119001908A018DDFD8
:101BC000FB01719261925192419231922192119254
:101BD00001921F910F91A2CF2F923F924F925F924D
:101BE0006F927F928F929F92AF92BF92CF92DF922D
:101BF000EF92FF92CF93DF93EB01DA01BF01F9017E
:101C0000719061905190419031902190119001908C
:101C1000F990E990D990C990B990A990999089903C
:101C20007F246E245D244C243B242A241924082478
:101C3000FB0109957D926D925D924D923D922D92A0
:101C40001D920D92019721F7D9017D926D925D92BF
:101C50004D923D922D921D920D92DF91CF915ECFCC
:101C60002F923F924F925F926F927F928F929F92AC
:101C7000AF92BF92CF92DF92EF92FF92CF93DF931A
:101C8000EB01DA01BF01788069805A804B803C808B
:101C90002D801E800F80FB010995F901F190E190E4
:101CA000D190C190B190A190919081907F246E24A9
:101CB0005D244C243B242A2419240824F990E9901B
:101CC000D990C990B990A99099908990F901F19211
:101CD000E192D192C192B192A192919281927D9220
:101CE0006D925D924D923D922D921D920D920197B3
:101CF00051F6DF91CF9112CFFDE0EDE66DCFFDE023
:101D0000EDE6AECFFDE0E6E867CFFDE0E6E8A8CF80
:101D1000FDE0E6E661CFFDE0EBE7A2CF15D10E9442
:101D200097190E94331AC9D21092520684E0809308
:101D3000420682E680938601C1E0C0932606C093E6
:101D4000210686E080932206C093310612E01093AC
:101D5000320610922A0610922B068FE080932906F5
:101D600089E5809380019AE59093810180938201B7
:101D700080E480934106809346069091B200907F64
:101D80009093B2009091B20092609093B20090E371
:101D9000909341069093460680935006C093460662
:101DA0001093450603E00093410683E18093010808
:101DB00021E030E02093260830932708209328085C
:101DC0003093290810928C08809380081092230386
:101DD00010922103D8E0D093220381E18093200365
:101DE000E091AD2FF091AE2F8285938580933803DB
:101DF000909339038CE380938203D0938003809384
:101E00008303D09381036FD10E94DE1BC0D155D7CD
:101E1000C093000210920102109302020093040288
:101E2000C0932002D09321020E94221819D1D2E03F
:101E3000C1E18091030481FF25C08091010480FDF0
:101E4000FCCFD09303040E94371AB6D10E94111C14
:101E50003CD70E949219E0919D2FF0919E2F1995E9
:101E60000E9451250E947B1BE091AD2FF091AE2F77
:101E70008781813011F4C093932C8681813011F4D5
:101E8000C093922C0E94E21BDED7E0919B2FF09131
:101E90009C2F1995E091952FF091962F1995C9CF08
:101EA000292F33272230310559F02330310569F0CD
:101EB00021303105F9F482E190E02AE832E01EC0D9
:101EC0008EE390E02CE432E019C09927813091052F
:101ED00041F08230910541F0892B61F4E8E4F2E0B1
:101EE00005C0ECE1F2E002C0ECEFF1E0849190E09B
:101EF0009F0104C080E090E020E030E0FA01208300
:101F0000318308951F920F920FB60F92112408B6D5
:101F10000F9218BEFFCF1F920F920FB60F9211248F
:101F200008B60F9218BE8F939F938EB19FB18058C1
:101F30009F4F8EB99FB99F918F910F9008BE0F90C0
:101F40000FBE0F901F9018958091780083FF0AC0F4
:101F500088E08093780088ED84BF81E080938000E2
:101F60000D94FE008BEC80935200809150008860AD
:101F7000809350008091510083FFFCCF82EC8093CE
:101F800055008091500080618093500080915100F5
:101F900084FFFCCF88ED84BF84E0809340001EB8AE
:101FA0001FB881E0809343002FE730E020930A04BC
:101FB00030930B0420930C0430930D0480930004A1
:101FC0008093020480E880930001089588ED84BF27
:101FD00081E080937900089588ED84BF8BE1809340
:101FE000800008958091500082608093500080911D
:101FF000510081FFFCCF82E08093CA01EDE1F0E067
:10200000E491E0936200ECE1F0E0E491E09363009E
:102010001092CA0180E8809365008BEB8093660084
:1020200080915600897F809356008091560084608D
:1020300080935600809160008160809360000895D5
:10204000E0E4F0E084818E7F8483E0E6F0E080814C
:102050008E7F8083E0E5F0E080818D7F808308952E
:1020600087E08093A20078940895089508950895D4
:10207000089508950895089580E090E008950895E2
:1020800008950F931F93CF93DF931F92CDB7DEB7C1
:1020900001E91FE2D8011296ED91FC911397898313
:1020A00019950E948925E091AD2FF091AE2F89817D
:1020B0008583B9E18B9FB001112464567D4F49E1BE
:1020C00050E0C8010E944C70D801ED91FC91199527
:1020D000D8011696ED91FC9117970F90DF91CF9153
:1020E0001F910F91199449E150E06CE972E081E988
:1020F0009FE20E944C70E091AD2FF091AE2F858150
:10210000C0CF0F931F93E091AD2FF091AE2F8B01B5
:102110009C01458161E185E494E00E94181B1F91B8
:102120000F910895FF920F931F93CF93DF931F9208
:10213000CDB7DEB78C019E012F5F3F4FAC0161E14F
:1021400085E494E00E94301BF82E882389F0898171
:1021500098DFF80140E08191882319F04F5F4F31FB
:10216000D1F7E091AA2FF091AB2FB80181E1199539
:102170008F2D0F90DF91CF911F910F91FF900895B8
:102180009B01AC0161E185E494E00C94571B089538
:102190000C943E7008951F93CF93DF93C82FD92FCF
:1021A000162F180F1C1721F00E943E708993FACF4A
:1021B000DF91CF911F9108950E943E700E943E7062
:1021C0000E943E700C943E70EF92FF920F931F930B
:1021D000CF93DF937C0161507109FA018A01020FEC
:1021E000131FDC0140E050E0E017F107F1F062302E
:1021F0007105D8F09191392F32953F703A3010F433
:10220000305D01C0395C3C939F709A3010F4905D52
:1022100001C0995C9701240F351FE901998312963B
:10222000625071094E5F5F4FDFCF1C92CA01DF9190
:10223000CF911F910F91FF90EF900895CF93DF936F
:10224000EC01DA01E0E0F0E04C91442391F11196C9
:102250009C911197992339F1E617F70721F180ED49
:10226000840F8A3020F08FEB840F8630D0F480ED1D
:10227000890F8A3020F02FEB290F263090F4242F7D
:1022800030E0413410F0275331092295207F9134FA
:1022900010F4982F01C09753292B29933196129649
:1022A000D3CF80E004C011968C91811102C090E0E0
:1022B00001C0CF01DF91CF910895E0E6F6E080E123
:1022C000858382E0868388E085838AE18183E0EAF2
:1022D000F9E01682178280EC858388E18483E0E050
:1022E000F1E0128A8BE6838B148A158A20EA208F0C
:1022F00099E0918F128E148E158E168E84E0808B4D
:1023000012A23CE633A314A215A210A611A612A68F
:1023100024A795A716A680A308954115510509F491
:1023200049C020E12093660623E02093A009209174
:10233000A10927FFFCCF2091A0097093A00920914B
:10234000A10927FFFCCF2091A0096093A00920914B
:10235000A10927FFFCCF2091A00921E020931201C1
:1023600080931C0190931D0140931401509315011B
:10237000109222018AE894E2809328019093290127
:10238000409324015093250180911001806880932F
:1023900010018091200180688093200180911001BC
:1023A00087FDFCCF80E3809311018093210180E1C0
:1023B0008093650608954115510509F469C020E12F
:1023C0002093660626E02093A0092091A10927FF0B
:1023D000FCCF2091A00920E12093650600000000B9
:1023E0002093660622E02093A0092091A10927FFEF
:1023F000FCCF2091A0097093A0092091A10927FF8B
:10240000FCCF2091A0096093A0092091A10927FF8A
:10241000FCCF2091A009109212012AE834E2209307
:102420001C0130931D01409314015093150120E1CC
:102430002093220180932801909329014093240145
:102440005093250180911001806880931001809144
:1024500020018068809320018091100187FDFCCFCE
:1024600080E3809311018093210180E180936506D0
:10247000E091AD2FF091AE2F8781863019F481E184
:102480008093932C8681863019F481E18093922C7D
:102490000895CF92DF92EF92FF92CF93DF93C09097
:1024A000AC2FD12CE12CF12C8DE0CC0CDD1CEE1CE2
:1024B000FF1C8A95D1F7C114D10481E0E806F1042C
:1024C00008F04EC080E18093660686E08093A00904
:1024D0008091A10987FFFCCF8091A00980E18093C2
:1024E0006506000000008093660682E08093A009E4
:1024F0008091A10987FFFCCF8091A0091092A009CB
:102500008091A10987FFFCCF8091A0091092A009BA
:102510008091A10987FFFCCF8FEFE81AF80A80911C
:10252000A009C0E0D0E1C701B6013CDA8093A00960
:102530008091A10987FFFCCF8091A0099093A00909
:102540008091A10987FFFCCF8091A00982E0C80E8D
:10255000D11CE11CF11C219731F780E180936506C5
:102560008091010480FDFCCF82E080930304DF9121
:10257000CF91FF90EF90DF90CF900895CF92DF92B0
:10258000EF92FF92CF93DF93C090AC2FD12CE12C30
:10259000F12C8DE0CC0CDD1CEE1CFF1C8A95D1F7D4
:1025A000C114D10481E0E806F10438F0DF91CF9145
:1025B000FF90EF90DF90CF906CCF8FEFE81AF80A82
:1025C000C1E2D0E0219791F308DAC701B601F1D951
:1025D00004DA8FEFD81AE80AF80AF4CFCF92DF9224
:1025E000EF92FF920F931F93CF93DF93C090AC2F86
:1025F000D12CE12CF12C8DE0CC0CDD1CEE1CFF1C51
:102600008A95D1F7C114D10481E0E806F10408F0FD
:102610004FC080E18093660683E08093A00980919B
:10262000A10987FFFCCF8091A0091092A009809199
:10263000A10987FFFCCF8091A0091092A009809189
:10264000A10987FFFCCF8FEFE81AF80A8091A00953
:10265000C1E2D0E0219749F1C0D9BCD9BED900E090
:1026600010E01092A0098091A10987FFFCCF609132
:10267000A00970E01092A0098091A10987FFFCCF0A
:102680008091A009782BC8019AD9A7D90E5F1F4F56
:10269000011581E0180729F7C701B60195D99DD921
:1026A0008FEFD81AE80AF80AD5CF80E18093650643
:1026B000E091AD2FF091AE2F8781863019F490E133
:1026C0009093932C9681963049F420E12093922C9C
:1026D000853059F483E18093932C02C08530D1F387
:1026E000953019F483E18093922C8091010480FD50
:1026F000FCCF82E080930304DF91CF911F910F9173
:10270000FF90EF90DF90CF900895CF92DF92EF92FD
:10271000FF920F931F934115E0E25E07610571057B
:1027200008F06BC06901E12CF12C00E010E220E020
:1027300030E0041B150B260B370BC016D106E20642
:10274000F30610F49701860120E12093660626E047
:102750002093A0092091A10927FFFCCF2091A00977
:1027600020E120936506000000002093660622E029
:102770002093A0092091A10927FFFCCF2091A00957
:102780005093A0092091A10927FFFCCF2091A00917
:102790004093A0092091A10927FFFCCF2091A00917
:1027A000109212012AE834E220931C0130931D019B
:1027B000009314011093150120E1209322018093CE
:1027C0002801909329010093240110932501809101
:1027D00010018068809310018091200180688093AF
:1027E00020018091100187FDFCCF80E380931101CF
:1027F0008093210180E18093650681E01F910F9114
:10280000FF90EF90DF90CF900895CF92DF92EF92FC
:10281000FF920F931F934115E0E25E07610571057A
:1028200008F05DC06901E12CF12C00E010E220E02D
:1028300030E0041B150B260B370BC016D106E20641
:10284000F30610F49701860120E12093660623E049
:102850002093A0092091A10927FFFCCF2091A00976
:102860005093A0092091A10927FFFCCF2091A00936
:102870004093A0092091A10927FFFCCF2091A00936
:1028800021E02093120180931C0190931D0100937D
:10289000140110931501109222018AE894E28093AA
:1028A0002801909329010093240110932501809120
:1028B00010018068809310018091200180688093CE
:1028C00020018091100187FDFCCF80E380931101EE
:1028D0008093210180E18093650681E001C080E062
:1028E0001F910F91FF90EF90DF90CF90089580910E
:1028F000CF0187FDFCCF0895FADF8091CF0181FFE2
:102900000BC086E38093CA01EBECF1E021E030E0FC
:1029100088ED90E084BF20830895EF92FF920F939B
:102920001F93CF93DF931F921F92CDB7DEB77C0129
:102930008A011092C20169837A83D9DF6981A62F47
:102940007A81B72FC701800F911F26E048ED50E034
:1029500061E070E0EBECF1E0E816F90689F0E09256
:10296000C0013F2D3F713093C1012093CA0144BF84
:1029700060833091C4013D933FEFE31AF30AECCF3B
:10298000C8010F900F90DF91CF911F910F91FF9091
:10299000EF9008952F923F924F925F926F927F92A5
:1029A0008F929F92AF92BF92CF92DF92EF92FF925F
:1029B0000F931F93CF93DF9300D0CDB7DEB76A019B
:1029C000282F2F711C01221A310829836A837B83E7
:1029D00093DF8DDF83E38093CA011092C1011092CF
:1029E000C2016A81E62E7B81F72E860185E3582E8F
:1029F00098ED892E912C66246394712C3BECA32EC8
:102A0000BB24B39443E3442E29810115110509F138
:102A10002093C001F70181917F018093C40101508F
:102A2000110919F02F5F203281F72092C001832D08
:102A30008F718093C1015092CA01C401F50184BF16
:102A4000608290E2290E311C52DF4092CA0120E0E0
:102A5000DCCFC6012396CDBFDEBFDF91CF911F91A2
:102A60000F91FF90EF90DF90CF90BF90AF909F902D
:102A70008F907F906F905F904F903F902F90089530
:102A80001F93CF93DF93CDB7DEB7A097CDBFDEBF47
:102A9000863009F4F2C0D8F4833009F472C030F4FF
:102AA000813061F1823009F440C000C1843009F402
:102AB0008DC0853009F0FAC0E091A12FF091A22FCE
:102AC000CE01019619958091A72F41E0ABC08930C6
:102AD00009F4D7C040F4873009F4D1C0883009F038
:102AE000E5C0D7DCE3C08B3009F4D6C008F4D2C00F
:102AF0008C3009F0DBC08EEC93E2D0C010E0809106
:102B0000A72F181750F444DBE1E0F0E0EC0FFD1FB5
:102B1000E10FF11D80831F5FF2CF8091A92F8530D7
:102B200009F098C080EE898395C011E08091A72FAD
:102B3000873009F010E0E091A12FF091A22FCE0193
:102B4000019619954091A72F31E0141708F082C023
:102B50003323A9F0812F90E0E1E0F0E0EC0FFD1FBE
:102B6000E80FF91F208131E02F3F09F030E0E1E06C
:102B7000F0E0EC0FFD1FE80FF91F2F5F20831F5FB0
:102B8000E4CFE091A12FF091A22FCE0101961995EB
:102B90008091A72F41E0815008F45CC04423D9F311
:102BA000282F30E0E1E0F0E0EC0FFD1FE20FF31F13
:102BB000908141E09F3F09F040E0E1E0F0E0EC0F60
:102BC000FD1FE20FF31F9F5F9083E5CF11E080911F
:102BD000A72F873009F010E0E091A12FF091A22FEC
:102BE000CE01019619954091A72F31E0141790F569
:102BF0003323A1F0812F90E0E1E0F0E0EC0FFD1F26
:102C0000E80FF91F208131E0211130E0E1E0F0E030
:102C1000EC0FFD1FE80FF91F215020831F5FE6CF47
:102C2000411103C08150E0F715C0282F30E0E1E0EA
:102C3000F0E0EC0FFD1FE20FF31F908141E09111D6
:102C400040E0E1E0F0E0EC0FFD1FE20FF31F9150D8
:102C50009083E8CFE091A32FF091A42FCE010196AD
:102C60001995E091AA2FF091AB2F4091A72FBE01AB
:102C70006F5F7F4F83E1199519C0BFD317C0AEDCDA
:102C800015C080910008813061F480918C088330F8
:102C900041F40AC0B9D20AC088EC93E20E948724AA
:102CA00005C00E94152602C00E943A26A096CDBFFC
:102CB000DEBFDF91CF911F910895E0E0F6E080E65E
:102CC000828388E1868B858B0895CF93C091080617
:102CD000C095C6FF12C080918C248A3050F08A3093
:102CE000E1F4E091AD2FF091AE2F8181C9DE8091AA
:102CF0008C248F5F80938C2410C08C2F807669F495
:102D000080918C2481508A3030F4E091AD2FF09185
:102D1000AE2F8081B5DE10928C24C5FF12C0809149
:102D20008B248A3050F08A30D9F4E091AD2FF091A5
:102D3000AE2F8381A5DE80918B248F5F80938B24BF
:102D40000FC0C07669F480918B2481508A3030F4B2
:102D5000E091AD2FF091AE2F828192DE10928B2404
:102D6000CF9108959B01AC016DE086E798E09FC488
:102D700020E030E090E0F901E80FF91FE455F04D54
:102D80006383245F3F4F20363105A9F708950F93E1
:102D90001F939B01E091AD2FF091AE2FE80FF11D35
:102DA0008A0140816DE086E798E042D41F910F913F
:102DB00008950F931F93CF93DF931F92CDB7DEB784
:102DC000082FAB019E012F5F3F4F6DE086E798E033
:102DD00047D4182F882319F06981802FC9DF812FEC
:102DE0000F90DF91CF911F910F9108950895EF9269
:102DF000FF920F931F93CF937B01C42F2EB13FB14E
:102E00000091080410910904022B132B682F83E012
:102E100090E20E94526E6C2F83E090E20E94526E0C
:102E2000612F83E090E20E94526E602F83E090E277
:102E30000E94526E6C2F70E0C701CF911F910F91CD
:102E4000FF90EF90B5C408953F924F925F926F92BA
:102E50007F928F929F92AF92BF92CF92DF92EF922A
:102E6000FF920F931F93CF93DF937C01E901C090F2
:102E70000020D0900120960122503843C901A0E0E3
:102E8000B0E0481759076A077B0708F05CC0E2E02A
:102E9000CE1AE0E4DE0A2A013B014C0E5D1E611CE5
:102EA000711C481659066A067B0648F0241B350B30
:102EB0008E01021B130BE9013324339403C000E09D
:102EC00010E0312C4601A12CB12C481559056A059A
:102ED0007B0510F5CA018E5F9F4B2A013B014C0E0A
:102EE0005D1E611C711C481459046A047B0428F49B
:102EF000AE01BC01C70111DA18C0C41AD50AA60177
:102F0000BC01C7010ADAAE014C195D0962E974E23D
:102F1000C7018C0D9D1D07C04C195D09BA016E5685
:102F20007B4DAE01C7010E947A70311002C081E072
:102F30000BC001501109D8F3F801EC0FFD1FEE0D85
:102F4000FF1D1082F6CF80E0DF91CF911F910F918E
:102F5000FF90EF90DF90CF90BF90AF909F908F90B9
:102F60007F906F905F904F903F90089520918E24B6
:102F700030918F2480E098E0821B930BE2E9F4E229
:102F80009F01225934422817390710F41192F8CFC3
:102F900082E994E2809390249093912480E098E0D9
:102FA00080938E2490938F2482E090E4809300207D
:102FB0009093012042E050E060E070E480E090E215
:102FC000FAD9E091AD2FF091AE2F87818A3019F4B4
:102FD00080E18093932C86818A3019F480E180937C
:102FE000922C089580918E2490918F249058209156
:102FF000002030910120821B930B089520E030E0E7
:10300000F901E455F04D8783245F3F4F20363105A9
:10301000B9F7813049F018F0823059F008951092D4
:103020008D2486EF96E109C080938D248DE798E189
:1030300004C010928D2487EF96E18093AA2F90937D
:10304000AB2F08950F931F93CF93DF931F92CDB7AC
:10305000DEB7E091AD2FF091AE2F8481CFDF82E912
:1030600094E2809390249093912400E018E00093E0
:103070008E2410938F2441E050E0BE016F5F7F4F9C
:1030800080E090E04ADCE0919024F0919124DF010F
:10309000C8011D920197E9F78981882341F042E038
:1030A00050E060E070E480E090E237D917C082E041
:1030B00090E4809300209093012042E050E060E093
:1030C00070E480E090E277D981E0898341E050E0CC
:1030D000BE016F5F7F4F80E090E05CDCE091AA2F43
:1030E000F091AB2F40E060E070E08FEF19950F900A
:1030F000DF91CF911F910F9108950F931F93CF935D
:10310000DF93AEB1BFB1C0910804D0910904209102
:103110008E2430918F24E42FF0E08F010C5F1F4F3D
:103120002017310758F1CA2BDB2B245031092E1BF5
:103130003F0B20938E2430938F24A0919024B09144
:1031400091248C9311964C9311971296DC931297BD
:10315000CD01049680939024909391241396CC9360
:10316000DB01EC01415018F02D912993FBCFE80FC2
:10317000F91FE0939024F093912412C080E03EDF89
:10318000E091AD2FF091AE2F87818A3019F481E163
:103190008093932C86818A3019F481E18093922C5C
:1031A000DF91CF911F910F9108951F93CF93DF93DC
:1031B0001F92CDB7DEB79E012F5F3F4FAC0163E09A
:1031C00083E29AE04DD2182F882311F0898116DF0F
:1031D000812F0F90DF91CF911F9108950F931F932F
:1031E000E091AD2FF091AE2F8B019C01448163E003
:1031F00083E29AE01DD21F910F9108959B01AC01CB
:1032000063E083E29AE053C2EF92FF920F931F9321
:10321000CF93DF9380918E2490918F24811528E0A5
:10322000920708F078C00091002010910120C0E0C2
:10323000D0E8C01BD10BE12C28E0F22EA701481BDF
:10324000590BC417D50760F1B80182E994E2B3D8ED
:1032500020918E2430918F24809100209091012024
:10326000985F821B930B8093002090930120E21AB9
:10327000F30AE2E9F4E2CF01825994428E159F05E8
:1032800010F41192F8CF82E994E280939024909305
:10329000912480E098E080938E2490938F242EC018
:1032A0002097C9F1AE01B80182E994E284D8A8015F
:1032B0005857BE016E567B4D82E994E20E9483709E
:1032C00080919024909191248C1B9D0B809390244D
:1032D0009093912480918E2490918F248C0F9D1F28
:1032E00080938E2490938F248091002090910120D0
:1032F000C80FD91FC0930020D093012042E050E0B6
:1033000060E070E480E090E2DF91CF911F910F9137
:10331000FF90EF9050C8DF91CF911F910F91FF90D8
:10332000EF90089580918D2481116ECF089543E62A
:1033300050E06CEA7FE281E090E0EFCA43E650E0C3
:103340006CEA7FE281E090E025CB0F931F93CF934F
:10335000DF93CFEFC80FC83008F047C0D82F0E94C6
:1033600089258091AC2FC81779F138D9C093AC2F3B
:103370008CE0C89F900111242155304D2093AD2F32
:103380003093AE2F86D8E091AD2FF091AE2F85818E
:103390000E944110E091AD2FF091AE2F84812EDE7E
:1033A00001E010E00C5A1F426091AC2FC801845517
:1033B000904D0E9406776091AD2F7091AE2FC8019D
:1033C0008355904D0E940F778FE18D0FE091AD2FC7
:1033D000F091AE2F9781943011F48093932C9681C5
:1033E000943029F48093922C02C080E001C081E0E7
:1033F000DF91CF911F910F9108958091AC2F99E0AB
:103400004CE0915099F0282F30E02F5F3F4F27700C
:103410003327822F429FF001439FF00D1124E45582
:10342000F04D2085222369F38F5F8FCF0895FC0133
:103430009091AC2F9F5C908311820895CF93FC01F3
:10344000C081818181110CC0BF01E091AA2FF09150
:10345000AB2F41E082E1199580ED8C0FCF9175CFB4
:1034600080E0CF91089588E18093010608958091CE
:10347000922C823191F030F48031B9F050F48823ED
:10348000A9F132C0833169F090EE980F983088F03E
:103490002BC088E08093050627C088E0809307064C
:1034A00023C08091040683FF12C088E08093060643
:1034B0001BC09091942C9F5F913019F09093942CA5
:1034C00015C01092942C9091040693FD04C088E0DE
:1034D000809305060BC098E090930606803221F099
:1034E00081508093922C02C01092922C8091932C48
:1034F000823191F030F48031C1F050F48823A9F189
:1035000032C0833169F090EE980F983088F02BC06C
:1035100080E18093050627C080E18093070623C0E1
:103520008091040684FF12C080E1809306061BC0D0
:103530009091952C9F5F913019F09093952C089560
:103540001092952C9091040694FD04C080E1809324
:103550000506089590E190930606803221F081508F
:103560008093932C08951092932C08959B01AC01A5
:103570006BE086E89AE09BC020E030E0982F9071E5
:103580008870992321F0F901E455F04D6287882372
:1035900021F0F901E455F04D6187245F3F4F20365B
:1035A000310579F7992329F090E19093060610925E
:1035B000932C882329F088E0809306061092922CA1
:1035C00008950F931F939B018A01803131F4E0919C
:1035D000AD2FF091AE2F478107C0883049F4E091BC
:1035E000AD2FF091AE2F46816BE086E89AE020D0B7
:1035F0001F910F9108950F931F93CF93DF931F9205
:10360000CDB7DEB7082FAB019E012F5F3F4F6BE0B8
:1036100086E89AE025D0182F882319F06981802F39
:10362000ABDF812F0F90DF91CF911F910F91089504
:103630000F931F93FC01662379F0949161509413CA
:1036400009C0BF016F5F7F4FA801C9010E945E7072
:1036500081E003C0B196EFCF80E01F910F910895F4
:10366000CF92DF92EF92FF921F93CF93DF93EC0103
:103670007A016901162F112389F0BE016F5F7F4F18
:10368000C7010E9455701150892B31F4FE01C4917D
:10369000F601C08381E003C0A196EDCF80E0DF9109
:1036A000CF911F91FF90EF90DF90CF900895CF932F
:1036B0000196CCE26623C9F0FC01DA01AD017491F8
:1036C000772341F021153105A1F07D9331962150EA
:1036D0003109F4CF623030F02115310551F04F5FE0
:1036E0005F4FCC9361508196E5CF232B11F0FA0107
:1036F0001082CF91089580912002806880932002EB
:103700008091230280FFFCCF81E080932302A0916F
:103710001002B0911102AE5BB109B7FF02C0A0E088
:10372000B0E020E038EB4BE050E00E94D86FE09131
:10373000AD2FF091AE2F61157105844F9140A8F423
:103740008781873019F480E18093932C86818730BC
:1037500019F480E18093922C8091A72F882389F01F
:10376000E091992FF0919A2F19948781873019F45D
:1037700081E18093932C8681873019F481E18093D5
:10378000922C0895BC0183E090E20C94046ECF93D8
:10379000DF93FC016491EC012196662331F083E014
:1037A00090E20E94526ECE01F4CFDF91CF91089546
:1037B000AB01BC0183E090E20C942E6E80E280931A
:1037C00062060895CF93DF938091962C823031F575
:1037D00083E090E20E94B76E0E94866983E090E2E7
:1037E0000E94D36EEC0197FD19C0E091AD2FF091CE
:1037F000AE2F8781833019F483E18093932C8681E7
:10380000833019F483E18093922C8C2FA2D68111FE
:1038100005C08C2FDF91CF910C94A724DF91CF911D
:1038200008958091962C813079F028F08230D9F07B
:10383000833011F12EC08091680685FF2AC08FE089
:103840008093022081E00CC08091022081508093FF
:10385000022081111EC00E94F20F0E94316D82E091
:103860008093962C16C08091680685FD12C08FE06B
:103870008093022083E0F4CF8091022081508093D6
:103880000220811106C00E94F66C0E942010109246
:10389000962C8091962C823019F4ACD70C9451253B
:1038A0000895E091AD2FF091AE2F8781823019F409
:1038B00081E18093932C8681823019F481E1809399
:1038C000922C0895E091AD2FF091AE2F8781823038
:1038D00019F480E18093932C8681823019F480E181
:1038E0008093922C089583E090E20C94DF6D83E046
:1038F00090E20C94266F27E83DE03F932F9321E858
:103900003DE03F932F932AE73DE03F932F9323E73A
:103910003DE03F932F9323ED3CE03F932F9322E034
:103920002F931F929F938F930E94E3708DB79EB742
:103930000E968DBF9EBF85E6089560E072E00E94FE
:10394000811085E60895FB0120812F3349F4218100
:10395000211106C060E072E00E94C01085E6089563
:10396000CB010E949210882371F0E091AD2FF0916D
:10397000AE2FCF01875A9F4265818F5F9F4F0E9474
:10398000067784E608958AEC0895EF92FF920F93EC
:103990001F93CF93DF93CDB7DEB7A097CDBFDEBF28
:1039A0007C010091A72F10E00115110591F48BEC1B
:1039B0009CE09F938F9382E08F931F92FF92EF92F0
:1039C0000E94E3700F900F900F900F900F900F9048
:1039D00010C0E091A12FF091A22FCE010196199570
:1039E0009801AE014F5F5F4F60E072E0C7010E9437
:1039F000E41085E6A096CDBFDEBFDF91CF911F9189
:103A00000F91FF90EF900895DF92EF92FF920F9346
:103A10001F93CF93DF93CDB7DEB7A097CDBFDEBFA7
:103A20007B010091A72F10E064EC7CE0C7010E94AD
:103A30005570892BC1F4D12CED2CF12CE016F10638
:103A400058F40E94C810E1E0F0E0EC0FFD1FEE0D0D
:103A5000FF1D8083D394F0CF8091A92F853069F426
:103A600080EE89830AC0A70160E270E0CE01019672
:103A70000E941E1180179107A1F4E091A32FF091ED
:103A8000A42FCE0101961995E091AA2FF091AB2FAA
:103A90004091A72FBE016F5F7F4F83E1199584E6A8
:103AA00001C08AECA096CDBFDEBFDF91CF911F9100
:103AB0000F91FF90EF90DF900895FC018091A82F67
:103AC000882311F081E301C080E38083118285E6C1
:103AD0000895FB012181211127C02081213321F488
:103AE00081E08093A82F04C0203321F41092A82FE6
:103AF00084E608952F33C1F41F9220E32F931F9281
:103B000021E32F932EEB3CE03F932F9322E02F9362
:103B10001F929F938F930E94E3708DB79EB70A9672
:103B20008DBF9EBF85E608958AEC089585E893E1F0
:103B3000DFD48EE6089585E094E1F5D48EE608950D
:103B4000E0ECF4E081818E7F81830E94F66C0E941C
:103B5000E60F84E60895E0ECF4E081818E7F8183B6
:103B60000E94F66C0E94EC0F84E60895E1E9FFE202
:103B700025892F9324892F932BEB3CE03F932F93A0
:103B800022E02F931F929F938F930E94E3708DB733
:103B90009EB708968DBF9EBF85E608952091A72FFA
:103BA0001F922F9328EB3CE03F932F9322E02F931B
:103BB0001F929F938F930E94E3708DB79EB70896D4
:103BC0008DBF9EBF85E6089540E052E0BC0180E0D5
:103BD000DED885E60895FB0120812F3341F4218151
:103BE000211105C060E072E0BDD885E6089580E04F
:103BF000E0D8882319F0A2DB84E608958AEC0895C2
:103C000040E052E0BC0181E0C2D885E60895FB01A6
:103C100020812F3341F42181211105C060E072E041
:103C2000A1D885E6089581E0C4D8882319F086DB01
:103C300084E608958AEC089540E052E0BC0182E0F9
:103C4000A6D885E60895FB0120812F3341F4218118
:103C5000211105C060E072E085D885E6089582E014
:103C6000A8D8882319F06ADB84E608958AEC0895C1
:103C700040E052E0BC0183E08AD885E60895FB016C
:103C800020812F3341F42181211105C060E072E0D1
:103C900069D885E6089583E08CD8882319F04EDB37
:103CA00084E608958AEC089540E052E0BC0180E18A
:103CB00088DC85E60895FB0120812F3341F42181C2
:103CC000211105C060E072E051DC85E6089580E1D5
:103CD00092DC882319F032DB84E608958AEC08959B
:103CE00040E052E0BC0188E06CDC85E60895FB0111
:103CF00020812F3341F42181211105C060E072E061
:103D000035DC85E6089588E076DC882319F016DB3B
:103D100084E608958AEC089560E072E05FDA85E653
:103D20000895FB0120812F3341F42181211105C029
:103D300060E072E063DA85E60895CB0136DA882325
:103D400019F0FCDA84E608958AEC0895CF93DF93A6
:103D5000EC0148D9813028E0920718F09C013850D6
:103D600002C020E030E03F932F939F938F9328E988
:103D70003CE03F932F9382E08F931F92DF93CF938A
:103D80000E94E3708DB79EB70A968DBF9EBF85E6F1
:103D9000DF91CF91089584E297E1C5D38EE608952F
:103DA00033DA84E60895E2D884E6089560E072E0AC
:103DB0003EDB85E60895CB0141DB811102C08AEC30
:103DC000089584E608950E94BE1284E608950E9434
:103DD000EE1284E608950E94491284E608958091C7
:103DE000680680FD02C089E7089588E70895DF929C
:103DF000EF92FF920F931F93CF93DF93EC010FEF9E
:103E000011E08AECE82E8EE0F82E9CE2D92EB70164
:103E100089EE93E20E945570892BD1F001151105AE
:103E2000B9F0DE01F7012491ED012196C801019757
:103E3000222341F00130110529F02C93DE01319647
:103E40008C01F1CFDC928C0188E1E80EF11CDFCF10
:103E50002197188285E6DF91CF911F910F91FF90F6
:103E6000EF90DF900895FC012091200220682093BC
:103E700020028091230280FFFCCF81E08093230207
:103E8000A0911002B0911102AE5BB109B7FF02C060
:103E9000A0E0B0E020E038EB4BE050E00E94D86FAB
:103EA000AA27BB279F938F9321E93CE03F932F9351
:103EB00082E08F931F92FF93EF930E94E3708DB780
:103EC0009EB708968DBF9EBF85E608952EB13FB17F
:103ED0004091080450910904242B352B3F932F93D4
:103EE0002BE83CE03F932F9322E02F931F929F9368
:103EF0008F930E94E3708DB79EB708968DBF9EBFCB
:103F000085E608950F931F93CF93DF931F921F921F
:103F1000CDB7DEB78B01E091AD2FF091AE2F85814B
:103F20008B3009F06FC0E091992FF0919A2F19957D
:103F300081E080931B2D60E270E0C8010E949B70BD
:103F40000097F9F4F80101900020E9F73197E01BA0
:103F5000F10BE0FD59C0F695E795E130F10539F434
:103F600087E090E080938F2F9093902F37C053E09D
:103F7000EE0FFF1F5A95E1F7E0938F2FF093902FEC
:103F80002DC098012C5F3F4F82179307E9F5A801D8
:103F900062E070E0CE0101960E941E11898190E0DE
:103FA000982F88272A81820F911D80938F2F9093BD
:103FB000902F0B5F1F4FF80101900020E9F7319718
:103FC000E01BF10BE0FD20C0F695E79533E0EE0F26
:103FD000FF1F3A95E1F7E817F907B0F060918F2FCE
:103FE0007091902F695F7F4F83E0769567958A95F2
:103FF000E1F7A8018DE89EE20E941E110E94F12EB9
:104000008FEF03C089EC01C08AEC0F900F90DF9115
:10401000CF911F910F910895EF92FF920F931F93ED
:10402000CF93DF931F921F92CDB7DEB78B01E09144
:10403000AD2FF091AE2F85818B3009F080C0E091DB
:10404000992FF0919A2F199582E080931B2D60E2B1
:1040500070E0C8010E949B707C01892B31F5F8014A
:1040600001900020E9F73197E01BF10BE0FD69C0FA
:10407000F695E795E130F10539F487E090E080931B
:104080008F2F9093902F47C063E0EE0FFF1F6A952C
:10409000E1F7CF0169E070E00E94C46FE81BF90B03
:1040A000E0938F2FF093902F36C0C8010496E81646
:1040B000F90609F046C0A80162E070E0CE01019661
:1040C0000E941E11298130E0322F22278A81280F79
:1040D000311D20938F2F3093902F2730310529F0F9
:1040E000C90187709927892B61F587010F5F1F4FE1
:1040F000F80101900020E9F73197E01BF10BE0FD9A
:1041000020C0F695E79543E0EE0FFF1F4A95E1F7D3
:10411000E217F307B0F060918F2F7091902F695FD5
:104120007F4F83E0769567958A95E1F7A8018DE842
:104130009EE20E941E110E94F12E8FEF03C089ECB7
:1041400001C08AEC0F900F90DF91CF911F910F91DA
:10415000FF90EF900895E091AD2FF091AE2F858103
:104160008B30A1F4E091992FF0919A2F199585E069
:1041700080931B2D0E9447500E94F12E81E590E50F
:104180008093A62C9093A72C8FEF089589EC089527
:104190008BE00E944110E091992FF0919A2F199590
:1041A00088E080931B2D0E9447500E94F12E81E5EC
:1041B00090E58093A62C9093A72C8FEF0895E09123
:1041C000AD2FF091AE2F85818B30A1F4E091992F26
:1041D000F0919A2F199583E080931B2D0E944750F0
:1041E0000E94F12E81E590E58093A62C9093A72C58
:1041F0008FEF089589EC0895E091AD2FF091AE2FE7
:1042000085818B30A1F4E091992FF0919A2F199527
:1042100086E080931B2D0E9447500E94F12E81E57D
:1042200090E58093A62C9093A72C8FEF089589ECAE
:104230000895E091AD2FF091AE2F4085518564E651
:10424000649F9001659F300D11243F932F9325E8C3
:104250003CE03F932F9322E02F931F929F938F93E5
:104260000E94E3708DB79EB708968DBF9EBF85E60E
:104270000895CF93DF931F921F92CDB7DEB7FB0156
:1042800020812F33B1F42181211113C023E53CE0BB
:104290003F932F9322E02F931F929F938F930E941F
:1042A000E3700F900F900F900F900F900F9085E696
:1042B0002EC089E592E089839A83CE0101969F936F
:1042C0008F938FE49CE09F938F937F936F930E94D3
:1042D00019710F900F900F900F900F900F90892BE6
:1042E000A9F069817A816935F2E07F0778F4E0917D
:1042F000AD2FF091AE2F60877187CF01845A9F4216
:104300008F5F9F4F0E940F7784E601C08AEC0F9069
:104310000F90DF91CF910895E091AD2FF091AE2FE6
:1043200023852F9322852F932CE43CE03F932F93FA
:1043300022E02F931F929F938F930E94E3708DB77B
:104340009EB708968DBF9EBF85E60895CF93DF93F5
:104350001F921F92CDB7DEB7FB0120812F33B1F43E
:104360002181211113C02FE02F932FEF2F932BEFDB
:104370003BE03F932F9322E02F931F929F938F93C5
:104380000E94E370CDBFDEBF85E630C019821A827D
:10439000CE0101969F938F9387EF9BE09F938F931E
:1043A0007F936F930E9419710F900F900F900F9051
:1043B0000F900F90892BC9F069817A81611590E186
:1043C000790798F46093380370933903E091AD2F27
:1043D000F091AE2F62877387CF01825A9F428F5F21
:1043E0009F4F0E940F7784E601C08AEC0F900F90D8
:1043F000DF91CF910895FB0120812F33D9F42181E2
:10440000211121C01F9220E32F931F9221E32F93AC
:1044100021EF3BE03F932F9322E02F931F929F9336
:104420008F930E94E3708DB79EB70A968DBF9EBF93
:1044300085E60895213311F4F8D303C0203319F42D
:1044400019D484E608958AEC0895FC01809100084F
:10445000813021F480918C08833011F080E301C019
:1044600081E38083118285E60895E091AD2FF0917C
:10447000AE2F85818B3079F4E091992FF0919A2FAE
:10448000199584E080931B2D0E9447500E94F12EC5
:1044900081E590E50EC08A3091F4E091992FF0917A
:1044A0009A2F199581E08093F72D0E9437588CE45C
:1044B00098E58093A62C9093A72C8FEF089589EC14
:1044C00008958BE00E944110E091992FF0919A2F6E
:1044D000199587E080931B2D0E9447500E94F12E72
:1044E00081E590E58093A62C9093A72C8FEF0895FB
:1044F00021E02093A52C2093A42C2CE32093A12C25
:1045000025E030E020939F2C3093A02C1092992C22
:1045100010929A2C10929B2C10929C2C8093972C8A
:104520009093982C089527E02093A52C2CE231E05D
:1045300020939F2C3093A02C1092992C10929A2C9F
:1045400010929B2C10929C2C8093972C9093982CDB
:104550000895CF939091A52C9530E1F130F49330EC
:1045600029F140F5913068F441C1973009F4A7C0B2
:1045700008F445C0983009F4AAC0993009F433C151
:1045800035C1813041F410929D2C10929E2C1092D6
:10459000A22C83E0FBC0843011F466E08BC088312C
:1045A00009F421C18B3109F0F3C01DC18093A32C04
:1045B00084E0ECC090E04091A32C2FEF30E0241B6E
:1045C00031098217930721F485E0E0C0981739F18B
:1045D00065E169C020919D2C30919E2CA9014F5F0F
:1045E0005F4F40939D2C50939E2CF901E15FFF4C4F
:1045F00080834038510509F0CBC086E0C7C02091C8
:10460000A32C9091A42C291346C0EFE0F0E390E096
:1046100020E3EF38F207D1F22191920FF9CF4091C8
:10462000992C50919A2C60919B2C70919C2CE0912C
:10463000972CF091982C20E830E08FE090E31995CA
:10464000C82F882311F18091A42C8F5F8093A42C14
:104650008091992C90919A2CA0919B2CB0919C2C9C
:1046600080589F4FAF4FBF4F8093992C90939A2CB7
:10467000A0939B2CB0939C2C66E083E090E20E9478
:10468000526E82E08093A52CB2C068E183E090E294
:104690000E94526E0EC030E0892F90E001972817DB
:1046A000390739F466E083E090E20E94526E82E0BE
:1046B0006DC068E183E090E20E94526E94C0853143
:1046C00019F41092A42C09C08B3109F48CC08831E4
:1046D00009F463CF863009F05DC08091A42C8F5F10
:1046E0008093A42C4091992C50919A2C60919B2CF2
:1046F00070919C2CE091972CF091982C20E830E060
:104700008FE090E31995C82F8823D1F161E083E011
:1047100090E20E94526E6091A42C83E090E20E948D
:10472000526E6091A42C609583E090E20E94526EDC
:1047300060E870E08FE090E33BD8EFE0F0E360E00A
:1047400080E3EF38F80719F08191680FF9CF83E023
:1047500090E20E94526E8091992C90919A2CA09197
:104760009B2CB0919C2C80589F4FAF4FBF4F809394
:10477000992C90939A2CA0939B2CB0939C2C37C08F
:1047800064E083E090E20E94526E89E08093A52C61
:10479000C1E02DC08531E1F761E083E090E20E9445
:1047A000526E6091A42C83E090E20E94526E609160
:1047B000A42C609583E090E20E94526E60E870E065
:1047C0008FE090E30E94D81BEFE0F0E360E020E38D
:1047D000EF38F20719F08191680FF9CF83E090E28A
:1047E0000E94526ED5CF1092A52CD2CFC0E08C2F54
:1047F000CF9108958091A52C813019F0873029F14F
:10480000089580919F2C9091A02C9C0121503109FA
:1048100020939F2C3093A02C892B31F58091A12CD3
:104820009FEF980F9093A12C882331F065E183E0EE
:1048300090E20E94526E02C01092A52C85E090E09A
:1048400080939F2C9093A02C089580919F2C909101
:10485000A02C9C012150310920939F2C3093A02C37
:10486000892B11F41092A52C0895E1EAFDE020E0D7
:1048700030E09491981309C041E2429FC001439FE8
:10488000900D11248E55924F08952F5F3F4FB19692
:104890002930310571F780E090E00895262FBA01A4
:1048A0002F3311F4469607C02D3311F4449611C0EE
:1048B00021110CC04096FC01259134912115310540
:1048C00021F18FE090E3F90119950DC02032E9F450
:1048D0004296FC012591349121153105B1F08FE00C
:1048E00090E3F90119958F3F89F491E09093AA2CF8
:1048F0002EB13FB14091080450910904242B352B6F
:104900002093A82C3093A92C089589EC08950F9337
:104910001F93CF93DF938C01CAECDEE0BE01C80188
:104920000E945570892B49F440E050E060E0CE01D0
:10493000DF91CF911F910F91B1CF689682E1C23A7A
:10494000D80761F7DF91CF911F910F910895EF92F2
:10495000FF921F93CF93DF93982F9F7D91549A31AD
:1049600060F090ED980F9A3040F08F3531F0982F2D
:104970009D7F9D3311F08032D1F49FE9980F9A31D9
:1049800008F480522091AB2C3091AC2C2F3F91E059
:10499000390708F07FC0A9014F5F5F4F4093AB2CF0
:1049A0005093AC2CF901E15FFF4C808373C08D30D4
:1049B00009F040C0E091AB2CF091AC2CE15FFF4CD2
:1049C00010821092AB2C1092AC2C8091AA2C8111E9
:1049D00061C080910F30982F9F7D09F440C08D7F7A
:1049E0008D33E9F1EFE0F0E37F011191112331F014
:1049F0001F3321F01D3311F01032B1F7F70110828F
:104A0000CAECDEE0BE018FE090E30E945570892B76
:104A100059F410920F30A7014F5F5F4F612FCE0105
:104A20003DDF8F3FB9F124C06896F2E1C23ADF075B
:104A300049F715C0883061F48091AB2C9091AC2C73
:104A4000009741F101978093AB2C9093AC2C22C03E
:104A50008B3101F51092AB2C1092AC2C1BC088EC62
:104A600004DF0E94C71B8EE99DE00E94C71B12C095
:104A7000FCDE0E94C71B8EE99DE00E94C71B80914F
:104A80000F30882339F08FE090E30E94C21B8BE93E
:104A90009DE0EBCF81E0DF91CF911F91FF90EF90F0
:104AA00008958091AA2C882399F1E091AD2FF0917F
:104AB000AE2F208531852115310551F18EB19FB181
:104AC0004091080450910904842B952B4091A82C07
:104AD0005091A92C841B950B64E670E00E94C46F72
:104AE00062177307A8F01092AA2C8BECBEDE0E940E
:104AF000C71B88E99DE00E94C71BE091A62CF0919E
:104B0000A72C309729F019951092A62C1092A72C5B
:104B100008958091AA2C8823A9F01092AA2C8BECDE
:104B2000A4DE0E94C71B88E99DE00E94C71BE0919C
:104B3000A62CF091A72C309729F019951092A62C4D
:104B40001092A72C0895CF93DF939091AA2C9923CC
:104B5000A9F0EB011092AA2C88DE0E94C71B85E900
:104B60009DE00E94C71B209749F0CE010E94C21B06
:104B700082E99DE0DF91CF910C94C71BDF91CF912B
:104B80000895EF92FF920F931F93CF937C019B01A7
:104B9000613081E0780710F020E031E08B01021BEA
:104BA000130BA70160E072E08FE090E30E94E41035
:104BB0008FE090E30E94C21BC1E0013081E0180742
:104BC000B0F01A956C2F70E0762F6627A701460F7C
:104BD000571F20E032E060E072E08FE090E30E9437
:104BE000E4108FE090E30E94C21BCF5FE6CF011577
:104BF000110591F0EC2FF0E0FE2FEE27A7014E0FEC
:104C00005F1F980160E072E08FE090E30E94E41083
:104C10008FE090E30E94C21B8FE89DE0CF911F912F
:104C20000F91FF90EF900C94C71B8091000881308A
:104C300029F480918C08833009F408958091AF2C79
:104C4000811117C081E08093000893E090938C0855
:104C50008093AD2C1092AE2C8EB19FB120910804A0
:104C600030910904822B932B8093B42C9093B52C14
:104C70000895089510928C0810920008EDEAFCE265
:104C80001082118208959091AD2C9923F1F08091BA
:104C9000AE2C811115C02091AD2C2223B9F02EB17C
:104CA0003FB14091080450910904242B352B4091C9
:104CB000B42C5091B52C241B350B2634310530F023
:104CC00081E08093AE2C892F089581E00895CF93E1
:104CD000DF931F92CDB7DEB78091AF2C8823D1F040
:104CE0002EB13FB14091080450910904242B352B7B
:104CF0004091B22C5091B32C241B350B4091B02C19
:104D00005091B12C2417350728F01092AF2C8983CD
:104D10008CDF89810F90DF91CF910895E091AD2FC5
:104D2000F091AE2F82879387809338039093390355
:104D30000895E091AD2FF091AE2F82859385409636
:104D40008287938780933803909339038285938574
:104D50000895E091AD2FF091AE2F80E991E0828728
:104D6000938780933803909339030895A0E2B6E0C7
:104D700081E015968C9315972FE032E328B939B965
:104D80002FE832E32AB93BB910B813B812B816B8F5
:104D900017B811B8E0E0F9E010A211A22FEF30E04F
:104DA00026A337A32FEF3FEF20A731A7808398E8F2
:104DB000938390E1948793E097831C968C931C9740
:104DC00082E01A968C9308951F920F920FB60F925D
:104DD000112408B60F9218BE0BB60F921BBE8F930C
:104DE0009F93EF93FF93E0E0F9E013828FE790E069
:104DF00086AB97AB81E190E080AF91AFE0E0FAE065
:104E000010A211A28FEF9FEF86A397A389E8838357
:104E1000168281E084878EE0808310922A06FF91BB
:104E2000EF919F918F910F900BBE0F9008BE0F9046
:104E30000FBE0F901F9018951F920F920FB60F92F2
:104E4000112408B60F9218BE0BB60F921BBE2F93FB
:104E50003F938F939F93EF93FF932091280693B1F5
:104E6000267081E009F080E0990F892B83B982B127
:104E7000882309F464C012B883B18770873059F56C
:104E80001092000980E180930C091092030A1B9B89
:104E900003C08CEA94E002C08CE694E08093260A7A
:104EA0009093270A82E081B981E080930C0A83E025
:104EB0008093060A86B197B1877049F090B18F5FF1
:104EC000893011F09695FBCFE8B1F9B1908381E07C
:104ED0008093B62C37C093B1892F8C7099F192FBD7
:104EE000992790F981E0982781B181111BC080B189
:104EF0008695911190E8892B80B926B137B12F5F43
:104F00003F4F26B937B927703327232BD9F4E8B19F
:104F1000F9B19F012F5F3F4F28B939B9808381E0F4
:104F200081B910C081B1813069F4EAB1FBB19F0150
:104F30002F5F3F4F2AB93BB9908311B803C082B1AC
:104F4000809582B988E880930309FF91EF919F9142
:104F50008F913F912F910F900BBE0F9008BE0F9035
:104F60000FBE0F901F9018951F920F920FB60F92C1
:104F7000112408B60F9218BE0BB60F921BBE2F93CA
:104F80003F938F939F93EF93FF9381B1823008F407
:104F90009DC081B18D3008F099C0E1B1F0E0EE0F15
:104FA000FF1FEA5DFF4D0190F081E02D19948FE71E
:104FB00090E08093260A9093270A88C08E9A8EE00C
:104FC000809340088FE390E08093260A9093270A0D
:104FD00085E06FC08E9886E081B98FEF82B914B8F2
:104FE00015B8E8B1F9B1808180B970C0009B05C0E7
:104FF0008E9A82B1809582B901C08E9887E059C09F
:10500000009B02C08E9801C08E9A80B1869580B9AF
:1050100084B195B1019684B995B984B195B1877081
:105020009927892B11F488E044C024B135B186B1A9
:1050300097B128173907B1F52BC0EAB1FBB130970A
:1050400011F0808101C082B1882311F08E9A01C0D5
:105050008E9889E02EC0EAB1FBB1309751F0808183
:10506000882311F08E9801C08E9A3196EAB9FBB967
:1050700008C082B1882311F08E9801C08E9A8FEFFC
:1050800082B924B135B186B197B12817390711F427
:105090008AE00FC0E8B1F9B1CF01019688B999B99A
:1050A000818180B986E005C08E988BE002C08E9821
:1050B0008CE081B90BC01092000A1092060A10927F
:1050C00040081092410881E08093B72CFF91EF9146
:1050D0009F918F913F912F910F900BBE0F9008BE23
:1050E0000F900FBE0F901F901895CF93DF93E6EBB4
:1050F000FCE21082118286EA99E280938B2E9093D3
:105100008C2E84EE96E280938D2F90938E2FE0E488
:10511000F6E0128A84E08283C0E8D1E082E68E83E2
:10512000A0E2B6E081E016968C93169711968C93C8
:10513000119796E012969C93129751968C935197E3
:1051400032E052963C9352971A961C921A971B96ED
:105150001C921B979FE019969C9399E598832AE5EA
:1051600029839A8390E491839683A0EBB0E0129612
:105170002C911297207F12962C93129712962C91B5
:105180001297226012962C9320E321832683908B22
:105190008683358383E08183E0E0F8E083E18183E7
:1051A00021E030E026A337A320A731A7E0E8F8E00C
:1051B00014868083E0E2F3E01382118288E0828328
:1051C00091E19083A091AD2FB091AE2F1A962D91C1
:1051D0003C911B97208F318FE0E8F3E09CE39283B2
:1051E000808393838183DF91CF91C0CDA0E2B6E02D
:1051F0001A961C921A97E6EBFCE210821182E0E00C
:10520000F9E010821382178280E18487E0E0FAE0FF
:1052100010821382168281E08487E0E4F8E0108235
:10522000118216968C938E980895CF93DF93809178
:10523000B62C882309F47EC01092B62CC6B1D7B123
:10524000C730D10508F471C0AE01495F5F4F93E0EC
:10525000569547959A95E1F7E091AA2FF091AB2FDB
:105260006FE072E380E41995E091AD2FF091AE2FDD
:105270008781883019F483E18093932C868188306C
:1052800019F483E18093922CE0919F2FF091A02F4D
:10529000BE018FE092E31995EC0194FF06C0DF7E1A
:1052A0008FE892E38AB99BB902C01AB81BB820975D
:1052B000E1F1AE01495F5F4F83E0569547958A95CE
:1052C000E1F7E091AA2FF091AB2F6FE072E381E458
:1052D0001995E091AD2FF091AE2F8781893019F4A7
:1052E00083E18093932C8681893019F483E1809344
:1052F000922CC6B9D7B98FE092E388B999B91092C8
:105300006008109261088FE090E0809366089093A7
:10531000670888E090E080936A0890936B0883E2C6
:105320008093410883E081B905C01092000A109271
:10533000060A1CDD8091B72C882329F01092B72C27
:10534000DF91CF9113CDDF91CF9108951F920F92EE
:105350000FB60F92112408B60F9218BE0BB60F921B
:105360001BBE2F933F938F939F93EF93FF93E0E0A8
:10537000F9E080E484871782E0E8F3E082E0878345
:1053800089EB81838FE092E38AB99BB981E090E059
:1053900084B995B916B88EB19FB1209108043091A7
:1053A0000904822B932B8093B92C9093BA2C81E023
:1053B0008093BD2C18B817B81092B82C88E0809351
:1053C0008706FF91EF919F918F913F912F910F90C1
:1053D0000BBE0F9008BE0F900FBE0F901F90189538
:1053E000CF93DF93E0E4F6E0128A84E08283C0E8A2
:1053F000D1E082E68E83A0E2B6E081E016968C933F
:10540000169711968C93119796E012969C9312978B
:1054100051968C93519732E052963C9352971A963C
:105420001C921A971B961C921B979FE019969C93AF
:10543000199799E598832AE529839A8390E49183C3
:105440009683C0EBD0E02A81207F2A832A812260C4
:105450002A8320E321832683908B8683358393E000
:105460009183E0E0F8E093E1918321E030E026A32E
:1054700037A320A731A7E0E8F8E014869083E0E2A4
:10548000F3E01382118298E0928321E12083C0919E
:10549000AD2FD091AE2F2A853B85208F318FE0E84C
:1054A000F3E02CE3228390832383918326EA39E27D
:1054B00020938B2E30938C2E15968C93E0E0F9E0A0
:1054C0002FEF30E026A337A312A613A614A615A625
:1054D00010821682178280831092000A1092B82CD4
:1054E000EBEBFCE2108212821182DF91CF910895E2
:1054F00081E080932606BEDBE0E0F9E010821782AF
:10550000E0E0FAE010821782EBEBFCE211821282FB
:1055100010820895E0E0F9E08FEF94E086A397A36E
:1055200080E6848780E387838FEF90E086AB97AB3C
:1055300088E08093870608951F920F920FB60F920E
:10554000112408B60F9218BE0BB60F921BBE2F93F4
:105550003F934F935F938F939F93EF93FF9310929B
:10556000070A1092000A1092470910924009809190
:1055700081038E7F8093810384B195B180FF1AC02F
:10558000379B03C086B1869503C086B18695806837
:1055900086B984B195B1019684B995B98770992778
:1055A000892B41F4EAB1FBB1CF0101968AB99BB9CD
:1055B00086B1808384B195B187709927892BC9F012
:1055C000E4B1F5B186B144B155B193E0F695E795F4
:1055D0009A95E1F7E15FFD4C90E04770552728E090
:1055E00030E0241B350B02C0959587952A95E2F78C
:1055F000808381E08093BC2C1092BD2C8FEF9FEFB5
:105600008093260A9093270A1092200A1092210A6A
:105610001092060A1092070A1092030A84E08093FF
:10562000000A83E08093B82CFF91EF919F918F91B6
:105630005F914F913F912F910F900BBE0F9008BE3D
:105640000F900FBE0F901F9018951F920F920FB6DC
:105650000F92112408B60F9218BE0BB60F921BBE04
:105660008F93EF93FF93E0E8F3E081818F7C818358
:10567000E0E0FAE088E8838381E08083FF91EF91A6
:105680008F910F900BBE0F9008BE0F900FBE0F9022
:105690001F9018951F920F920FB60F92112408B603
:1056A0000F9218BE0BB60F921BBE8F939F93EF9372
:1056B000FF9380916009109260091092610993E054
:1056C00090934009813520F4813308F472C01BC0E7
:1056D0008137E8F484B195B180FF2EC086B18695FC
:1056E000806886B984B195B1019684B995B98770FF
:1056F0009927892B41F4EAB1FBB1CF0101968AB910
:105700009BB986B1808386B1869580682CC086B1AE
:105710008695806886B984B195B1019684B995B9AA
:1057200087709927892B41F4EAB1FBB1CF0101962B
:105730008AB99BB986B1808386B18695806886B91F
:1057400084B195B1019684B995B987709927892B51
:1057500041F4EAB1FBB1CF0101968AB99BB986B198
:10576000808386B1869586B984B195B1019684B956
:1057700095B987709927892B41F4EAB1FBB1CF0124
:1057800001968AB99BB986B1808386B1869586B920
:1057900084B195B1019684B995B987709927892B01
:1057A00041F4EAB1FBB1CF0101968AB99BB986B148
:1057B0008083FF91EF919F918F910F900BBE0F907F
:1057C00008BE0F900FBE0F901F9018950F931F9358
:1057D000CF93DF93CDB7DEB7DA95CDBFDEBF809133
:1057E000BD2C882309F483C08EB19FB14091080479
:1057F000509109042091B92C3091BA2C842B952B0F
:10580000821B930B20911E2030911F202F5F3F4F52
:105810002817390708F06BC01092070A1092000A87
:105820001092470910924009809181038E7F8093E6
:10583000810384B195B180FF1AC0379B03C086B144
:10584000869503C086B18695806886B984B195B186
:10585000019684B995B987709927892B41F4EAB1EB
:10586000FBB1CF0101968AB99BB986B1808384B11F
:1058700095B187709927892BC9F0E4B1F5B186B14C
:1058800044B155B113E0F695E7951A95E1F7E15F5C
:10589000FD4C90E04770552728E030E0241B350B85
:1058A00002C0959587952A95E2F7808381E08093E1
:1058B000BC2C1092BD2C2FEF3FEF2093260A309383
:1058C000270A1092200A1092210A1092060A1092BA
:1058D000070A1092030A94E09093000A93E09093D1
:1058E000B82C14B815B88093BC2C1092BD2CEFD9ED
:1058F00081116FC2C8D9882309F46BC28091BD2C75
:10590000811167C28091BB2C811105C08091BC2C94
:10591000882309F45EC28091B82C833041F48091D1
:10592000200A9091210A8532914008F452C2809158
:10593000BC2C882309F4A2C084B195B1892B09F449
:105940009DC084B195B1089718F414B815B896C0E5
:1059500044B155B1495F5F4FB3E056954795BA954D
:10596000E1F76FE072E3CE0101960E947A708FE05A
:1059700092E38AB99BB944B155B114B815B889817D
:1059800086958695898322E030E024173507B0F5A7
:10599000F901A3E0F695E795AA95E1F781E090E09B
:1059A0008C0F9D1FE80FF91F8081982F9695969573
:1059B00090838370813049F030F08230D1F486B129
:1059C0008695806804C081E015C086B1869586B949
:1059D00084B195B1019684B995B987709927892BBF
:1059E00041F4EAB1FBB1CF0101968AB99BB986B106
:1059F000808380E02E5F3F4F882339F284B195B1D8
:105A000087709927892BC9F0E4B1F5B186B144B10B
:105A100055B173E0F695E7957A95E1F7E15FFD4CB6
:105A200090E04770552728E030E0241B350B02C07A
:105A3000959587952A95E2F78083E091AD2FF091B7
:105A4000AE2F8781883019F483E18093932C86816F
:105A5000883019F483E18093922C44B155B1495FA9
:105A60005F4F63E0569547956A95E1F7E091AA2F5D
:105A7000F091AB2F6FE072E382E419951092BB2C8A
:105A80001092BC2C64B175B1E0919F2FF091A02FC2
:105A90008FE092E3199584B995B984B195B1892BBA
:105AA00009F497C189E8809381031092000A10924B
:105AB000200A1092210A2FEF3FEF2093260A3093FD
:105AC000270A8FE590E08093280A9093290A109284
:105AD000060A80E180930C0A93E09093070A1092E3
:105AE000600910926109209366093093670920EAE2
:105AF00030E0209368093093690910924609809339
:105B00004C0981E08093470981E1809380011092E4
:105B100088011092800310922906E091AD2FF09138
:105B2000AE2F8781893019F483E18093932C86818D
:105B3000893019F483E18093922C44B155B1495FC7
:105B40005F4F33E0569547953A95E1F7E091AA2FDC
:105B5000F091AB2F6FE072E383E4199504B115B1B6
:105B6000013094E0190708F024C114B815B8A80151
:105B7000495F5F4F23E0569547952A95E1F76FE01F
:105B800072E38FE892E30E947A708FE092E38AB921
:105B90009BB986B18695806886B984B195B1019626
:105BA00084B995B987709927892B39F480E192E3FC
:105BB0008AB99BB986B180930F3286B1869586B932
:105BC00084B195B1019684B995B987709927892BCD
:105BD00041F4EAB1FBB1CF0101968AB99BB986B114
:105BE000808380E041E050E0EFE8F2E3041715071E
:105BF00008F495C0908190FF2BC086B1869586B938
:105C000084B195B1019684B995B987709927892B8C
:105C100041F4AAB1BBB1CD0101968AB99BB986B155
:105C20008C9386B18695806886B984B195B10196CA
:105C300084B995B987709927892B09F063C0AAB1F7
:105C4000BBB1CD0101968AB99BB986B18C935AC07C
:105C5000882351F186B1869586B984B195B10196B4
:105C600084B995B987709927892B41F4AAB1BBB142
:105C7000CD0101968AB99BB986B18C9386B1869580
:105C800086B984B195B1019684B995B98770992781
:105C9000892B41F4AAB1BBB1CD0101968AB99BB958
:105CA00086B18C9380E02FC096B19695906896B996
:105CB00024B135B12F5F3F4F24B935B92770332751
:105CC000232B49F4AAB1BBB19D012F5F3F4F2AB9E5
:105CD0003BB996B19C9396B1969596B924B135B1DE
:105CE0002F5F3F4F24B935B927703327232BD1F6C7
:105CF000AAB1BBB19D012F5F3F4F2AB93BB996B105
:105D00009C9301C081E09081969590839A012770C1
:105D10003327232B09F431964F5F5F4F67CF8111F3
:105D200029C086B18695806886B984B195B10196FF
:105D300084B995B987709927892B41F4EAB1FBB1F1
:105D4000CF0101968AB99BB986B1808386B18695C9
:105D500086B984B195B1019684B995B987709927B0
:105D6000892B41F4EAB1FBB1CF0101968AB99BB905
:105D700086B1808384B195B187709927892BC9F04A
:105D8000E4B1F5B186B144B155B193E0F695E7952C
:105D90009A95E1F7E15FFD4C90E04770552728E0C8
:105DA00030E0241B350B02C0959587952A95E2F7C4
:105DB000808381E08093B82C8FE092E38AB99BB90D
:105DC00080E280930C098CE08093070985E58A9531
:105DD000F1F7D395CDBFDEBFDF91CF911F910F912A
:105DE000089514B815B881E08093BB2C0C94152647
:105DF0001092070A1092000A109247091092400967
:105E0000809181038E7F8093810384B195B180FF5F
:105E10001AC0379B03C086B1869503C086B18695AC
:105E2000806886B984B195B1019684B995B98770B7
:105E30009927892B41F4EAB1FBB1CF0101968AB9C8
:105E40009BB986B1808384B195B187709927892BDE
:105E5000C9F0E4B1F5B186B144B155B193E0F6951E
:105E6000E7959A95E1F7E15FFD4C90E04770552783
:105E700028E030E0241B350B02C0959587952A95C4
:105E8000E2F7808381E08093BC2C1092BD2C8FEFD1
:105E90009FEF8093260A9093270A1092200A10926F
:105EA000210A1092060A1092070A1092030A84E04F
:105EB0008093000A83E08093B82C1092B82C109243
:105EC000BC2C1092BB2C0C943A2680916009109245
:105ED00060091092610993E090934009813520F4A4
:105EE000813308F4A7C003C0813758F165C08091A1
:105EF000BE2C9091BF2C80FF0AC08091BE2C909147
:105F0000BF2C0297C0F085B18695806802C085B12C
:105F1000869585B986B197B1019686B997B987708C
:105F20009927892B41F4ECB1FDB1CF0101968CB9D1
:105F30009DB985B180838091BE2C9091BF2C029633
:105F400075C08091BE2C9091BF2C80FF1BC08091AA
:105F5000BE2C9091BF2C0297A8F085B186958068E1
:105F600085B986B197B1019686B997B98770992797
:105F7000892B41F4ECB1FDB1CF0101968CB99DB9EB
:105F800085B1808385B1869585B986B197B1019633
:105F900086B997B987709927892B41F4ECB1FDB187
:105FA000CF0101968CB99DB985B180838091BE2CBB
:105FB0009091BF2C03963AC08091BE2C9091BF2C3B
:105FC00080FF2FC08091BE2C9091BF2C0297A8F02B
:105FD00085B18695806885B986B197B1019686B9F5
:105FE00097B987709927892B41F4ECB1FDB1CF01A6
:105FF00001968CB99DB985B1808385B1869585B9A7
:1060000086B197B1019686B997B987709927892B80
:1060100041F4ECB1FDB1CF0101968CB99DB985B1C8
:1060200080838091BE2C9091BF2C04968093BE2CCF
:106030009093BF2C08951F920F920FB60F921124C8
:1060400008B60F9218BE0BB60F921BBE8F939F938C
:10605000EF93FF9384E080938506E0E0F9E01382FC
:106060008FE790E086AB97AB81E190E080933E09AB
:1060700090933F0910922B06FF91EF919F918F9182
:106080000F900BBE0F9008BE0F900FBE0F901F9089
:1060900018951F920F920FB60F92112408B60F9207
:1060A00018BE0BB60F921BBE2F933F934F935F9377
:1060B0008F939F93EF93FF932091280694B12670BE
:1060C00081E009F080E0990F892B84B983B188239E
:1060D00009F4E5C013B884B18770873009F0B5C002
:1060E00084E0809386061092000980E880930C0972
:1060F000109207091092290686B197B1877049F06E
:1061000090B18F5F893011F09695FBCFE8B1F9B16E
:10611000908386B197B18093C22C9093C32C8091C9
:10612000C22C9091C32C079708F45CC081E0809347
:10613000C62C2FE033E32CB93DB921E030E02093A9
:10614000BE2C3093BF2C16B817B815B899E89093A9
:1061500080031092000A1092200A1092210A4FEF39
:106160005FEF4093260A5093270A2FE530E02093F3
:106170002A0A30932B0A1092060A20E220930C0A76
:106180009CE09093070A1092600910926109409375
:1061900066095093670940EA50E040936A095093BA
:1061A0006B091092460920934C099093470990E19E
:1061B0009093820110928A01109281038093870349
:1061C00089EB809380038EB19FB1209108043091B8
:1061D0000904822B932B8093C42C9093C52C82E0CE
:1061E00081B963C08CE0809329068FE092E388B97F
:1061F00099B98FE892E38AB99BB910B814B813B86B
:1062000016B817B811B810922009109221098FEF13
:1062100090E080932609909327098FEF9FEF80935A
:106220002E0990932F0981E08093000988E88093DC
:10623000030980E880930C0980EC8093070982E0D1
:1062400080932C0680932B0630C094B1892F8C70DC
:1062500049F181B181111EC080B1869592FF02C0C3
:1062600090E001C090E8892B80B926B137B12F5F4B
:106270003F4F26B937B927703327232B99F4E8B15C
:10628000F9B19F012F5F3F4F28B939B9808381E071
:1062900081B908C081B1813029F411B803C083B13C
:1062A000809583B988E880930309FF91EF919F91CE
:1062B0008F915F914F913F912F910F900BBE0F9057
:1062C00008BE0F900FBE0F901F9018951F920F924F
:1062D0000FB60F92112408B60F9218BE0BB60F928C
:1062E0001BBE8F93EF93FF93E0E8F3E080818F7CF8
:1062F0008083E0E0FAE08AE8838381E0808383E0C2
:1063000081B9FF91EF918F910F900BBE0F9008BE56
:106310000F900FBE0F901F9018951F920F920FB6FF
:106320000F92112408B60F9218BE09B60F9219BE2B
:106330000BB60F921BBE2F933F934F935F936F93B8
:106340007F938F939F93AF93BF93EF93FF93E091CE
:10635000892EF0918A2E1995FF91EF91BF91AF91FF
:106360009F918F917F916F915F914F913F912F916D
:106370000F900BBE0F9009BE0F9008BE0F900FBE7E
:106380000F901F9018951F920F920FB60F92112425
:1063900008B60F9218BE0BB60F921BBE2F933F93F9
:1063A0004F935F938F939F93EF93FF931092070AFE
:1063B0001092000A1092030A1092470910924009A5
:1063C000809180038E7F809380038091BE2C90917A
:1063D000BF2C80FF15C085B18695806885B986B1D0
:1063E00097B1019686B997B987709927892B41F49F
:1063F000ECB1FDB1CF0101968CB99DB985B1808317
:1064000086B197B187709927892BC9F0E6B1F7B1AA
:1064100085B146B157B193E0F695E7959A95E1F7C6
:10642000E15FFC4C90E04770552728E030E0241BEA
:10643000350B02C0959587952A95E2F7808386B142
:1064400097B18093C02C9093C12C86B197B10497DB
:1064500018F081E08093C72C1092000A1092070A6E
:106460001092820110928A018CE38093820388E06B
:10647000809380038CE0809329068FE092E388B9B3
:1064800099B98FE892E38AB99BB910B814B813B8D8
:1064900016B817B811B810922009109221098FEF81
:1064A00090E080932609909327098FEF9FEF8093C8
:1064B0002E0990932F0981E08093000988E880934A
:1064C000030980E880930C0980EC8093070982E03F
:1064D00080932C0680932B06FF91EF919F918F91D3
:1064E0005F914F913F912F910F900BBE0F9008BE7F
:1064F0000F900FBE0F901F901895CF93DF934CE035
:1065000040938106A0E4B6E052961C92529784E034
:1065100012968C931297C0E8D1E082E68E83E0E277
:10652000F6E081E08683818396E09283818B92E01E
:10653000928B128613862FE0218729E528833AE57E
:1065400039832A8320E411962C93119716962C9365
:106550001697C0EBD0E03A81307F3A833A813260BF
:106560003A8330E311963C93119716963C93169715
:1065700050962C93509716968C93169715969C933D
:10658000159723E011962C93A0E0B8E023E1119633
:106590002C93119761E070E096966D937C9397979A
:1065A00098966D937C939997A0E8B8E01C961C92FE
:1065B0001C972C93A0E2B3E013961C9213971196AC
:1065C0001C92119728E012962C93129731E13C937C
:1065D000C091AD2FD091AE2F6A857B8558966D9373
:1065E0007C935997A0E8B3E03CE312963C93129752
:1065F0002C9313963C93139711962C9325E63FE228
:106600002093892E30938A2E8583A6ECBCE21C92BF
:1066100011961C9241872FE032E328B939B92FE84F
:1066200032E32AB93BB910B814B813B816B817B882
:1066300011B8A0E0B9E090961D921C9291972FEFAF
:1066400030E096962D933C9397972FEF3FEF9E96D1
:106650002D933C939F978C9388E813968C93139774
:1066600080E81C968C931C9780EC17968C939487EB
:106670009387DF91CF910895E0E0FAE010821782CE
:10668000E0E8F1E012821286E0E8F3E08CE3828336
:1066900088E08083A0E2B6E01B961C921B971996B7
:1066A0001C921997E0E0F9E010821382178280E8CB
:1066B000848781E016968C93089588E08093850600
:1066C0008091C62C882391F11092C62C4091C22C47
:1066D0005091C32C495F5F4F93E0569547959A952B
:1066E000E1F7E091AA2FF091AB2F6FE072E384E421
:1066F0001995E091AD2FF091AE2F8781883019F474
:1067000083E18093932C8681883019F483E1809310
:10671000922C1092882E6091C22C7091C32CE09123
:106720009F2FF091A02F8FE092E319958091C72CB5
:10673000882399F11092C72C4091C02C5091C12C04
:10674000495F5F4F83E0569547958A95E1F7E09161
:10675000AA2FF091AB2F6FE073E387E41995E091D6
:10676000AD2FF091AE2F8781883019F483E18093AB
:10677000932C8681883019F483E18093922C81E0F8
:106780008093882E6091C02C7091C12CE0919F2F36
:10679000F091A02F8FE093E3199521B1223009F0F9
:1067A00055C08EB19FB16091080470910904409169
:1067B000C42C5091C52C862B972B841B950B409194
:1067C0001E2050911F204817590708F03FC0109213
:1067D000000A1092070A1092820110928A018CE33B
:1067E0008093820388E0809380038CE08093290665
:1067F0008FE092E388B999B98FE892E38AB99BB99F
:1068000010B814B813B816B817B811B810922009F8
:10681000109221098FEF90E0809326099093270929
:106820008FEF9FEF80932E0990932F0981E0809343
:10683000000988E88093030980E880930C0980ECC4
:106840008093070920932C0620932B0688E08093E1
:1068500086060895282F8091F02C882359F0809186
:10686000EA2C811108C081E09091E92C291718F0D9
:1068700080E0089581E008950F931F93CF93DF93F5
:106880001F92CDB7DEB70091ED2C000F000F005125
:1068900082E08093F02C10E0B8016D5F7F4F41E003
:1068A00050E089EE9CE20E948D11B8016C5F7F4F31
:1068B00041E050E0CE0101960E948D118981881F30
:1068C0008827881F8093E82C81E08093EF2C10921A
:1068D000EE2C1092EA2C1092EC2C0F90DF91CF91BD
:1068E0001F910F9108950F931F93CF93DF931F92E2
:1068F0001F92CDB7DEB78C0142E050E069E270E054
:10690000CE0101960E948D1129813A81F801908172
:106910002115310549F4218130E0322F2227A901C8
:10692000490F511DCA010DC09F70F8019083892F36
:1069300090E0A901409550954817590770F0820FD3
:10694000931F89839A8342E050E069E270E0CE01B0
:1069500001960E94DB1181E001C080E00F900F9052
:10696000DF91CF911F910F910895CF93DF931F92E5
:10697000CDB7DEB781E08093F02C40E150E060EBD2
:1069800070E088EC9CE20E948D116091CE2C5091B9
:10699000CD2C4091CC2C3091CB2C2091CA2C9091B5
:1069A000C92C8091C82C7091CF2C7093C82C609307
:1069B000C92C5093CA2C4093CB2C3093CC2C2093D1
:1069C000CD2C9093CE2C8093CF2C6091D62C5091CF
:1069D000D52C4091D42C3091D32C2091D22C909155
:1069E000D12C8091D02C7091D72C7093D02C6093A7
:1069F000D12C5093D22C4093D32C3093D42C209371
:106A0000D52C9093D62C8093D72C80E38093ED2CBB
:106A100041E050E068EA70E089EE9CE20E948D114E
:106A200041E050E06CEA70E0CE0101960E948D11C9
:106A300081E09981911180E08093E82C81E080933E
:106A4000EF2C1092EE2C1092EA2C1092EC2C0F905E
:106A5000DF91CF9108951092F02C80E18093ED2C7E
:106A60008FEF8093E92C1092E82C81E08093EF2C3B
:106A70001092EE2C1092EA2C1092EC2C089584E1E6
:106A80008093ED2CF9CE89E28093ED2CF5CE81E058
:106A90008093EF2C08951092EA2C81E08093EF2CE4
:106AA000089508958F929F92AF92BF92CF92DF92F6
:106AB000EF92FF920F931F93CF93DF93CDB7DEB783
:106AC0006097CDBFDEBF7C01DC018C919091EF2CF3
:106AD0009230F9F038F0943081F128F1963009F4D1
:106AE00056C0C2C021E09227292F21702093EE2C9E
:106AF000911102C0863219F0823509F0B5C084E4E4
:106B0000F7018083118282E08093EF2C80E190E096
:106B1000CAC39091EE2C911102C08632B9F0823531
:106B200009F0A5C013C09091EE2C911102C08632DD
:106B300069F0823509F0CDC009C09091EE2C911119
:106B400002C0863219F0823509F075C184E4D7019C
:106B50008C9311961C9281E0892716C0D7018C91E5
:106B60009091EC2C91117BC1803509F476C008F02E
:106B700086C1803309F4A2C19091F02C913009F4C0
:106B800008C208F02DC281E08093EF2C6DC08F3ACF
:106B900009F05AC0695F7F4F93E0769567959A95A3
:106BA000E1F762507109C7010E946D41882309F421
:106BB0004BC0FE0131966F0188E0DF011D928A957E
:106BC000E9F75701BFEFAB1ABB0A08EC1CE228ED4E
:106BD0003CE2AF01B50181E090E00E94850E28ED16
:106BE0003CE2AE01475F5F4FB701675F7F4F81E0D7
:106BF00090E00E94850E9091E02C8889981324C023
:106C00009091E12C898598131FC09091E22C8A8580
:106C100098131AC09091E32C8B85981315C090910E
:106C2000E42C8C85981310C09091E52C8D859813D9
:106C30000BC09091E62C8E85981306C09091E72C9E
:106C40008F85981709F40DC381E08093EF2C86E0BF
:106C5000F701808384E090E026C3D70111968C91E0
:106C600081111CC11092EF2C80E090E01CC383398D
:106C700009F089CF19821A821B821C8288E88983D5
:106C800043E050E060E070E0CE0102960E948D117A
:106C9000F7018181803261F1803709F05CC0F70132
:106CA000928189819813C2C093818A819813BEC052
:106CB00094818B819813BAC095818C819813B6C04A
:106CC00084E0808361E070E0C7010E94424183E07C
:106CD0003EC0853909F057CF44E050E064E070E0F1
:106CE000CE0101960E948D11F70181818032A9F4B5
:106CF0002981D7012C933A8111963C9311979B815E
:106D000012969C9312978C8113968C93139723273A
:106D10009227892714968C9387C08037E1F4F70176
:106D200092818981981382C093818A8198137EC051
:106D300094818B8198137AC095818C81981376C049
:106D4000108261E070E0C7010E94424184E08093BC
:106D5000EF2C38E16CC0082F02950F700250182FED
:106D60001F7088E090E0811B91092FEF30E06901EE
:106D700002C0D594C7948A95E2F7053021F004301B
:106D800051F51123E1F044E050E0B7016E5F7F4F11
:106D9000CE0101960E946D70892B69F49A818981D8
:106DA00089279B8189279C818927D70116969C91E9
:106DB00089278C2161F1043071F4111137C044E04E
:106DC00050E0B7016E5F7F4FCE0101960E946D705B
:106DD000892BE9F02BC0043048F510E0A801B70179
:106DE0006E5F7F4FCE0101960E946D70892BF1F48A
:106DF000D701A00FB11FE1E0F0E0EC0FFD1FE00FA5
:106E0000F11F12969C9180818927C82279F42981EB
:106E1000F70120833A8131839B8192838C81838324
:106E2000232792278927848338E201C030E020E0BD
:106E3000832F922F38C2695F7F4F83E076956795E5
:106E40008A95E1F76330710508F49DCE62507109AF
:106E5000C7010E946D41811181CE81E0F9CE10926F
:106E6000EC2C6091EB2C6932E1F48091F02C8130B4
:106E7000C1F4C701029637DD882381F0CCC1803A86
:106E800009F471C0823A09F077CED70111961C91AE
:106E9000193209F44CC0123008F04EC0D7011C92D0
:106EA000D9CE8091A82F8111B6C1B4E06B9FB001FB
:106EB000112444E050E0C7010296ABC1F7011181F3
:106EC0008091F02C882369F09091E82C992339F077
:106ED0009091EA2C911103C00091E92C06C08130F9
:106EE00019F00091ED2C01C00CE21017B8F6C12C7E
:106EF000D12CF4E01F9FB001112444E050E0C70101
:106F00008C0D9D1D0E948D111F5F101301C010E09C
:106F100024E0C20ED11C80E1C816D10451F760E113
:106F200070E0C7010E94424180E990E0BCC18091BD
:106F3000F02C813009F49DCF8091ED2C181708F0CA
:106F4000ADCF812F87DC882309F481CEC70102965B
:106F50002091A82F21115FC1F4E01F9FB0011124DF
:106F600044E050E056C1D70111961C91123008F44C
:106F700095CF8091ED2C181708F090CF812F6ADC07
:106F8000882309F464CE1093EB2C81E08093EC2CE1
:106F900042C18A3109F0F7CD86E08093EF2C68E09A
:106FA00080EE9CE20E94CB1088E0E8EDFCE2DF017D
:106FB0001D928A95E9F7A7014F5F5F4F08EC1CE22D
:106FC0009F0160EE7CE281E090E00E947C0E8FEAFF
:106FD000F701808369E070E0C7010E94424161C10E
:106FE0008C3309F41AC148F4893309F4B0C08A33E8
:106FF000D9F18B3109F0C7CD75C08B3409F41CC1B0
:1070000038F48E3309F0BFCD8DEBD7018C9321C1BD
:10701000803621F0853A09F4B5C0B5CDD7011C9270
:1070200084E011968C93119783E012968C931297BB
:1070300081E013968C93139714968C93149715965E
:107040001C928091ED2C843111F08EE001C08BE018
:10705000F701868383E0878368E070E0C7010E94C0
:10706000424180E590E01FC1D7011196DC90119755
:1070700012960C910D1508F411CF8091ED2CD816B5
:1070800008F00CCF081708F009CF8091E82C88236E
:1070900051F08D2DDFDB882309F4D9CD802FDADB89
:1070A000882309F4D4CD10E06D2D70E0061B170B7A
:1070B0000F5F1F4F000F111F000F111F660F771F6B
:1070C000660F771FA801C7010E948D11B801C70183
:1070D0000E944241C8010296A3E0880F991FAA9519
:1070E000E1F7E1C00091ED2C000F000F005110E01E
:1070F000B801685F7F4F44E050E0CE0101960E94E6
:107100008D119981F701818198130CC09A81828138
:10711000981308C09B818381981304C09C8184814B
:10712000981711F086E065C081E08093EA2CB801E1
:10713000645F7F4F42E050E0C7010E948D1162E022
:1071400070E0C7010E94424180E290E0ACC0F701CC
:107150006181633008F0A2CE8091ED2C70E0680F61
:10716000711D660F771F660F771F43E050E0C70160
:107170000E948D1163E070E0C7010E94424188E2E5
:1071800090E091C0D70111962C91022F10E0902F22
:107190008827856A092E000CAA0BBB0BF7013281E8
:1071A0004C015D01A32A233010F0108253CD809151
:1071B000ED2CB801680F711D660F771F660F771FE2
:1071C00044E050E0CE0101960E948D1149815A8120
:1071D0006B817C81D501C401840F951FA61FB71F49
:1071E00089839A83AB83BC830097A105B14020F0CB
:1071F00084E0D7018C932ECD8091ED2CB801680FDF
:10720000711D660F771F660F771F44E050E0CE01B7
:1072100001960E94DB118AE01BCD40E250E06AEC4F
:1072200070E0C7010E94947060E270E0C7010E94A4
:10723000424180E191E037C06091ED2C660F660F0E
:10724000605170E06B5F7F4F41E050E0C7010E94EA
:107250008D1161E070E0C7010E94424188E190E039
:1072600022C0198147E050E0BE016E5F7F4FC6012A
:107270000E948370188708EC1CE228ED3CE2A5010F
:10728000B60181E090E00E947C0ED7011C9269E07B
:1072900070E0C701F7D781E08093EA2C84E0809307
:1072A000EF2C88E590E06096CDBFDEBFDF91CF91F7
:1072B0001F910F91FF90EF90DF90CF90BF90AF9014
:1072C0009F908F900895CF93DF93EC0143E050E0BF
:1072D00060E070E00E948D1144E050E064E070E0F6
:1072E000CE010396DF91CF910C948D110F931F93D4
:1072F000CF93DF931F921F92CDB7DEB78C01FC01B5
:1073000090818181892798E88927928189278A83BA
:10731000948183818927958189279681892789830B
:1073200043E050E060E070E0C8010E94DB1141E002
:1073300050E063E070E0CE0102960E94DB1144E071
:1073400050E064E070E0C80103960E94DB1141E068
:1073500050E068E070E0CE0101960E94DB110F90D2
:107360000F90DF91CF911F910F91089581E080934D
:10737000142D84E090E08093F32C9093F42C89E01A
:107380008093F22C1092F12C089581E08093142DBB
:1073900084E090E08093F32C9093F42C88E0809329
:1073A000F22C1092F12C089581E08093142D84E446
:1073B00090E08093F32C9093F42C88E08093F22C4F
:1073C0001092F12C089581E08093142D82E090E0DA
:1073D0008093F32C9093F42C88E18093F22C1092FC
:1073E000F12C089581E08093142D82E490E0809345
:1073F000F32C9093F42C88E18093F22C1092F12CD2
:10740000089581E08093142D089508958F929F929E
:10741000AF92BF92CF92DF92EF92FF920F931F93A2
:10742000CF93DF93CDB7DEB76397CDBFDEBF8C01BF
:107430005B018091142D6730710501F5F801908191
:10744000882311F0963211F09235C1F421E08111B8
:1074500020E02093F12C4091F32C3091F42C211159
:1074600002C0963211F0923539F4F801408331832D
:107470008FEF8093F52C38C0A12CB12C853009F406
:107480009CC050F48230A9F1C8F0833009F469C07F
:10749000843009F482C0C2C5883009F425C138F4AB
:1074A000863009F49AC0873009F4D3C0B7C5893053
:1074B00009F44FC38D3008F471C3B0C591E089273A
:1074C000982F91709093F12C3091F32C2091F42C03
:1074D000F8019081811102C0963219F0923509F0BD
:1074E00019C4F8013083218384E08093142D80E156
:1074F00096C5F8018081982F9D7F913419F48AE018
:10750000808367C38033C1F462E070E0C801E5D6D0
:10751000882309F49CC0F8016181F0E16F9FB001FC
:10752000112440E150E0C8010E948D1160E170E03B
:10753000C801A8D680E973C5803A79F462E070E0AA
:10754000C801CBD6882309F482C0F80181818093D9
:107550000B2D83E08093142DD2CF803509F05EC5CA
:1075600052C060E170E0C801B8D6882389F08091EC
:10757000A82F81110BC060910B2DF0E16F9FB0011E
:10758000112440E150E0C8010E94DB118AE001C0F3
:1075900081E0F801808382E01AC39091F12C309150
:1075A000F32C2091F42CF8018081911102C08632D5
:1075B00011F1823509F0B6C31EC09091F12C3091C3
:1075C000F32C2091F42CF8018081911102C08632B5
:1075D00091F0823509F053C40EC09091F12C309196
:1075E000F32C2091F42CF8018081911102C0863295
:1075F00011F0823531F4F8013083218381E089274D
:1076000086C38035C9F4F8018181882319F0F80117
:107610001082DFC262E070E0C8015FD68823B9F053
:10762000E091AA2FF091AB2F40E060E070E081E99B
:1076300019951092142DF2C490EA980F923008F028
:10764000C1C462E070E0C80148D68111EAC481E09B
:1076500054C2C8010E94404764E07801F4E0EF0E94
:10766000F11CC7010E94574AE091AA2FF091AB2F5D
:1076700044E0B70180EA1995F801948180910C2DBE
:10768000981329C0958180910D2D981324C096815F
:1076900080910E2D98131FC0978180910F2D981304
:1076A0001AC08091102D80838091112D818380914B
:1076B000122D82838091132D838364E0C8010E9480
:1076C000494CE091AA2FF091AB2F44E0B80181EA38
:1076D000199588E009C2E091AA2FF091AB2F44E000
:1076E0006CE07DE280EC32C2F8018081803551F49B
:1076F0008181811107C08281873521F483818D3C8E
:1077000009F40AC264E0C8010E94574AF801808166
:10771000803309F0C2C062E070E0C801DED5882382
:1077200009F4ACC0F801618167FD04C0862F837045
:10773000833029F0862F8F708F3009F084C06093DA
:107740000B2D8091F62C9091F72C3091F82C282F4E
:1077500022952095422F4927407F09F043C02327D7
:107760002F7009F03FC0929590959327907FD1F5A7
:10777000262F67FD02C0237003C02F7009F023E09D
:10778000982F9095432F42954F702223C1F0892F57
:1077900090E0022E02C0959587950A94E2F7982F03
:1077A000E32FF0E0022E02C0F595E7950A94E2F788
:1077B0003E2F50E002C0559547952A95E2F740FBD1
:1077C000CC24C0F8D12CCC0CDD1CCC0CDD1C30FB47
:1077D000EE24E0F8F12CEE0CFF1CEC28892F8170D0
:1077E0008E2901C087E020910A2D30E0280F311D3D
:1077F000280F311DF901E05CFF4D8081F8019801EF
:10780000205F3F4F1192E217F307E1F79091F92CB7
:10781000F801918782FF09C09091F62C9683909190
:10782000F72C97839091F82C908784FF15C06360A4
:10783000F0E16F9FB0011124665F7F4F46E050E09A
:10784000C8010A9607C080E1689FB001112440E199
:1078500050E0C8010E948D1160E170E0C80112D5AE
:10786000E091AA2FF091AB2F42E1B80180E8199581
:1078700062E1C8010E94494C80E939C10E94624915
:1078800091E08927F8018083E091AA2FF091AB2F36
:1078900044E0B80181EC19959CC1803A61F462E042
:1078A00070E0C8011AD58823D9F1F801818180934D
:1078B0000B2D89E00DC0803C89F462E070E0C801C6
:1078C0000CD5882369F1F801818180930B2D8BE021
:1078D0008093142D0E9462499AE00EC1813C91F47C
:1078E00062E070E0C801F9D48823D1F0F801818109
:1078F00080930B2D4AE0F42EF092142D0E946249E1
:107900008F25FBC0823C99F462E070E0C801E5D4A9
:10791000882331F0F801818180930B2D8CE0D8CF42
:10792000E091AA2FF091AB2F44E0B80121C0803B39
:1079300011F562E070E0C801D0D4E091AA2FF09177
:10794000AB2F44E0B801882399F086E8199580911F
:10795000A82F8111BFCFF8016181F0E16F9FB001C5
:10796000112440E150E08AEF9CE20E94DB11B2CF8B
:1079700081EC1995BEC090EA980F923008F0BFC014
:1079800062E070E0C801A9D4882309F4B2C0F8010C
:107990008081803621F03AE3C32ED12C03C020E34E
:1079A000C22ED12CF801818187FF0CC0807FF0E1CD
:1079B0008F9F7001112480ECC80ED11C96EFA92E68
:1079C000B12C08C08C7F90E1899F7001112486E35F
:1079D000A82EB12CE091AA2FF091AB2F42E0B80174
:1079E00080E91995F8018081817080930A2DC70183
:1079F000B4E096958795BA95E1F780930B2D909119
:107A0000F52C981769F0B7016A0D7B1D44E050E032
:107A100086EF9CE20E948D1180910B2D8093F52CB6
:107A200068E0CE0101960E94CB108091A72F44E020
:107A300050E0873019F463E070E002C060E070E06D
:107A4000CE010F960E948D11B7016C0D7D1D46E091
:107A500050E0CE0109960E948D11898180930C2DF2
:107A60008A8180930D2D8B8180930E2D8C81809344
:107A70000F2D60E48CE09DE20E948F4E80910C2DD2
:107A80008093102D80910D2D8093112D80910E2DBE
:107A90008093122D80910F2D8093132D60E280E151
:107AA0009DE20E948F4E20E0AE014F5F5F4FBE010E
:107AB000615F7F4FCE010996F7D68981F8018083F7
:107AC0008A8181838B8182838C818383E058FF4FFD
:107AD0008D81808331968E81808331968F818083E2
:107AE00031968885808387E08093142D80E290E131
:107AF00074C30E94624991E08927F80101CD803565
:107B0000B9F4F8018181811182CD62E070E0C80191
:107B1000E4D3882309F49BCD1092142DE091AA2F71
:107B2000F091AB2F40E060E070E081E9199576C2FA
:107B3000A501495F5F4FA3E056954795AA95E1F7E8
:107B4000E091AA2FF091AB2FB80182E9199581E05D
:107B5000DEC062E1C8010E94574A60E170E0C801DE
:107B6000BCD3E091AA2FF091AB2F882329F142E1F9
:107B7000B80181E819958091A82F81110BC06091FF
:107B80000B2DF0E16F9FB001112440E150E0C801DE
:107B90000E94DB110E9462499AE015C066E0C801AC
:107BA0000E94574A64E070E0C80197D3811113C066
:107BB000E091AA2FF091AB2F44E0B80181EC199528
:107BC0000E94624991E08927F801808388E08093D0
:107BD000142D84E024C260910B2DF0E16F9FB00161
:107BE000112440E150E08AEF9CE20E948D119091B7
:107BF000FA2C8091FE2C80959813EBC28091022D77
:107C00009813E7C22091FB2C8091FF2C80952813BC
:107C1000E0C28091032D2813DCC2C090FC2C80911F
:107C2000002D8095C812D5C28091042DC812D1C2F2
:107C30008091FD2C3091012D30958313CAC2309173
:107C4000052D8313C6C24091062D3091072D309526
:107C50004313BFC23091082D4313BBC23091092D8D
:107C600030954313B6C2F801308141818280912C56
:107C7000A12CB12C540199248824942A832A33817D
:107C8000B32AD12CE12CF12C7601DD24CC24D22A8C
:107C9000C92AF82A8091142D8B3009F07FC2E09117
:107CA000AA2FF091AB2F46E0B80185E81995C818C6
:107CB000D908EA08FB08C092FA2C33272F2D1E2D75
:107CC0000D2D0093FB2CA701662777274093FC2CF2
:107CD0008F2D9927AA27BB278093FD2CEC2DE095AB
:107CE000E093FE2CE02FE095E093FF2CE42FE0954D
:107CF000E093002DE82FE095E093012DC092022D36
:107D00000093032D4093042D8093052D88E08093EC
:107D1000142D84C1903409F081C182E08093142D28
:107D20008AE0EBCE833909F084CC8091A72F87308D
:107D300009F0A0C043E050E060E070E0CE010296A0
:107D40000E948D1188E88983F8019181903219F0A1
:107D5000903761F024C0F80180833A8131832B8110
:107D600022839C8193832327822728C1F801828163
:107D7000883809F053C193818A8198134FC1948147
:107D80008B8198134BC195818C81981347C184E0F6
:107D9000808361E070E0C80175D285E09EC0E92E65
:107DA000E2942FE0E2222EEF2E0D9F70F92E88E054
:107DB00090E08F1991094FEF50E06A0102C0D5940D
:107DC000C7948A95E2F7253021F0243059F5FF2039
:107DD000E9F044E050E0B8016E5F7F4FCE010196BC
:107DE0002B8B0E946D702B89892B61F49A818B817A
:107DF000892798E889279C818927F8019681892716
:107E00008C2181F1243071F4F11008C144E050E07C
:107E1000B8016E5F7F4FCE0101960E946D70892B75
:107E200009F1FCC0243008F0F9C0E22EF12CA701C2
:107E3000B8016E5F7F4FCE0101960E946D70892B55
:107E400009F0ECC0D801AE0DBF1DE1E0F0E0EC0F91
:107E5000FD1FEE0DFF1D12969C9180818927C8227F
:107E600009F0DCC098E8F80190833A8131832B81D6
:107E70002283A0C044E050E060E070E007C0853994
:107E800009F0D7CB44E050E063E070E0CE0101960A
:107E90000E948D119091F22CF8018181803209F4B9
:107EA00082C08037F1F4F801228189812813B6C09D
:107EB00023818A812813B2C024818B812813AEC00C
:107EC00025818C812813AAC0908361E070E0C801ED
:107ED000D9D18FEF8093F52C86E08093142D88E123
:107EE0009EC0E82EE2949FE0E9222EEF2E0D8F70C7
:107EF000F82E88E090E08F1991094FEF50E06A0169
:107F000002C0D594C7948A95E2F7253021F0243039
:107F100059F5FF20E9F044E050E0B8016E5F7F4F73
:107F2000CE0101962B8B0E946D702B89892B61F4F9
:107F30009A81898189279B8189279C818927F801DA
:107F4000968189278C2179F1243071F4F11066C073
:107F500044E050E0B8016E5F7F4FCE0101960E9471
:107F60006D70892B01F15AC0243008F057C0E22E01
:107F7000F12CA701B8016E5F7F4FCE0101960E94E0
:107F80006D70892B09F04AC0D801AE0DBF1DE1E02C
:107F9000F0E0EC0FFD1FEE0DFF1D12969C9180810D
:107FA0008927C822D9F52981F80120833A813183B4
:107FB0009B8192838C8183832327922789278483C3
:107FC00088E22DC0823C09F0CBC0F8019181903E3F
:107FD00009F0C8C09281943B09F0C4C046E050E06B
:107FE0006AEA74E0CE0101960E948D1189818B347A
:107FF00009F02DCB8A81893709F029CB8B818B3110
:1080000009F025CB8C818A3E09F021CB8D818B37FD
:1080100009F01DCB8E818C3C09F019CB80E090E0FB
:10802000DCC0F8018081803621F08AE3C82ED12C93
:1080300003C0B0E3CB2ED12CF801818187FF0CC0A7
:10804000807FF0E18F9F7001112480ECC80ED11C5D
:10805000A6EFAA2EB12C08C08C7F90E1899F7001F9
:108060001124F6E3AF2EB12CE091AA2FF091AB2FA3
:1080700042E0B80180E91995F80180818170809310
:108080000A2DC701E4E096958795EA95E1F780937C
:108090000B2DB7016A0D7B1D44E050E086EF9CE29A
:1080A0000E948D1180910B2D8093F52C68E0CE01FC
:1080B00001960E94CB108091A72F44E050E08730BA
:1080C00019F463E070E002C060E070E0CE010F964A
:1080D0000E948D11B7016C0D7D1D46E050E0CE0170
:1080E00009960E948D11898180930C2D8A8180933D
:1080F0000D2D8B8180930E2D8C8180930F2D60E44C
:108100008CE09DE20E948F4E80910C2D8093102D6B
:1081100080910D2D8093112D80910E2D8093122D25
:1081200080910F2D8093132D60E280E19DE20E94EB
:108130008F4E87E08093142D8981F80180838A8196
:1081400081838B8182838C818383AE014F5F5F4FFC
:10815000BE01615F7F4FCE010996F0D080E25FCF14
:10816000803339F0982F9F7E903A19F0805C8330ED
:1081700078F481E08093142D84E0F8018083E0910D
:10818000AA2FF091AB2F40E060E070E082EC83CB4F
:10819000E091AA2FF091AB2F40E0D6CC8A3069F461
:1081A000E091AA2FF091AB2F46E0B80184E8199531
:1081B000C80CD91CEA1CFB1C7ECD8C3009F07BCD91
:1081C000E091AA2FF091AB2F46E0B80187E819950E
:1081D00072CD0E94624996E0F6CC6396CDBFDEBFB9
:1081E000DF91CF911F910F91FF90EF90DF90CF9093
:1081F000BF90AF909F908F900895CF93DF93209181
:10820000A72F273071F4EC0143E050E060E070E00C
:108210000E948D1144E050E063E070E0CE010396CF
:1082200004C044E050E060E070E0DF91CF910C9436
:108230008D11CF93DF931F92CDB7DEB72091A72F7B
:10824000273029F447E050E060E070E015C0FC0101
:1082500031812081232732812327338123272983DA
:1082600044E050E060E070E00E94DB1141E050E04B
:1082700064E070E0CE0101960E94DB110F90DF9167
:10828000CF91089520E42093D00026EC2093D500D0
:108290002093D40021E02093D000DC01680F791FE7
:1082A000A617B70741F0ED91F0E0EA58F84FE491D6
:1082B000E093D300F5CFE091D500F0E0EA58F84F15
:1082C000E491EC93E091D400F0E0EA58F84FE491A7
:1082D0001196EC931092D000089520E42093D000E2
:1082E00026EC2093D5002093D40021E02093D000E9
:1082F000DC01680F791FA617B70741F0ED91F0E098
:10830000EA58F84FE491E093D300F5CFE091D5001F
:10831000F0E0EA58F84FE4918C918E130AC0E09196
:10832000D400F0E0EA58F84FE49181E011969C9176
:108330009E1380E01092D000817008958F929F92DA
:10834000AF92BF92CF92DF92EF92FF920F931F9363
:10835000CF93DF93DC018C9110E0E0E086951795D8
:108360008695E795869517958695E7958695179551
:108370008695E795869517958695E79511968C9144
:108380001197869517958695E79586951795869505
:10839000E795869517958695E79586951795869521
:1083A000E79512968C911297F0E030E08695F7955C
:1083B000869537958695F795869537958695F795A1
:1083C000869537958695F7958695379513968C9172
:1083D00013978695F795869537958695F7958695A3
:1083E00037958695F795869537958695F795869571
:1083F000379514968C91149790E020E08695979588
:108400008695279586959795869527958695979530
:1084100086952795869597958695279515968C919F
:108420008695979586952795869597958695279510
:108430008695979586952795869597958695279500
:108440005B01DA014A0144E0840E911C6C91E50164
:1084500079915E017627C32ED12CA60140555E4D41
:10846000EE2EF12CE701C055DF4D7E01EA01D880E8
:10847000E7010881ED2CE02AC22ED12CA60140553F
:108480005D4DEA010881E02AF12CA70140575F4DBC
:10849000EA01088106958795DF2FD071FD2E012F07
:1084A000017EF026092F0072F0260E2F0479F026A7
:1084B000032F0377F026022F0A73F0260F2D029563
:1084C000F0260F2D06950695F0260F2D0727F6941A
:1084D0000F2506959795F79517957695CF2ED12C64
:1084E000A60140555E4DE12EF12CE701C055DF4D50
:1084F0007E01EA01D880E7010881ED2CE02AC92E2F
:10850000D12CA60140555D4DEA010881E02AF12CED
:10851000A70140575F4DEA01088106958795D32F43
:10852000D071FD2E0E2F017EF026022F0072F02654
:10853000012F0479F0260F2F0377F026092F0A73F5
:10854000F0260F2D0295F0260F2D06950695F026A4
:108550000F2D0727F6940F25069527953795E79554
:108560007695C32ED12CA60140555E4DEE2EF12CF2
:10857000E701C055DF4D7E01EA01D880E70108819F
:10858000ED2CE02AC22ED12CA60140555D4DEA010A
:108590000881E02AF12CA70140575F4DEA010881CC
:1085A00006958795DF2FD071FD2E012F017EF026D5
:1085B000092F0072F0260E2F0479F026032F03777F
:1085C000F026022F0A730F25F02EF2940F25F02EBD
:1085D000F694F6940F25F02EF72606950F25D12E4A
:1085E000102F16959795F795D79476950F2F10E045
:1085F000A80140555E4D0D2D10E000551F4DEA01BC
:10860000F880E80118810F2D012BE92EF12CA7012C
:1086100040555D4DEA011881012B10E000571F4DB8
:10862000E801188116958795032F00711E2F117E82
:108630000127122F107201271D2D147901271F2FDA
:1086400013770127192F1A730127102F129501276D
:10865000102F169516950127102F1727069510270E
:10866000169527953795E7957695032F10E0A80185
:1086700040555E4D0E2F10E000551F4DEA01F88069
:10868000E80118810F2D012BE22EF12CA701405596
:108690005D4DEA011881012B10E000571F4DE801E4
:1086A0001881169587950F2F00711D2D117E0127BA
:1086B000192F107201271E2F14790127132F1377FA
:1086C0000127122F1A730127102F12950127102F3F
:1086D000169516950127102F172706950127102F9D
:1086E00016959795F795D79476950F2F10E0A801DA
:1086F00040555E4D0D2D10E000551F4DEA01F880EC
:10870000E80118810F2D012BE92EF12CA70140550E
:108710005D4DEA011881012B10E000571F4DE80163
:10872000188116958795032F00711E2F117E012742
:10873000122F107201271D2D147901271F2F137777
:108740000127192F1A730127102F12950127102FB7
:10875000169516950127102F1727069510271695A1
:1087600027953795E7957695032F10E0A80140559A
:108770005E4D0E2F10E000551F4DEA01F880E80114
:1087800018810F2D012BE22EF12CA70140555D4DD4
:10879000EA011881012B10E000571F4DE8011881F4
:1087A000169587950F2F00711D2D117E1027092F0B
:1087B000007210270E2F04791027032F037710273C
:1087C000022F0A731027012F02951027012F0695FB
:1087D00006951027012F0727169501271D2D0695B1
:1087E0009795F7951795CF2ED12CA60140555E4D44
:1087F000E12EF12CE701C055DF4D7E01EA01D88062
:10880000E7010881ED2CE02AC92ED12CA6014055A4
:108810005D4DEA010881E02AF12CA70140575F4D28
:10882000EA01088106958795D32FD071FD2E0E2F72
:10883000017EF026022F0072F026012F0479F02627
:108840000F2F0377F026092F0A730F25F02EF294CD
:108850000F25F02EF694F6940F2576957027069541
:108860007027769527953795E79568276D93A81516
:10887000B90509F0EBCD1093152DF093162D9093BB
:10888000172DE093182D3093192D20931A2DDF9179
:10889000CF911F910F91FF90EF90DF90CF90BF90FD
:1088A000AF909F908F9008954F925F926F927F92BA
:1088B0009F92AF92BF92CF92DF92EF92FF920F936F
:1088C0001F93CF93DF93DC018C9110E0B12CEB2D43
:1088D0008695E795869517958695E79586951795DC
:1088E0008695E795869517958695E79586951795CC
:1088F00011968C911197BE2E8695B79486951795F3
:108900008695B794869517958695B794869517950D
:108910008695B7948695179512969C91129730E09C
:1089200080E0969587959695379596958795969537
:1089300037959695879596953795969587959695BB
:10894000379513969C91139796958795969537959D
:10895000969587959695379596958795969537959B
:1089600096958795969537951496EC91149790E087
:1089700000E0E6950795E6959795E6950795E695C7
:108980009795E6950795E6959795E6950795E6956B
:1089900097951596DC90D6940795D6949795D6948E
:1089A0000795D6949795D6940795D6949795D6948F
:1089B0000795D6949795E32FF0E0E055FE4DA12F53
:1089C000B0E0A055BF4DF081EC91EF2BA92FB0E0A6
:1089D000A055BD4DFC91EF2BF0E0E057FF4DE0803E
:1089E0002B01BA016C5F7F4FDA013B01AC90E201D1
:1089F000C9902E01CA24FD2DE694F795D82FD07189
:108A0000FD2EEB2DE17EFE26E02FE072FE26E12F0B
:108A1000E479FE26E32FE377FE26E92FEA73EF25BC
:108A2000FE2EF294EF25FE2EF694F694EF25FE2E00
:108A3000FC24E695FE26EB2D20FDFE24F6940795FA
:108A40008795E795BC2CB694C82ED12CA60140552D
:108A50005E4DEE2EF12CE701C055DF4D7E01EA019F
:108A6000D880E701F880ED2CEF28C02ED12CA6018C
:108A700040555D4DEA01F880EF28F12CA7014057E1
:108A80005F4DEA01D880D694F795D32FD071ED2EA3
:108A9000412F417EE426592F5072E526CE2FC4790E
:108AA000EC26D82FD377ED26402F4A73E426FE2CF0
:108AB000F294EF24FE2CF694F694EF24FE2CFB2483
:108AC000E694FE2420FDFD24F6949795379517959E
:108AD000B694C32ED12CE601C055DE4DE12EF12C0B
:108AE000A70140555F4DD880EA01F880ED2CEF28B2
:108AF000C92ED12CA60140555D4DEA01F880EF2822
:108B0000F12CA70140575F4DEA01D880D694F79524
:108B1000D82FD071ED2E4E2F417EE426502F50726B
:108B2000E526C12FC479EC26D32FD377ED26492F24
:108B30004A73E426FE2CF294EF24FE2CF694F6946D
:108B4000EF24FE2CFB24E694FE2420FDFD24F69465
:108B500007958795E795B694C82ED12CE601C055A8
:108B6000DE4DEE2EF12CA70140555F4DD880EA0175
:108B7000F880ED2CEF28C02ED12CA60140555D4D7C
:108B8000EA01F880EF28F12CA70140575F4DEA0178
:108B9000D880D694F795D32FD071ED2E412F417EFA
:108BA000E426592F5072E526CE2FC479EC26D82F13
:108BB000D377ED26402F4A73E426FE2CF294EF245F
:108BC000FE2CF694F694EF24FE2CFB24E694FE246F
:108BD00020FDFD24F694979537951795B694C32EEE
:108BE000D12CE601C055DE4DE12EF12CA7014055F8
:108BF0005F4DD880EA01F880ED2CEF28C92ED12CEA
:108C0000A60140555D4DEA01F880EF28F12CA7013F
:108C100040575F4DEA01D880D694F795D82FD07190
:108C2000ED2E4E2F417EE426502F5072E526C12FA7
:108C3000C479EC26D32FD377ED26492F4A73E42647
:108C4000FE2CF294EF24FE2CF694F694EF24FE2CE6
:108C5000FB24E694FE2420FDFD24F69407958795D9
:108C6000E795B694C82ED12CE601C055DE4DEE2E08
:108C7000F12CA70140555F4DD880EA01F880ED2C1A
:108C8000EF28C02ED12CA60140555D4DEA01F88099
:108C9000EF28F12CA70140575F4DEA01D880D69408
:108CA000F795D32FD071ED2E412F417EE426592F19
:108CB0005072E526CE2FC479EC26D82FD377ED2637
:108CC000402F4A73E426FE2CF294EF24FE2CF694F7
:108CD000F694EF24FE2CFB24E694FE2420FDFD24D4
:108CE000F6949795379517959B2C9694C32ED12C77
:108CF000E601C055DE4DE12EF12CA70140555F4D38
:108D0000D880EA01F880ED2CEF28C92ED12CA601DD
:108D100040555D4DEA01F880EF28F12CA70140573E
:108D20005F4DEA01D880D694F795D82FD0714E2F99
:108D3000417EF42EFD26502F5072F526C12FC479A6
:108D4000FC26D32FD377FD26492F4A73F426EF2C28
:108D5000E294FE24EF2CE694E694FE24EF2CE92422
:108D6000F694FE24BE2EEF2D20FDED25E695079509
:108D70008795B794C82ED12CE601C055DE4DEB2C5B
:108D8000F12CA70140555F4DD880EA01E881ED2C18
:108D9000EE2AC02ED12CA60140555D4DEA01E88196
:108DA000EE2AF12CA70140575F4DEA01F880DF2E33
:108DB000F694D794F32FF071E12FE17EEF27F92F8E
:108DC000F072EF27FB2DF479EF27F82FF377EF27D9
:108DD000F02FFA73EF27FE2FF295EF27FE2FF6956F
:108DE000F695EF2796949E26E6959E2620FD9F24D5
:108DF0009694979537951795E32FF0E0AF0140557E
:108E00005E4DE12FF0E0E055FF4DEA01F880E08192
:108E1000EF29E92EF12CA70140555D4DEA01F881BB
:108E2000EF2BF0E0E057FF4DE080EA2DF0E0EA584C
:108E3000F94FE491EE25E301E9933E01AD24AD92B3
:108E4000A617B70709F0D2CDB092152D8093162D35
:108E50000093172D1093182D3093192D90931A2DE0
:108E6000DF91CF911F910F91FF90EF90DF90CF9006
:108E7000BF90AF909F907F906F905F904F900895BC
:108E8000AF92BF92CF92DF92EF92FF920F931F9318
:108E9000CF93DF936091152D5091162D2091172DB2
:108EA0004091182D3091192DD0911A2DFC015C01A3
:108EB00004E0A00EB11C8191C52FC071962F917E48
:108EC000C927922F9072C927942F9479C927932F7D
:108ED0009377C9279D2F9A73C9277C2F7295C7272F
:108EE0007C2F76957695C727A32FB0E08D0100558E
:108EF0001E4D6801A42FB0E08D0100551F4D780173
:108F0000D6010C91D7019C91092BED2EF12CD701A4
:108F1000A055BD4D9C91092B10E000571F4DD80165
:108F20007C9178277C27C6957C2786957695279512
:108F300057956795C32FC071942F917EC9279D2F98
:108F40009072C927962F9479C927952F9377C927AF
:108F5000922F9A73C9277C2F7295C7277C2F7695FD
:108F60007695C727052F10E0D801A055BE4D6D019D
:108F7000062F10E0D801A055BF4D7D01D6010C9100
:108F8000D7019C91092BE22EF12CD701A055BD4DA4
:108F90009C91092B10E000571F4DD8017C91782738
:108FA0007C27C6957C2786959D2F76959795379536
:108FB0004795C52FC071762F717EC727722F7072AB
:108FC000C727742F7479C727732F7377C727792F13
:108FD0007A73C7277C2F7295C7277C2F7695769555
:108FE000C727032F10E0D801A055BE4D6D01042FF7
:108FF00010E0D801A055BF4D7D01D6010C91D701DD
:109000007C91072BE92EF12CD701A055BD4D7C9109
:10901000072B10E000571F4DD8017C9178277C2743
:10902000C6957C2786957695279557956795C32F86
:10903000C071742F717EC727792F7072C727762F62
:109040007479C727752F7377C727722F7A73C7274D
:109050007C2F7295C7277C2F76957695C727052F8D
:1090600010E0D801A055BE4D6D01062F10E0D801CB
:10907000A055BF4D7D01D6010C91D7017C91072BE6
:10908000E22EF12CD701A055BD4D7C91072B10E0AD
:1090900000571F4DD8017C9178277C27C6957C27E7
:1090A00086957695979537954795C52FC071762FFC
:1090B000717EC727722F7072C727742F7479C727E4
:1090C000732F7377C727792F7A73C7277C2F7295F1
:1090D000C7277C2F76957695C727032F10E0D801F8
:1090E000A055BE4D6D01042F10E0D801A055BF4D15
:1090F0007D01D6010C91D7017C91072BE92EF12C33
:10910000D701A055BD4D7C91072B10E000571F4D96
:10911000D8017C9178277C27C6957C278695769503
:10912000279557956795C32FC071742F717EC727F8
:10913000792F7072C727762F7479C727752F7377A9
:10914000C727722F7A73C7277C2F7295C7277C2F6A
:1091500076957695C727052F10E0D801A055BE4D0E
:109160006D01062F10E0D801A055BF4D7D01D6013D
:109170000C91D7017C91072BE22EF12CD701A05541
:10918000BD4D7C91072B10E000571F4DD8017C91FD
:1091900078277C27C6957C27869576959795379571
:1091A0004795C52FC071762F717EC727722F7072B9
:1091B000C727742F7479C727732F7377C727792F21
:1091C0007A73C7277C2F7295C7277C2F7695769563
:1091D000C727032F10E0D801A055BE4D6D01042F05
:1091E00010E0D801A055BF4D7D01D6010C91D701EB
:1091F0007C91072BE92EF12CD701A055BD4D7C9118
:10920000072B10E000571F4DD8017C9178277C2751
:10921000C6957C277695279557956795C32FC0717E
:10922000742F717E7C27C92FC0727C27C62FC4790A
:109230007C27C52FC3777C27C22FCA737C27C72FF3
:10924000C2957C27C72FC695C6957C278695C52FC6
:10925000D0E0C055DE4D062F10E000551F4DD881DF
:10926000D801CC91CD2B022F10E000551D4DD80117
:10927000DC91CD2BD0E0C057DF4DC8818C278727EC
:1092800076958727D92F8695D79537954795EA15EF
:10929000FB0509F010CE6093152D5093162D2093E9
:1092A000172D4093182D3093192DD0931A2DDF913F
:1092B000CF911F910F91FF90EF90DF90CF90BF90D3
:1092C000AF900895CF93DF93E5E1FDE2A081718136
:1092D0006281338124819581472F40718A2F817E5D
:1092E0008427462F40728427432F44798427422FB6
:1092F00043778427492F4A738427482F4295842730
:10930000482F469546958427482F4695842786956D
:1093100067957795A795C22FD0E0C055DE4D432FB6
:1093200050E040555F4DB881EA018881B82B492F44
:1093300050E040555D4DEA018881CB2FC82BD0E02D
:10934000C05BDF4D88818695522F5071432F417E3F
:109350004527592F507245275A2F54794527572FA3
:1093600053774527562F5A734527542F5295452733
:10937000542F569556954527542F56954527469573
:10938000979527953795C72FD0E0C055DE4D4A2FCA
:1093900050E040555F4DB881EA014881B42B462F1B
:1093A00050E040555D4DEA014881CB2FC42BD0E001
:1093B000C05BDF4D4881842B8695572F50714A2F13
:1093C000417E4527562F50724527532F5479452704
:1093D000522F53774527592F5A734527542F5295AB
:1093E0004527542F569556954527542F5695452772
:1093F000469567957795A795C22FD0E0C055DE4D6D
:10940000432F50E040555F4DB881EA014881B42BAD
:10941000492F50E040555D4DEA014881CB2FC42BC8
:10942000D0E0C05BDF4D4881842B8695C72FD0E00C
:10943000C055DE4D4A2F50E040555F4DB881EA01DE
:109440004881B42B462F50E040555D4DEA014881DC
:10945000CB2FC42BD0E0C05BDF4D4881842B522F33
:109460005071432F417E4527592F507245275A2F5F
:1094700054794527572F53774527562F5A73452739
:10948000542F52954527542F569556954527542FBE
:10949000569545274695979527953795A0837183CF
:1094A0006283338324839583DF91CF9108950F9353
:1094B0001F93CF93DF93A091152D7091162D2091BE
:1094C000172D5091182D4091192D30911A2DFC0116
:1094D000615008F4CDC1972F90718A2F817E892722
:1094E000922F90728927952F94798927942F9377BB
:1094F0008927932F9A738927982F92958927982FD8
:10950000969596958927982F9695892786952795DC
:109510007795A795C42FD0E0C055DE4D852F90E0FC
:1095200080559F4DB881EC018881B82B832F90E046
:1095300080559D4DEC018881CB2FC82BD0E0C059C0
:10954000DF4DB881B695942F9071852F817E892744
:10955000932F907289279A2F94798927972F937741
:109560008927922F9A738927982F92958927982F68
:10957000969596958927982F96958927869537955C
:1095800047955795C72FD0E0C055DE4D8A2F90E004
:1095900080559F4D1881EC018881182B822F90E017
:1095A00080559D4DEC018881C12FC82BD0E0C0595A
:1095B000DF4D8881B82BB695972F90718A2F817EC9
:1095C0008927922F90728927952F94798927942F34
:1095D00093778927932F9A738927982F92958927B4
:1095E000982F969596958927982F969589278695F1
:1095F00027957795A795C42FD0E0C055DE4D852FD0
:1096000090E080559F4D1881EC018881182B832FA5
:1096100090E080559D4DEC018881C12FC82BD0E092
:10962000C059DF4D8881B82BB695942F9071852F46
:10963000817E8927932F907289279A2F9479892781
:10964000972F93778927922F9A738927982F92952E
:109650008927982F969596958927982F96958927EB
:109660008695379547955795C72FD0E0C055DE4D65
:109670008A2F90E080559F4D1881EC018881182B2E
:10968000822F90E080559D4DEC018881C12FC82B21
:10969000D0E0C059DF4D8881B82BB695972F9071D7
:1096A0008A2F817E8927922F90728927952F94790E
:1096B0008927942F93778927932F9A738927982F37
:1096C00092958927982F969596958927982F969504
:1096D0008927869527957795A795C42FD0E0C05503
:1096E000DE4D852F90E080559F4D1881EC018881DB
:1096F000182B832F90E080559D4DEC018881C12F60
:10970000C82BD0E0C059DF4D8881B82BB695942F77
:109710009071852F817E9827832F807298278A2FBA
:1097200084799827872F83779827822F8A739827A1
:10973000892F82959827892F869586959827892F36
:1097400086959827832F9695879547955795C72F88
:10975000D0E0C055DE4D0A2F10E000551F4D388176
:10976000E8019881392B022F10E000551D4DE801CA
:109770009881C32FC92BD0E0C059DF4D3881B32B5E
:10978000B695372F30719A2F917E9327322F3072F2
:109790009327352F34799327342F33779327382F16
:1097A0003A739327392F32959327392F369536956B
:1097B0009327392F36959327969527957795A795D3
:1097C000C42FD0E0C055DE4D052F10E000551F4DD1
:1097D0003881E8019881392B082F10E000551D4D84
:1097E000E8019881C32FC92BD0E0C059DF4D988183
:1097F0003B2F392B3695C72FD0E0C055DE4D0A2FB1
:1098000010E000551F4DB881E8019881B92B022F57
:1098100010E000551D4DE8019881CB2FC92BD0E0F9
:10982000C059DF4DB881B32B342F3071952F917E05
:109830009327382F307293273A2F34799327372F75
:1098400033779327322F3A739327392F3295932703
:10985000392F369536959327392F36959327382FFC
:10986000969537954795579580818B27819330CE74
:10987000A093152D7093162D2093172D5093182D0E
:109880004093192D30931A2DDF91CF911F910F9195
:109890000895CF92DF92EF92FF921F93CF93DF93C1
:1098A0001091152DD091162DC091172D7091182D56
:1098B0004091192D20911A2DE42FF0E0E055FE4D36
:1098C000A72FB0E0A055BF4DE0813C91E32BA22F24
:1098D000B0E0A055BD4D3C91E32BF0E0E057FF4DCB
:1098E0003081DC0180E0615008F405C2582F3695C4
:1098F00057959D2F9071812F817E89279C2F907283
:109900008927972F94798927942F93778927322F46
:109910003A738327982F92958927982F9695969535
:109920008927982F969589279C2F86959795D79567
:1099300017955695342F3071872F817E8327322FCC
:1099400030728327312F347983273D2F3377832754
:10995000392F3A738327382F32958327382F36953E
:1099600036958327382F36958327869527954795F3
:109970007795CD2ED12CF601E055FE4D6F01E12EED
:10998000F12CF701E055FF4D7F01F6013081F70121
:109990008081832BE92EF12CF701E055FD4D3081BC
:1099A000E82FE32BF0E0E059FF4D8081582B5695CE
:1099B0003D2F3071812F817E8327392F307283278D
:1099C000372F34798327342F33778327322F3A7315
:1099D0008327382F32958327382F3695369583275E
:1099E000382F3695832786959795D7951795C42E4A
:1099F000D12CF601E055FE4D6F01E72EF12CF70159
:109A0000E055FF4D7F01F6013081F7018081832B06
:109A1000E22EF12CF701E055FD4D3081E82FE32BCC
:109A2000F0E0E059FF4DC0815C2B5695342F30712A
:109A3000872F817E8327322F30728327312F34790D
:109A400083273D2F33778327392F3A738327382F86
:109A500032958327382F369536958327382F3695BC
:109A600083278695279547957795CD2ED12CF6019E
:109A7000E055FE4D6F01E12EF12CF701E055FF4D51
:109A80007F01F6013081F7018081832BE92EF12CD3
:109A9000F701E055FD4D3081E82FE32BF0E0E05970
:109AA000FF4DC081C52BC6953D2F3071812F817E22
:109AB0008327392F30728327372F34798327342F28
:109AC00033778327322F3A738327382F32958327B2
:109AD000382F369536958327382F369583278695E8
:109AE0009795D7951795C42ED12CF601E055FE4DCC
:109AF0006F01E72EF12CF701E055FF4D7F01F601D4
:109B00003081F7018081382BE22EF12CF701E055EE
:109B1000FD4D8081E32FE82BF0E0E059FF4D80817F
:109B2000C82BC695342F3071872F817E8327322F23
:109B300030728327312F347983273D2F3377832762
:109B4000392F3A738327382F32958327382F36954C
:109B500036958327382F36958327542F869527955A
:109B600057957795CD2ED12CF601E055FE4D6F011E
:109B7000E12EF12CF701E055FF4D7F01F601308118
:109B8000F7018081832BE92EF12CF701E055FD4D83
:109B90003081E82FE32BF0E0E059FF4D80818C2BE2
:109BA000482F46953D2F3071812F817E3827892F90
:109BB00080723827872F84793827852F8377382735
:109BC000822F8A733827832F82953827832F869593
:109BD00086953827832F86953827C92F3695C795C0
:109BE000D7951795E52FF0E0E055FE4D872F90E0D3
:109BF00080559F4D3081FC018081382B822F90E071
:109C000080559D4DFC019081E32FE92BF0E0E05958
:109C1000FF4D9081842F892B382F3695ED2FF0E062
:109C2000CF0180559E4D6C01E12FF0E0CF018055B2
:109C30009F4DF6014081FC019081492BEC2EF12CC7
:109C4000C70180559D4DFC019081E42FE92BF0E088
:109C5000E059FF4D9081832F892B352F3071972F3D
:109C6000917E3927922F90723927912F9479392735
:109C70009D2F937739274C2F4A733427932F929532
:109C80003927932F969596953927932F96953927AF
:109C9000452F3695279547957795C42ED12CF601FB
:109CA000E055FE4D6F01E72EF12CF701E055FF4D19
:109CB0007F01F6013081F7019081392BE22EF12CE2
:109CC000F701E055FD4D9081E32FE92BF0E0E057DF
:109CD000FF4D30819C91E92FF0E0EA58F94FE49173
:109CE0007D01F0E8EF0EF11C5E2F5327F701508342
:109CF00098279D93F8CD1093152DD093162DC093D2
:109D0000172D7093182D4093192D20931A2DDF9144
:109D1000CF911F91FF90EF90DF90CF9008950F9318
:109D20001F93FC01862F90812181428150E060E0E9
:109D300070E0BA0155274427522B492B9381792B88
:109D40008B0122273327803208F471C0D80123E029
:109D5000B695A7952A95E1F70A271B27980136950E
:109D6000279536952795BBE0769567955795479546
:109D7000BA95D1F70227132720E030E095E1000FD4
:109D8000111F221F331F9A95D1F7402B512B622BA5
:109D9000732B8B0122273327D80133E0B695A79583
:109DA0003A95E1F70A271B279801369527953695AE
:109DB0002795BBE07695679557954795BA95D1F766
:109DC0000227132720E030E095E1000F111F221F2A
:109DD000331F9A95D1F7402B512B622B732B8B019C
:109DE00022273327D80133E0B695A7953A95E1F7B6
:109DF0000A271B2798013695279536952795BAE0AF
:109E00007695679557954795BA95D1F70227132709
:109E100020E030E096E1000F111F221F331F9A95BA
:109E2000D1F7402B512B622B732B805289CF40836B
:109E30005183028373831F910F910895AF92BF9254
:109E4000CF92DF92EF92FF920F931F93CF93DF9306
:109E50006730710509F451C09B0127703327232B0C
:109E600009F04EC0EB016C015B0183E0B694A7944E
:109E70008A95E1F77B0196E0F694E7949A95E1F7ED
:109E8000EA0CFB1CEC0CFD1C8501015011090C0DAA
:109E90001D1DA701401B510B60E070E0C801019639
:109EA0000E9494700C151D0520F1D801EC91F0E092
:109EB000EA58F94F44919701D7010A171B0768F434
:109EC0008C91982F990FF90182919F01881F882703
:109ED000881F892B8C931197F0CF11968C91119735
:109EE0008E7FE42FE170E82B1196EC93015011095D
:109EF000D9CFC5018C0F9D1F04C087E090E001C041
:109F0000CB01DF91CF911F910F91FF90EF90DF90E8
:109F1000CF90BF90AF900895CF93DF93EC0182EC88
:109F2000888361E070E0CE010E9442418AE0809324
:109F3000F52D1092F62D68E170E0CE01DF91CF9102
:109F40007DCFEF92FF920F931F93CF93DF93EC019E
:109F5000CB0167307105D1F169E070E00E94C46FF8
:109F6000DE0120E030E088E090E02617370739F185
:109F7000F90143E0F695E7954A95E1F7E20FF31F03
:109F8000EC0FFD1F408150E0890107701127002E62
:109F900002C0559547950A94E2F74C9301151105B7
:109FA00051F0E1817C01E01AF10A01C0EE0FEA9460
:109FB000EAF74E2B4C932F5F3F4F1196D6CFC90136
:109FC00023E0880F991F2A95E1F702C087E090E00F
:109FD000DF91CF911F910F91FF90EF900895EF9235
:109FE000FF920F931F93CF93DF93EC01CB01673068
:109FF000710509F442C069E070E00E94C46F20E07E
:10A0000030E088E090E026173707B9F1D90143E046
:10A01000B695A7954A95E1F7A20FB31FA90147701E
:10A020005527AC0FBD1FEC91F0E0042E02C0F59552
:10A03000E7950A94E2F74115510559F011960C91F4
:10A0400011977C01E41AF50A01C0000FEA94EAF7BF
:10A05000E02BF0E0EA58F94FE4911196AC91B0E0B2
:10A060008D0102C0159507954A95E2F7A8014E2784
:10A0700040FD05C02F5F3F4FC6CF81E001C080E0AB
:10A08000DF91CF911F910F91FF90EF900895109263
:10A09000F52D08951092F52D10921B2D1092F62D8E
:10A0A0000895F8DF0E94F82E1092F52D0895089576
:10A0B0000895DC0123E633E66150E8F04D91942FDA
:10A0C000922780E1989FA00111244927E42FF0E016
:10A0D00042954F70232F3327C9018427AC013E2FAF
:10A0E00022272427352743E0EE0FFF1F4A95E1F78B
:10A0F0002E273F27E1CFC9010895EF92FF921F93CA
:10A10000CF93DF93EC017B018091F62D882339F00A
:10A110008091F52D823008F0EDC01092F62DE114FB
:10A12000F10461F0B701CE015ADF882309F4E5C0DC
:10A13000B701CE0106DF7C0181E001C082E0109111
:10A14000F52D163090F4133090F51230A8F484E019
:10A1500090E080931E2090931F2082E5888382E008
:10A160008093F52D87E090E0D9C0193008F479C0CC
:10A170001A3009F4A8C0BEC090E1E916F10411F448
:10A1800080FD03C01092F52DA4C0898190E0982F26
:10A1900088272881822B8093E72D9093E82D83E9EF
:10A1A000888380E2898383E08093F52D78C080FFE7
:10A1B000E9CF88E2E816F10428F328818981822713
:10A1C0009A8189279B8189279C818913DBCF812FE5
:10A1D00090E00397283879F49C01220F331F820FF7
:10A1E000931FFC01E651F24D29813A814B81208376
:10A1F0003183428310C0FC01EE0FFF1F8E0F9F1FA3
:10A20000FC01E651F24D88819981AA81BB8180834E
:10A210009183A283B38345E050E0BE01CE01029654
:10A220000E948370133021F0143021F087E903C0BD
:10A2300083E901C085E9888380E7898367E070E06E
:10A24000CE010E9442418091F52D8D5F8093F52DC6
:10A2500068E470E0CE01DF91CF911F91FF90EF9005
:10A26000EDCD80FF8FCF98E1E916F10409F08ACF98
:10A2700063E0CE011EDF009709F084CF288122FF22
:10A2800011C0183079F0163011F087E901C085E966
:10A29000888380E289832EEF210F2093F52D60E1E2
:10A2A00070E0D8CF21E02093F62D212F30E026500A
:10A2B0003109322F330F230F2C5F2093F42D288187
:10A2C0002093E92D2BC0982F927031F081E080937C
:10A2D000F52D0E94F12E0EC080FF05C063E0CE0177
:10A2E000E8DE892B99F3CE01DF91CF911F91FF908A
:10A2F000EF9012CE80E090E011C0A701495F5F4F60
:10A3000083E0569547958A95E1F7E091AA2FF09161
:10A31000AB2FBE0181EC199580E011CFDF91CF9179
:10A320001F91FF90EF9008959F92AF92BF92CF92AE
:10A33000DF92EF92FF920F931F93CF93DF93CDB7EE
:10A34000DEB7C756D109CDBFDEBF8C017B01FB0153
:10A3500060817181D2DED090F62DDD2009F445C1F7
:10A360008091F52D9AEF980F933008F058C0F801BE
:10A37000C080C5FACC24C0F81092D72D5AE1A52E82
:10A3800053E1B52E912C47E650E0B501CE01019680
:10A390000E944C708B81882349F029813A818091F9
:10A3A000E72D9091E82D28173907B9F48D8188237E
:10A3B00029F09C818091E92D98130FC08F89882303
:10A3C00011F0CC2051F0E091D72D81E08E0F8093D9
:10A3D000D72DF0E0E852F24D90829394F7E6AF0E5D
:10A3E000B11C8FE09812CFCFC1100DC08091F52D18
:10A3F0009AEF980F943008F0ADC09091D72D28EDCA
:10A400003DE2F9018CC080EEF801808380E8818311
:10A4100062E070E0C8010E94424189E094C0893046
:10A4200029F7F70160817181C801D9DDF7016081E9
:10A430007181811115C0CB01089667E070E00E9420
:10A44000C46F462FE091AA2FF091AB2FB80181EC99
:10A450001995C80161DDF70180839183D12CC8C0B3
:10A46000C8016FDDF70180839183F8016081262F99
:10A4700030E043E0969587954A95E1F702972817D3
:10A48000390739F76E5FC80114DE892B11F7C12C2B
:10A4900097E6992E5801FFEFAF1ABF0A8091D72D8A
:10A4A000C81608F0A3CFEC2DF0E0E852F24D608121
:10A4B000969EB0011124665E7C4E47E650E0CE01C8
:10A4C00001960E944C708F89882339F14E8950E0A3
:10A4D000F801808190E001974817590739F4B501D8
:10A4E000CE0106960E946D70892BB9F02091D72D70
:10A4F000422F50E0415051093C2D832F90E08417AA
:10A5000095073CF4FC01E852F24D818180833F5F66
:10A51000F4CF21502093D72DCA94C394BFCF8E2F50
:10A52000821B891708F064C0819184508230B8F78B
:10A5300082E0F801808380E6818362E070E0C801F8
:10A540000E9442418BE08093F52D60E270E0C801EB
:10A5500075DC81CF8B3009F04BC0F70160817181D0
:10A560006115710509F43EC0C80139DDD82EF70127
:10A5700060817181811113C0CB01089667E070E0A2
:10A580000E94C46F462FE091AA2FF091AB2FB80123
:10A5900081EC19951092D72DC801BEDC26C0C801E8
:10A5A000D0DCF70180839183BC0183E076956795C9
:10A5B0008A95E1F7C8017DDD892B19F01092D72D1E
:10A5C00048CFF8018581882331F0813059F4809398
:10A5D000D72D85E004C081E08093D72D84E080935F
:10A5E000D82D06C01092D72D03C0F7018083918328
:10A5F0008D2DC959DF4FCDBFDEBFDF91CF911F91A8
:10A600000F91FF90EF90DF90CF90BF90AF909F9011
:10A6100008955F926F927F928F929F92AF92BF92B6
:10A62000CF92DF92EF92FF920F931F93CF93DF931E
:10A63000CDB7DEB7C254D240CDBFDEBF7C01CF5B09
:10A64000DD4F68837983C154D24080911B2D8430C3
:10A6500009F48EC140F4823009F4D9C008F063C116
:10A66000813069F0AFC4863009F441C308F44BC2AD
:10A67000873009F4EAC3883009F445C2A3C40091C5
:10A680008F2F1091902F01151105C1F0A801495F7E
:10A690005F4FE3E056954795EA95E1F76DE87EE276
:10A6A000C7010E947A7060918F2F7091902FC7011F
:10A6B000C5DB10928F2F1092902F23C2CF5BDD4FFE
:10A6C00068817981C154D2406115710509F4C7C010
:10A6D000C70185DCD82ECF5BDD4F68817981C154FD
:10A6E000D240C7012EDCCF5BDD4F88839983C154F4
:10A6F000D2409C01295F3F4FC901880F991F73E029
:10A70000969587957A95E1F706968138910578F0C8
:10A7100068ED73E2CE0101960E94A67010921B2D87
:10A72000BE016F5F7F4F85E60E94A3258BC443E087
:10A73000369527954A95E1F7A70160E870E0CE01CC
:10A7400001960E94E4107C01CF5BDD4F8881C154EB
:10A75000D240CE5BDD4F9881C254D240CF5FDD4FF7
:10A760009883C150D240CE5FDD4F8883C250D24023
:10A7700087EE93E29F938F9350E8A52EB12CC501ED
:10A780008E199F099F938F9381E090E08C0F9D1FFE
:10A790008E0D9F1D9F938F930E94AD70E80EF91E42
:10A7A000B5016E197F0922E030E0AE014F5F5D4FC9
:10A7B00081E090E08C0F9D1F8E0D9F1D0E94E41084
:10A7C0008E0D9F1D0F900F900F900F900F900F9078
:10A7D000A501481B590B21E030E02C0F3D1F280F2D
:10A7E000391FD11003C08AEE93E202C089EF93E2D1
:10A7F0009F938F935F934F933F932F930E94AD70DE
:10A800000F900F900F900F900F900F9087CF0091A7
:10A810008F2F1091902F01151105C1F0A801495FEC
:10A820005F4F93E0569547959A95E1F76DE87EE284
:10A83000C7010E947A7090918F2F8091902F109273
:10A840008F2F1092902F092F182FFCC3CF5BDD4F55
:10A8500028813981C154D2402115310551F488E055
:10A86000E1E8F4E2DE01119601900D928A95E1F79C
:10A8700055CF295F3F4FB3E036952795BA95E1F75D
:10A88000A70160E870E0CE0101960E94E4107C010F
:10A89000CF5BDD4F8881C154D240CE5BDD4F9881C4
:10A8A000C254D240CF5FDD4F9883C150D240CE5FBB
:10A8B000DD4F8883C250D24087EE93E29F938F93FF
:10A8C00080E8C82ED12CC6018E199F099F938F93C3
:10A8D00081E090E08C0F9D1F8E0D9F1D9F938F93A5
:10A8E0000E94AD708E0D9F1DB601681B790B22E092
:10A8F00030E0AE014F5F5D4FA1E0B0E0AC0FBD1F97
:10A900008A0F9B1F0E94E41010921B2DBE016F5FE7
:10A910007F4F85E60E94A3250F900F900F900F9018
:10A920000F900F908FC3CF5BDD4F68817981C15449
:10A93000D240C701E2DB2091F62D222309F445C362
:10A940002091F42D30E04AEE5DE264E170E0CE014A
:10A9500001960E94E410BE016F5F7F4F85E60E9462
:10A96000A3251092F62D10921B2D0E943A262AC381
:10A970008091D62D811108C080E890E00E948E263B
:10A9800081E08093D62D7DC0813009F07CC080911C
:10A99000F52D823008F077C08091D52D8F5F8093A0
:10A9A000D52D803109F06FC00E9499268C019350FB
:10A9B000409768F00115B8E01B0708F462C060E139
:10A9C00070E0E0E0F0E0A12CB12C90E042C0ADE5F9
:10A9D000BDE240E050E0E0E0F0E020E030E060E0A8
:10A9E00070E090E08D91803149F44732510509F4CF
:10A9F00026C391110EC0BA0191E00BC0992349F012
:10AA0000CA01861B970B8217930710F0FB019C016C
:10AA100090E04F5F5F4F4832510521F724303105F8
:10AA200008F05AC22EC0D601ED906D01F12CE61649
:10AA3000F706C0F491111BC04F5F5F4F48375105B7
:10AA400091F72115310509F047C26150710909F4E8
:10AA500043C2ADE5CA2EADE2DA2E40E050E020E080
:10AA600030E0E1CF9111E8CF5A0191E0E5CFCA0182
:10AA70008A199B098217930710F0F5019C0190E059
:10AA8000DBCF1092D52DCF5BDD4F68817981C1542A
:10AA9000D240C70132DB2091F62D222309F495C262
:10AAA000E091AD2FF091AE2F0284F385E02DE058B8
:10AAB000F10954E0F695E7955A95E1F7E35AF24D1E
:10AAC00080818F5F80838091D52D803121F40E9419
:10AAD00099261092D52D1092F52D0E94F12E80E529
:10AAE000F7018083118262E070E0C7010E94424159
:10AAF00081E08093F52D1092F62D60E270E0C701A1
:10AB00009DD98C019FC2CF5BDD4F68817981C15493
:10AB1000D240C701F2DA2091F62D222309F455C262
:10AB2000D0905C2DDD2009F446C0CF5BDD4F08815D
:10AB30001981C154D2400115110549F410925C2DC0
:10AB40001092F62D1092F52D0E94F12E7BC2023A42
:10AB5000110540F0B801C70142DA01E08027082F53
:10AB600010E002C001E010E0CF5BDD4F6881798129
:10AB7000C154D240C701E5D9CF5BDD4F88839983AB
:10AB8000C154D240012B29F462E1C70192DA892B2A
:10AB900029F0ACEFAD0DA0935C2D2AC0F4E0DF9E50
:10ABA000D0011124A45FB24D80E1F70101900D9214
:10ABB0008A95E1F71DC042E050E06FE474E1CE01F8
:10ABC00001960E944C70E2E5F4E1E4912091E72DBA
:10ABD0003091E82D89819A812817390721F48091D5
:10ABE000E92D8E1729F01092F52D0E94F12EEAC161
:10ABF00080915C2D803109F06AC01092F62D109280
:10AC00005C2D80911B2D10921B2D853009F047C0C3
:10AC100020E130E04CE15DE267E870E0CE010196B2
:10AC20000E94E41067EE73E2CE0181960E94A67046
:10AC300020E130E04CE25DE265E670E0CE01839613
:10AC40000E94E41067EE73E2CE018D5B9F4F0E947D
:10AC5000A67020E130E04CE35DE263E470E0CE01F9
:10AC60008B5B9F4F0E94E41067EE73E2CE018B591D
:10AC70009F4F0E94A67020E130E04CE45DE261E26B
:10AC800070E0CE0189599F4F0E94E4100E943A263D
:10AC9000BE016F5F7F4F85E60E94A32593C10E948E
:10ACA0003A2620E430E040E050E0BA018CE19DE239
:10ACB0000E9485136FE074E285E60E94A32581E07F
:10ACC0000E9441100E94EE120E949E197BC190E3E7
:10ACD000D7019C9311968C9362E070E0C7010E94AB
:10ACE000424180915C2D8C5F80935C2D06CFBE012C
:10ACF0006F5B7D4FC70118DB882309F4E6C08091A4
:10AD0000D72D811103C063E274E213C08130A9F42E
:10AD10006091D82DB7E66B9FB00111246F5B7C4E1C
:10AD200040E450E0CE0101960E944C70BE016F5F7E
:10AD30007F4F85E60E94A32568C0912C80E090E0BB
:10AD400000E010E027E6822E7E013FEFE31A3DEFA0
:10AD5000F30A36E3A32E34E2B32EC12C42E0D42E04
:10AD60002091D72D921680F50130E2E01E0720F0E9
:10AD7000081B190BF12C2EC0E92DF0E0E852F24D22
:10AD80006081869EB00111246F5B7C4E40E450E0F0
:10AD9000C7010E944C70FF92EF92BF92AF92C60122
:10ADA000801B910B9F938F9381E090E08C0F9D1FF0
:10ADB000800F911F9F938F930E94AD70080F191FF2
:10ADC0009394CDBFDEBFCCCF0130A2E01A0780F64E
:10ADD000FF24F394EDEFFFEFEC0FFD1FE00FF11FE9
:10ADE0008EE28083EEEFFFEFEC0FFD1FE00FF11F0F
:10ADF0001082BE016F5F7F4F85E60E94A325F11090
:10AE000004C085EB92E10E94C71B8EEA92E10E948A
:10AE1000C71B62E070E087EE9DE20E94C12588EAD0
:10AE200092E10E94C71B6091F42D70E08AEE9DE2D2
:10AE30000E94C12582EA92E10E94C71B61E070E096
:10AE400089EE9DE20E94C12537C0BE016F5B7D4F38
:10AE5000C7016ADA8823C9F18091D72D813039F58D
:10AE60008091D82D833009F4BFC028F4813059F087
:10AE7000823099F0E1C08A3031F008F4DDC08D50A5
:10AE8000823058F0D9C08091F42D843009F4AEC0DE
:10AE9000873009F0D1C017E0ACC08091F42D843028
:10AEA00009F4A6C0873009F0C7C019E0A2C06DE35D
:10AEB00074E285E60E94A32510921B2D1092D72DD7
:10AEC0000E943A261092F62D7DC0CF5BDD4F08819F
:10AED0001981C154D240B6C01092D62D211531052A
:10AEE00009F475C0CF01089636952795820F931FF8
:10AEF00054E0880F991F5A95E1F70E948E26E09141
:10AF0000AD2FF091AE2F62857385CF01825A9F429B
:10AF10008F5F9F4F0E940F7760E070E085E60E9490
:10AF2000A3250115184008F455C0B8E7AB2EB12C85
:10AF30000DE51DE260E8E62EF12C75E0872E74E247
:10AF4000972EEAE05E2EFE0131966F01FBE06F2E38
:10AF5000F4E27F2EFF92EF929F928F921F925F9268
:10AF6000DF92CF920E94AD70C6010E94C21BD80131
:10AF70008C91CDBFDEBF882389F11F928F937F9282
:10AF80006F921F925F92DF92CF920E94AD70C601C6
:10AF90000E94C21BCDBFDEBF87E193E10E94C71BA9
:10AFA000D8011D928D01B0E1EB0EF11CC8018D5549
:10AFB0009D428A159B0570F21092F62D10921B2D62
:10AFC0000E94F82E00E010E03DC08C013BC00E94C2
:10AFD000A92695CFA8E2AA2EB12CAACF6DE283E0D4
:10AFE00090E20E94526ED8CF11E003C016E001C07B
:10AFF00018E063E674E285E60E94A325812F0E9493
:10B000004110E091992FF0919A2F1995E091A32F7B
:10B01000F091A42F8AEE9DE21995E091AA2FF0916C
:10B02000AB2F4091A72F6AEE7DE283E119950E9434
:10B03000EE120E949E1940CF6EE674E23ACF911153
:10B04000DFCCECCCC801CE5BDD4FCDBFDEBFDF91E6
:10B05000CF911F910F91FF90EF90DF90CF90BF9015
:10B06000AF909F908F907F906F905F90089581E058
:10B070008093702EE091AD2FF091AE2F8285938555
:10B08000809320209093212008951092702E10928A
:10B09000F72D089508950895F8CF0F931F93CF9338
:10B0A000DF93CDB7DEB72A97CDBFDEBF2091F72D56
:10B0B000213009F023C18C018091702E833009F476
:10B0C00046C028F4813061F08230D1F017C185305C
:10B0D00009F451C008F474C0863009F497C00EC159
:10B0E00088E0809306068091882E811107C1F801BF
:10B0F0008081863219F0823509F000C182E074C087
:10B100008091882E8130B1F46231710599F4F80193
:10B11000808185FD0FC08181807E61F4828180FD08
:10B1200009C062E170E0C8010E94EF4F882311F06E
:10B1300083E05AC08091882E811159C0F801808126
:10B14000863209F4DBC0823509F051C0D7C0809146
:10B15000882E81114CC06031710509F048C0F8019A
:10B160008081982F907F903909F041C0897081309B
:10B17000F1F585E039C08091882E813061F46D321F
:10B18000710549F46DE270E0C8010E94EF4F882319
:10B1900011F084E029C081E08093702E88E08093D4
:10B1A00006068091202090912120811528E09207A9
:10B1B00008F493C060E070E088E70E94A3259EC079
:10B1C0008091882E811113C06834710581F4F801D3
:10B1D0008081982F907F903951F48970813039F4B3
:10B1E0008181803721F486E08093702E87C081E0D2
:10B1F0008093702E88E080930606809120209091A5
:10B2000021208115F8E09F07A8F667C08091882E5D
:10B21000813009F053C06B31710509F04FC06BE10B
:10B2200070E0C8010E94EF4F882309F447C0F8017D
:10B23000808182FD7DCF81E08093702E88E08093B5
:10B240000506E0912020F0912120E058F10994E0DA
:10B25000F695E7959A95E1F7E850F24D80818F5F7A
:10B26000808360E070E085E60E94A3258091212024
:10B270008F93809120208F9385E094E29F938F930A
:10B280001F928AE08F938E010F5F1F4F1F930F93C2
:10B290000E94AD70C8010E94C21BE091AD2FF091D9
:10B2A000AE2F62857385CF01825A9F428F5F9F4F79
:10B2B0000E940F77EADECDBFDEBF20C081E0809321
:10B2C000702E88E0809306068091202090912120A6
:10B2D0008115E8E09E0708F06DCFFC01E058F10908
:10B2E00084E0F695E7958A95E1F7E850F24D1082F3
:10B2F0000E949926809320209093212080E090E066
:10B300002A96CDBFDEBFDF91CF911F910F91089597
:10B310001F920F920FB60F92112408B60F9218BE0B
:10B320000BB60F921BBE8F93EF93FF93E0E0F9E013
:10B3300080E4848780E3878310922A06FF91EF914F
:10B340008F910F900BBE0F9008BE0F900FBE0F9005
:10B350001F9018951F920F920FB60F92112408B6E6
:10B360000F9218BE0BB60F921BBE2F933F938F9375
:10B370009F93EF93FF9393B120912806267081E06D
:10B3800009F080E0990F892B83B986B197B10196B6
:10B3900086B997B9089709F0C9C016B817B880914F
:10B3A0007B2E8130E9F020F0823009F44EC0BEC01F
:10B3B00083B18B3749F481E080937B2E1092732EFA
:10B3C0001092742E12B8B2C083B18E3709F079C0D2
:10B3D00082E080937B2E1092732E1092742EA6C062
:10B3E00083B18F3DB1F183B18095803439F482B15E
:10B3F0008F5F82B980B18695869521C0803149F4EE
:10B4000082B18F5F82B980B18695869580B9069AA0
:10B4100017C0843049F482B18F5F82B980B18695BC
:10B42000869580B9079A0CC0813051F482B18F5F44
:10B4300082B980B18695869580B980B1806C80B9DB
:10B4400082B1843009F072C062C083B18F3D09F0CF
:10B4500040C080E094E08093772E9093782E809186
:10B460000F32982F927081FF06C020E031E02093C8
:10B47000772E3093782E80FF0BC020EF33E020939F
:10B48000752E3093762E992359F08CEF90E004C0FE
:10B490008091772E9091782E8093752E9093762EB2
:10B4A0001092030A80E280930C0A8CE08093070AD2
:10B4B0008091772E9091782E01978093360A909301
:10B4C000370A81E080937D2E1092000910920709BF
:10B4D0002DC08091732E9091742E9695879523B1EF
:10B4E0002095203411F484500BC0203111F4835086
:10B4F00007C0243011F4825003C0213029F4815058
:10B5000080B982B18F5F82B982B1813079F412B88B
:10B51000E8B1F9B180B1808388B199B1019688B959
:10B5200099B98091792E8F5F8093792E8091732EB7
:10B530009091742E01968093732E9093742EFF91A8
:10B54000EF919F918F913F912F910F900BBE0F9094
:10B5500008BE0F900FBE0F901F90189581B18823E1
:10B5600009F459C181B18C3008F055C1E1B1F0E066
:10B57000EE0FFF1FE055FC4D0190F081E02D199476
:10B580008DE180937A2E14B815B880917A2E87FFBA
:10B5900002C08E9A01C08E988EE080934008809100
:10B5A0007A2E880F80937A2E84B195B1019684B952
:10B5B00095B984B195B187709927892B11F483E0EF
:10B5C00082C082E01BC180917A2E80FF02C08E98DB
:10B5D00001C08E9A84E012C180917A2E80FF02C051
:10B5E0008E9A01C08E9880917A2E869580937A2EBD
:10B5F00084B195B1019684B995B983E081B984B1DC
:10B6000095B187709927892B09F005C18091792E12
:10B6100081508093792E8111B6C088EB80937A2E69
:10B6200018C080917A2E87FF02C08E9A01C08E9832
:10B6300080917A2E880F80937A2E84B195B10196ED
:10B6400084B995B984B195B187709927892B09F48C
:10B65000D2C085E0D3C08DE180937A2E14B815B89E
:10B660008E9A8EE08093400880917A2E87FF0BC0DF
:10B670008FE190E080936608909367088091772E21
:10B680009091782E0AC08BE190E0809366089093A9
:10B6900067088091752E9091762E01978093260AE7
:10B6A0009093270A80917A2E880F80937A2E84B106
:10B6B00095B1019684B995B984B195B187709927F0
:10B6C000892B19F488E081B95EC087E097C080912A
:10B6D0007A2E80FF0BC08BE190E0809366089093F8
:10B6E00067088091752E9091762E0AC08FE190E0C8
:10B6F00080936608909367088091772E9091782EBA
:10B7000001978093260A9093270A89E077C0809159
:10B710007A2E80FF0BC08FE190E0809366089093B3
:10B7200067088091772E9091782E0AC08BE190E087
:10B7300080936608909367088091752E9091762E7D
:10B7400001978093260A9093270A80917A2E8695F6
:10B7500080937A2E84B195B1019684B995B988E029
:10B7600081B984B195B187709927892B09F053C0AD
:10B770008091792E81508093792E811104C088EBBD
:10B7800080937A2E3AC0E8B1F9B1CF01019688B919
:10B7900099B9808180937A2E089580917A2E87FFBF
:10B7A0000BC08FE190E080936608909367088091CA
:10B7B000772E9091782E0AC08BE190E080936608F6
:10B7C000909367088091752E9091762E01978093C3
:10B7D000260A9093270A80917A2E880F80937A2EDA
:10B7E00084B195B1019684B995B984B195B187704A
:10B7F0009927892B11F48BE001C08AE081B9089563
:10B800001092000A1092070A109240081092410804
:10B8100081E080937E2E08958FE092E388B999B9F4
:10B82000EDE7FEE21082118210927B2E11B810B863
:10B8300013B816B817B81092732E1092742E12B84F
:10B840001092792E10927A2EA0E2B6E081E0159641
:10B850008C931597E0E0F9E010A211A28FE790E039
:10B8600086A397A381E390E084A795A782E08083D5
:10B8700098E8938320E424871782E0E0FAE093833A
:10B880002FE531E126AB37AB168217829EE090831D
:10B8900093E01C969C931C971A968C930895CF93D3
:10B8A000DF93E0E4F6E0128A84E08283C0E8D1E02E
:10B8B00082E68E83A0E2B6E081E016968C9316971E
:10B8C00011968C93119796E012969C93129751962D
:10B8D0008C93519732E052963C9352971A961C9251
:10B8E0001A971B961C921B979FE019969C9399E5BB
:10B8F00098832AE529839A8390E491839683A0EB29
:10B90000B0E012962C911297207F12962C931297EA
:10B9100012962C911297226012962C9320E3218389
:10B920002683908B8683358383E08183E0E0F8E093
:10B9300083E1818321E030E026A337A320A731A74C
:10B94000E0E8F8E014868083E0E2F3E013821182FD
:10B9500088E0828391E19083A091AD2FB091AE2FCA
:10B960001A962D913C911B97208F318FE0E8F3E0E0
:10B970009CE392838083938381838AEA99E5809311
:10B980008B2E90938C2E88E899E580938D2F909341
:10B990008E2F8EEA9AE58093892E90938A2EDF91DE
:10B9A000CF913ACFA0E2B6E01A961C921A978FE098
:10B9B00092E388B999B9EDE7FEE210821182109204
:10B9C0007B2E11B810B813B816B817B81092732E92
:10B9D0001092742E12B81092792E10927A2EE0E006
:10B9E000F9E010821382178280E48487E0E0FAE0B5
:10B9F0001382178280E28487E0E4F8E010821182EB
:10BA000081E016968C938E9808950F931F93CF9391
:10BA100080917D2E882309F47EC010927D2E409166
:10BA2000792E042F10E00115110509F46FC0E09183
:10BA3000AA2FF091AB2F6FE072E380E41995E091AB
:10BA4000AD2FF091AE2F8781883019F483E1809378
:10BA5000932C8681883019F483E18093922CC091D5
:10BA60000F32C170E0919F2FF091A02FB8018FE0AD
:10BA700092E319958C01009709F448C0E091AA2F30
:10BA8000F091AB2F482F6FE072E381E41995E091BC
:10BA9000AD2FF091AE2F8781893019F483E1809327
:10BAA000932C8681893019F483E18093922C009342
:10BAB000792E8FE092E388B999B9109260081092BC
:10BAC0006108CC2389F08BE190E080936608909325
:10BAD00067088EE090E080936A0890936B0883E299
:10BAE0008093410886E010C08FE190E08093660863
:10BAF0009093670880E190E080936A0890936B08C8
:10BB000083E28093410881E081B905C01092000A68
:10BB10001092070A81DE80917E2E882331F01092E8
:10BB20007E2ECF911F910F9177CECF911F910F91C4
:10BB300008951092802E08951092802E08950895F1
:10BB40000895EF92FF920F931F93CF93DF93CDB79A
:10BB5000DEB72997CDBFDEBF6430710518F480E0F1
:10BB600090E0C8C08C0162507109BED48823B9F33B
:10BB7000F80121814091A72F50E060E070E0CE01F4
:10BB8000019629870E948D118091802E2985882316
:10BB900021F0823009F46CC0A2C02130B9F4F80160
:10BBA00010821182888582838F8183838E81848332
:10BBB0008D8185838C8186838B8187838A81808731
:10BBC000898181879AE0E92EF12C8DC0223041F5E0
:10BBD000F801808185FF20C09281888598137FC0FD
:10BBE00093818F8198137BC094818E81981377C045
:10BBF00095818D81981373C096818C8198136FC045
:10BC000097818B8198136BC090858A81981367C048
:10BC100091858981981363C082E08093802E5FC0F4
:10BC20002B3209F05CC0F801808185FFB8CF92818A
:10BC30008885981354C093818F81981350C0948144
:10BC40008E8198134CC095818D81981348C0968140
:10BC50008C81981344C097818B81981340C0908544
:10BC60008A8198133CC091858981981338C097CFF9
:10BC70002632A9F54091A72F50E060E070E0CE0198
:10BC800001960E948D11F801808185FF20C092816C
:10BC90008885981324C093818F81981320C0948144
:10BCA0008E8198131CC095818D81981318C0968140
:10BCB0008C81981314C097818B81981310C0908544
:10BCC0008A8198130CC091858981981308C0F80166
:10BCD00010821092802EEE24E394F12C04C0E12C0B
:10BCE000F12CC70107C0B701C801EED3F2E0EF0E97
:10BCF000F11CF7CF2996CDBFDEBFDF91CF911F9109
:10BD00000F91FF90EF9008954091A72F50E060E0D1
:10BD100070E00C948D114091A72F50E060E070E02E
:10BD20000C94DB111092812E08951092812E0895AB
:10BD3000089508956F927F929F92AF92BF92CF9293
:10BD4000DF92EF92FF920F931F93CF93DF93CDB7C4
:10BD5000DEB72A97CDBFDEBF8C016430710518F4C1
:10BD600080E090E0C7C162507109BED38823C1F35F
:10BD7000F80121814091A72F50E060E070E0CE01F2
:10BD8000019629870E948D118091812E2985882313
:10BD900021F0823009F474C1AAC12130B1F4F80154
:10BDA00010821182888582838F8183838E81848330
:10BDB0008D8185838C8186838B8187838A8180872F
:10BDC000898181874AE050E087C1223041F5F8013E
:10BDD000808185FF20C092818885981388C19381D6
:10BDE0008F81981384C194818E81981380C195812D
:10BDF0008D8198137CC196818C81981378C197812D
:10BE00008B81981374C190858A81981370C1918534
:10BE1000898198136CC182E08093812E68C12B3296
:10BE200009F042C0F8019081888595FF1FC092817A
:10BE300098135DC123819F81291359C124819E815B
:10BE4000291355C125819D81291351C126819C81CA
:10BE500029134DC127819B81291349C120859A81CE
:10BE6000291345C121859981291341C1F801108207
:10BE70009FE0918382838F8183838E8184838D81F0
:10BE800085838C8186838B8187838A818087898162
:10BE90008187128682EC838783E08487858781E0AF
:10BEA00086874FE050E018C1203209F045C0F80104
:10BEB000808185FF20C022819885291318C12381A4
:10BEC0009F81291314C124819E81291310C12581CA
:10BED0009D8129130CC126819C81291308C12781CA
:10BEE0009B81291304C120859A81291300C12185D2
:10BEF00099812913FCC0F801628570E086FF0FC0AC
:10BF000010821182660F771F660F771F44E050E0A2
:10BF1000C80102960E948D1146E050E0DDC01192EA
:10BF2000CF01660F771F660F771F44E050E00E9435
:10BF30008D1145E050E0D0C0233209F06AC0F8010D
:10BF4000808185FF20C0228198852913D0C023815C
:10BF50009F812913CCC024819E812913C8C02581CB
:10BF60009D812913C4C026819C812913C0C02781CB
:10BF70009B812913BCC020859A812913B8C02185D3
:10BF800099812913B4C0F8016285E384F12CFFEF95
:10BF9000EF1AFF0A58019FEFA91AB90A70E086FF4D
:10BFA00026C06B01CC0CDD1CCC0CDD1C612C712C73
:10BFB000912C892D90E08E159F0590F4F50111923A
:10BFC000CF01B3016C0D7D1D44E050E00E948D1146
:10BFD000F5E0AF0EB11C939484E0680E711CE9CFBC
:10BFE00085E08E9DA0018F9D500D11240DC0EE0C9B
:10BFF000FF1CEE0CFF1C660F771F660F771FA70153
:10C00000C5010E948D11A7014F5F5F4FF80110829B
:10C0100063C02C3209F06BC0F801808185FF20C01D
:10C0200092818885981363C093818F8198135FC034
:10C0300094818E8198135BC095818D81981357C030
:10C0400096818C81981353C097818B8198134FC030
:10C0500090858A8198134BC091858981981347C038
:10C06000F80143854F5F1082902FF8018E2F891BB6
:10C07000841710F41192FACF50E04F5F5F4F2CC03D
:10C080002632A9F5F801808185FF20C0928188853C
:10C0900098132DC093818F81981329C094818E812C
:10C0A000981325C095818D81981321C096818C812C
:10C0B00098131DC097818B81981319C090858A8130
:10C0C000981315C091858981981311C0F8011082C9
:10C0D0001092812E41E050E0BA01C80149875A8789
:10C0E000F3D149855A854E5F5F4FCA0103C040E0D6
:10C0F00050E0FBCF2A96CDBFDEBFDF91CF911F91DD
:10C100000F91FF90EF90DF90CF90BF90AF909F90F6
:10C110007F906F9008954091A72F50E060E070E00D
:10C120000C948D114091A72F50E060E070E00C94CA
:10C13000DB111092862E8091822E9091832E936037
:10C140008093822E9093832EE0E1F4E3108211829B
:10C15000128213821482158216821782108641E0A1
:10C1600050E068E270E08FE094E30C948D1110923F
:10C17000862EE0E1F4E3108211821282138214828F
:10C180001582168217821086089508950895E09109
:10C19000A72FF0E03197E80FF91FDC01AE17BF07BA
:10C1A00030F48C9190819D9380833197F7CF0895DF
:10C1B000CF93DF93EC014091A72F50E060E270E055
:10C1C0000E948D11CE01DF91CF91E1CF6F927F92CE
:10C1D0008F929F92AF92BF92CF92DF92EF920F9386
:10C1E0001F93CF93DF93CDB7DEB76C013B018DB6C4
:10C1F0009EB68091A72F2DB73EB7281B31092DBFC2
:10C200003EBF8DB79EB701965C01D2DF94E0691600
:10C21000710408F41AC1B30162507109C60164D1F6
:10C22000882309F412C121E08091862E813009F023
:10C2300020E0E0900F34850140E154E3B301C601F2
:10C2400069D1882309F401C18091862E8111FDC036
:10C25000E0911234F09113348081813031F5F60190
:10C2600010821182F5018781F6018283F5018681B2
:10C27000F6018383F5018581F6018483F5018481CC
:10C28000F6018583F5018381F6018683F5018281BC
:10C29000F6018783F5018181F6018087F5018081B0
:10C2A000F60181870AE010E0CAC0823041F4909123
:10C2B0001734992309F4BDC08093862EC6C08032FE
:10C2C00009F047C0E0911434F091153460818091F9
:10C2D0001634813009F0B9C0F6016B3018F0808354
:10C2E00080E1AAC0808186FF25C081E090E0062E13
:10C2F00002C0880F991F0A94E2F72091822E309194
:10C30000832E28233923232B11F082E00AC02091A9
:10C31000842E3091852E82239323892B21F081E076
:10C32000F601818302C0F6011182C601029606E081
:10C3300010E004C0C601019605E010E0F60110828D
:10C34000F4E06F9FB001112444E050E00E948D1191
:10C3500076C08132C9F58091143490911534FC0176
:10C36000608120911634253009F06FC06C3028F0C0
:10C3700081E0F601808383E05FC021E030E0062E9B
:10C3800002C0220F331F0A94E2F74091822E50918F
:10C39000832E42235323452B59F74091842E5091ED
:10C3A000852E24233523232B29F081E0F601808379
:10C3B00082E142C0F4E06F9FB001112444E050E0FC
:10C3C00001960E94DB1130C0823299F5E09114345D
:10C3D000F09115342081809116348130B1F52C30E4
:10C3E00038F681E090E002C0880F991F2A95E2F7A5
:10C3F0002091822E3091832E28233923232B49F438
:10C400002091842E3091852EAC0142235323452B5D
:10C4100029F081E0F601808381E10EC0822B932B0D
:10C420008093842E9093852EF601108201E010E017
:10C4300006C081E0F6018083818302E010E0B8014C
:10C44000C60142D0C801029602C080E090E08DBED5
:10C450009EBEDF91CF911F910F91EF90DF90CF9013
:10C46000BF90AF909F908F907F906F900895CF93E3
:10C47000DF93EC018CDE4091A72F50E060E270E08A
:10C48000CE01DF91CF910C94DB11A82FFC018FEF2F
:10C490009FEF2E2F2A1B30E02617370790F42191AB
:10C4A000822728E0AC015695479580FF06C0CA0157
:10C4B00038E0832734E8932701C0CA01215091F75F
:10C4C000E8CF8095909508950F931F93CF93DF93B6
:10C4D0008C01EB01DADFC00FD11F88839983DF91D4
:10C4E000CF911F910F9108950F931F93CF93DF93D7
:10C4F0008C01EB01CADFC00FD11F2881281303C0B4
:10C5000081E02981291380E08170DF91CF911F9113
:10C510000F910895EF920F931F93CF93DF93DC0158
:10C52000FA01E801808391830196828393838C9141
:10C5300082FD09C085FB882780F987838C918295CD
:10C540008170808702C0178210863781CD01332326
:10C5500011F00A9601C002968483958311968C91FE
:10C560001197803A40F012969C9112978981981702
:10C5700061F080E04AC0813069F48C9184FF0AC088
:10C5800012968C9112978E11F4CF84819581019629
:10C59000848395834481558162507109A60FB71F2A
:10C5A000A41BB50BA683332349F1DA0118979C919C
:10C5B0008F819813DECF11969C918E819813D9CFDD
:10C5C00011969C918D819813D4CF11969C918C815A
:10C5D0009813CFCF11969C918B819813CACF119647
:10C5E0009C918A819813C5CF11969C91898198134B
:10C5F000C0CF11969C9188819813BBCF80858823EA
:10C6000019F0211102C0B5CF81E0DF91CF911F91C8
:10C610000F91EF9008950F931F93CF93DF93CDB7B2
:10C62000DEB72897CDBFDEBFF90187818983868178
:10C630008A8385818B8384818C8383818D838281AE
:10C640008E8381818F8380818887FA01A481B5815F
:10C650002D91822F8695869586958E010F5F1F4FAF
:10C66000BD01A801942F901B981748F4FA0131914D
:10C67000AF01FB019191BF013917A1F317C0892FB9
:10C6800090E0A80FB91FF801E80FF91F9C91808175
:10C69000392F3827277081E090E001C0880F2A9554
:10C6A000EAF78150932F982381E009F080E02896E3
:10C6B000CDBFDEBFDF91CF911F910F9108951092F2
:10C6C000872EE0E1F4E31082118212821382148239
:10C6D00015821682178210861092193441E050E0BC
:10C6E00068ED70E08FE094E30C948D111092872E2A
:10C6F000E0E1F4E310821182128213821482158227
:10C70000168217821086109219340895089508959C
:10C71000FF920F931F93CF93DF931F92CDB7DEB796
:10C72000E0911434F0911534F08019820F2D10E04F
:10C7300000521F4F41E050E0B801CE0101960E9427
:10C740008D1180911634813071F494E39F1558F067
:10C750009981911108C0898341E050E0B801CE0170
:10C7600001960E94DB1180E090E00F90DF91CF9165
:10C770001F910F91FF900895CF92DF92EF92FF9259
:10C780000F931F93CF93DF931F92CDB7DEB7C09067
:10C790001434D0901534F60100811982209116349A
:10C7A000253019F080E090E01FC00533D8F77C01F8
:10C7B00010E0B80160527F4F41E050E0CE01019699
:10C7C0000E948D119981937069F7B801660F771FE8
:10C7D000660F771F44E050E0C60101960E94DB110E
:10C7E000F701108281E090E00F90DF91CF911F91CF
:10C7F0000F91FF90EF90DF90CF900895CF92DF924E
:10C80000EF92FF920F931F93CF93DF931F92CDB7B9
:10C81000DEB7E0911434F091153460811982F09004
:10C82000163421E0F21244C0643358F020911734DA
:10C830002223F1F1FC01F0822FE0218382E090E0DD
:10C8400039C08C01FC018081C62ED12C86FF1BC013
:10C8500041E050E0B60160527F4FCE0101960E9448
:10C860008D11898181FF04C082E0F801818305C0B8
:10C87000F80180FF06C0F18282E0EE24E394F12CFF
:10C8800005C01182F9CF81E0E12CF12CB601660FD1
:10C89000771F660F771F44E050E09801280F311D85
:10C8A000C9010E948D11F8011082C701059602C0CE
:10C8B00080E090E00F90DF91CF911F910F91FF905A
:10C8C000EF90DF90CF9008953F924F925F926F92DA
:10C8D0007F928F929F92AF92BF92CF92DF92EF9210
:10C8E000FF920F931F93CF93DF93CDB7DEB77C01F9
:10C8F0004DB65EB6E0911434F091153480813180EC
:10C9000090911634923009F0A3C0843370F0809176
:10C910001734882309F49CC081E0D7018C938FE001
:10C9200011968C9382E090E095C03394A82EB12CA0
:10C930009501230D311D243331051CF094E3392E6C
:10C94000381AF7018081032D10E086FD0FC0000F1B
:10C95000111F000F111FB501660F771F660F771F9C
:10C96000A801C70101960E948D116DC06DB67EB6FB
:10C97000A801440F551F440F551F8DB79EB7841B48
:10C98000950B8DBF9EBFADB7BEB711966D01EDB7CC
:10C99000FEB7E01BF10BEDBFFEBF8DB79EB7019652
:10C9A0004C01B501660F771F660F771FCD010E94FE
:10C9B0008D11B50160527F4FA801C4010E948D11F5
:10C9C000F40100E081E0B4E0CB0ED11C0315A9F125
:10C9D0009191D701A80FB11D9C9391E0980FA701E9
:10C9E000490F511D960124503109D9019C91DA015A
:10C9F0009C9392E0980FA701490F511D2F5F3F4F65
:10CA0000D9019C91DA019C9393E0980FA701490FFB
:10CA1000511D2F5F3F4FD9019C91DA019C9394E007
:10CA2000980FA701490F511D8B5F2F5F3F4FD90111
:10CA30009C91DA019C930F5FC6CFE5E00E9F8001C9
:10CA400011246DBE7EBED7011C92C801019602C0A2
:10CA500080E090E04DBE5EBEDF91CF911F910F91BF
:10CA6000FF90EF90DF90CF90BF90AF909F908F900E
:10CA70007F906F905F904F903F900895CF93DF939A
:10CA80001F921F92CDB7DEB7E0911434F0911534A8
:10CA900080818A831982809116348130B1F441E01B
:10CAA00050E06CED70E0CE0101960E948D118981FD
:10CAB00080FD0BC041E050E068ED70E0CE010296D1
:10CAC0000E94DB118A8180930F3480E090E00F9008
:10CAD0000F90DF91CF910895CF93DF931F92CDB741
:10CAE000DEB7198280911634811115C041E050E003
:10CAF0006CED70E0CE0101960E948D11898180FD60
:10CB00000AC08160898341E050E06CED70E0CE01A5
:10CB100001960E94DB1180E090E00F90DF91CF91B1
:10CB20000895CF93DF931F921F92CDB7DEB7E091A8
:10CB30001434F091153480818A83198280911634DF
:10CB4000813099F441E050E06CED70E0CE01019647
:10CB50000E948D11898181FD08C041E050E069ED9E
:10CB600070E0CE0102960E94DB1180E090E00F9011
:10CB70000F90DF91CF910895CF93DF931F92CDB7A0
:10CB8000DEB7198280911634811115C041E050E062
:10CB90006CED70E0CE0101960E948D11898181FDBE
:10CBA0000AC08260898341E050E06CED70E0CE0104
:10CBB00001960E94DB1180E090E00F90DF91CF9111
:10CBC00008950F931F93CF93DF93E0911434F09166
:10CBD00015342081C181309116343230D1F425339F
:10CBE000C0F4CF5F622F70E0AB014C0F511D443396
:10CBF000510514F0C4E3C21B8C01D0E060527F4F9A
:10CC0000AE0101960E948D11F8011082CE010196AD
:10CC100002C080E090E0DF91CF911F910F910895C5
:10CC2000FC01DA01928117968C911797981328C00E
:10CC3000938116968C911697981322C0948115961D
:10CC40008C91159798131CC0958114968C9114970C
:10CC5000981316C0968113968C911397981310C051
:10CC6000978112968C91129798130AC0908511960D
:10CC70008C911197981304C081E021859C91291310
:10CC800080E0908195FF12C094FD10C0811103C017
:10CC90001092872E0BC08091872E8130C9F381E0DE
:10CCA0008093872E108281E090E0089580E090E0EC
:10CCB0000895E0E1F4E3108211821282138214825B
:10CCC00015821682178210861092872EFC01108220
:10CCD00081E090E00895FF920F931F93CF93DF932D
:10CCE00000D01F92CDB7DEB719821A821B821C8238
:10CCF00020911634243049F520911734222329F14C
:10CD000020911834222309F1F090872E21E0F212AD
:10CD10001CC08C0144E050E064E171E0CE0101965A
:10CD20000E948D11F092193444E050E064E171E00A
:10CD300080911434909115340E94DB11F0921934D3
:10CD4000F801108281E090E002C080E090E024963B
:10CD5000CDBFDEBFDF91CF911F910F91FF9008955E
:10CD6000FC0180911634813059F4108211821282B4
:10CD70001382148215821682178288E090E008954B
:10CD800080E090E00895209116342B3049F4FC01A6
:10CD9000119263E0CF010E94CB1084E090E00895EF
:10CDA00080E090E008954091A72F50E060ED70E0A2
:10CDB0000C948D11CF92DF92EF92FF920F931F93FD
:10CDC000CF93DF93CDB7DEB78C01CDB6DEB68091C1
:10CDD000163481114AC08FE0F80181838091A72F1A
:10CDE0002DB73EB7281B31092DBF3EBF8DB79EB76B
:10CDF00001967C01D8DFF7018781F8018283F70172
:10CE00008681F8018383F7018581F8018483F70126
:10CE10008481F8018583F7018381F8018683F70116
:10CE20008281F8018783F7018181F8018087F7010A
:10CE30008081F801818741E050E069ED70E0C80130
:10CE40000A960E948D1141E050E068ED70E0C80143
:10CE50000B960E948D1183E3F801848783E0858718
:10CE600082E0868710828FE001C080E0CDBEDEBE0A
:10CE7000DF91CF911F910F91FF90EF90DF90CF90B6
:10CE800008956F927F928F929F92AF92BF92CF92AE
:10CE9000DF92EF920F931F93CF93DF93CDB7DEB75F
:10CEA0006C015B016DB67EB68091A72F2DB73EB7A2
:10CEB000281B31092DBF3EBF8DB79EB701964C018F
:10CEC00072DF94E0A916B10418F480E090E0E6C0A7
:10CED000B50162507109C60107DB8823B1F3F60181
:10CEE0008181853231F4A401B501C60199DE8C013E
:10CEF00012C021E08091872E813009F020E0E0907F
:10CF00000F34840140E154E3B501C60103DB8823FB
:10CF1000E1F200E010E08091872E823008F0ACC092
:10CF2000E0911234F091133480818130C9F5809101
:10CF30001634882351F2940140E154E3B501C6014F
:10CF40006ADB882309F4A1C0F6011192CF0141E008
:10CF500050E069ED70E00E948D11F4018781F601C7
:10CF60008283F4018681F6018383F4018581F601D1
:10CF70008483F4018481F6018583F4018381F601C1
:10CF80008683F4018281F6018783F4018181F601B1
:10CF90008087F4018081F6018187065F1F4F75C08D
:10CFA000823041F490911734992309F45AC0809348
:10CFB000872E6BC0803221F4B501C6011FDC05C08D
:10CFC000813229F4B501C601D7DB8C015EC0823203
:10CFD00021F4B501C6019CDBF8CF833221F4B50101
:10CFE000C60172DCF2CF873221F4B501C60146DDFD
:10CFF000ECCF883221F4B501C6016EDDE6CF89326F
:10D0000021F4B501C6018DDDE0CF8A3221F4B501EE
:10D01000C601B2DDDACF8B3231F4B501C601CADE0A
:10D02000082F10E032C08C3221F4B501C601C9DDF1
:10D03000CCCF863221F4B501C6013BDEC6CF843E9B
:10D0400021F4B501C60147DEC0CF803E21F4B50111
:10D05000C60186DEBACF813E21F4B501C60193DE5A
:10D06000B4CF80911734882381F081E0F60180836A
:10D07000818302E010E00DC0823039F4E091123477
:10D08000F091133480818632B1F20115110509F453
:10D090001CCFB801C60118DAC80102966DBE7EBE6B
:10D0A000DF91CF911F910F91EF90DF90CF90BF90C4
:10D0B000AF909F908F907F906F9008954091A72F91
:10D0C00050E060ED70E00C94DB11FF920F931F9322
:10D0D000CF93DF93CDB7DEB7EA97CDBFDEBF0FE1C9
:10D0E00014E388E0F82EF00E91D2F80181938F01BD
:10D0F000FE12FACF0E94771C04D3882309F4F7C0EC
:10D1000080911F3490912034953009F46FC030F431
:10D11000913069F168F0933051F1E9C0983009F429
:10D12000C2C0993009F4C8C0963009F0E0C072C09E
:10D13000803891F0823809F0DAC0809123348F7002
:10D1400085D2E0912934F0912A34118112FB112704
:10D1500010F980E07BD206C010911B3480911C3402
:10D1600081111260E8D2812F61D280E0A1C0282F06
:10D170002D7F09F0BCC0882319F0823061F0B7C060
:10D1800080912134813009F0B2C0933009F080E001
:10D1900080931C3427C080912134811123C0E091F9
:10D1A00023341E2F1F7009F4A2C0812F4FD280910B
:10D1B0002034833011F4EBD215C0E0912934F09182
:10D1C0002A3481818B7F818324E8129FF00111240E
:10D1D000E359FB4C1082E0912934F0912A3480818C
:10D1E0008E7F808380E032D2A6D264C081117FC05E
:10D1F000109121341F779FD2A1D35DD28823E9F308
:10D200001093C304111102C082E001C083E0809337
:10D210001E346DC08058823008F069C0809121347E
:10D22000909122348C3DE3E09E0761F583E08A8390
:10D230008AE389834FB7F894DE01139620E038E043
:10D2400052E05093CA01E32FF0E0E4911092CA013A
:10D2500020FF03C0E295EF703F5FEF708E2F90E0EC
:10D26000EA3010F0C79601C0C0968D939D932F5F52
:10D270002C3139F74FBF5FD26AE370E0CE010196DF
:10D28000A3D00FC0AE014F5F5F4F609123340E9467
:10D29000500F8C01892B59F14ED2B80189819A81A6
:10D2A0000FD1A5D124C0803811F545D280911A3410
:10D2B000BDD184D143D31BC0811119C080912134C9
:10D2C0008230A8F438D28091213480931A3436D336
:10D2D00080911A34811106C08091C304811102C06B
:10D2E00081E001C084E080931E340E94731C09D247
:10D2F000882311F020D24BD2EA96CDBFDEBFDF915A
:10D30000CF911F910F91FF9008950895CF93809131
:10D310001E34882351F0C0912B3480E097D1F1D195
:10D320008111D3DE8C2FCF9191C1CF910895CF92EF
:10D33000DF92EF92FF920F931F93CF93DF93EC0155
:10D340008B017A0111D3811136C0E114F10439F057
:10D35000F70180819181081B190BC80FD91FC12CBF
:10D36000D12C0115110531F1809127349091283489
:10D37000FC01EF5BFF4F208131978081281790F0EF
:10D380001DD1C4DFE114F10449F0F70180819181DE
:10D39000C80ED91EC082D18285E00DC0E5D2882397
:10D3A00001F309C0899142D101501109FFEFCF1A51
:10D3B000DF0AD7CF80E0DF91CF911F910F91FF90CF
:10D3C000EF90DF90CF900895DF92EF92FF920F934E
:10D3D0001F93CF93DF93D82FC92F8B0180912B34CC
:10D3E000806834D1209125343091263420173107BC
:10D3F00028F00115110519F4E1D001C08901ED2EC5
:10D40000FC2ED12C0115110509F440C080911E3469
:10D41000811102C082E04CC0853011F483E048C025
:10D4200070D1882311F081E043C051D181113CC0FB
:10D4300042D1882339F320912B3480912734909165
:10D440002834FC0127FF05C0EF5BFF4FC081D0E00F
:10D4500013C0E05CFF4FC08131968081D0E0C81BD3
:10D46000D1090AC0C830D10550F4F70181917F017C
:10D47000DDD00150110921960115110599F7DD2420
:10D48000D394289709F0D12C99D0BCCFD110BECF1E
:10D490000BC080911E34882309F4BCCF853009F479
:10D4A000BDCF2FD18111BFCF12D1882391F380E05E
:10D4B000DF91CF911F910F91FF90EF90DF90089532
:10D4C000DF92EF92FF920F931F93CF93DF93D82FAA
:10D4D000C92F8B0180912B348068B8D020912534DE
:10D4E000309126342017310728F00115110519F461
:10D4F00065D001C08901ED2EFC2ED12C011511053E
:10D5000009F442C080911E34811102C082E04EC0F5
:10D51000853011F483E04AC0F4D0882311F081E013
:10D5200045C0D5D081113EC0C6D0882339F32091A3
:10D530002B348091273490912834FC0127FF05C0BB
:10D54000EF5BFF4FC081D0E015C0E05CFF4FC081B2
:10D5500031968081D0E0C81BD1090CC0C830D105FC
:10D5600060F4F701849162D0FFEFEF1AFF0A0150D7
:10D57000110921960115110589F7DD24D394289707
:10D5800009F0D12C1BD0BACFD110BCCF0BC08091E9
:10D590001E34882309F4BACF853009F4BBCFB1D04B
:10D5A0008111BDCF94D0882391F380E0DF91CF919A
:10D5B0001F910F91FF90EF90DF900895E091293433
:10D5C000F0912A34A0912734B0912834AF5BBF4F3B
:10D5D0008C9190E08283938380818D798083E09128
:10D5E0002734F0912834EF5BFF4F10820895E091CB
:10D5F0002934F0912A3480818D798083E091273419
:10D60000F0912834EF5BFF4F10820895809127340A
:10D6100090912834FC01EF5BFF4F208131E0320F05
:10D620003083FC01E20FF11D8081089520912734A1
:10D6300030912834F901EF5BFF4F908141E0490FB1
:10D640004083F901E90FF11D8083089580932B3405
:10D65000482F4F7050E06091C6047091C7049A0142
:10D6600094E0220F331F9A95E1F7E4E887FF11C099
:10D67000E49FC001E59F900D112482599B4C80933B
:10D68000273490932834C90108969B01280F391F2D
:10D690000DC0E49FC001E59F900D1124845D9B4C5B
:10D6A0008093273490932834260F371F20932934F2
:10D6B00030932A34089580912B348068C7DFE0913D
:10D6C0002934F0912A348081869581700895809163
:10D6D0002B348F77BBDFA0912934B0912A348C9101
:10D6E00085FF0DC0E0912734F091283412968D917A
:10D6F0009C911397E05CFF4F808381E0089580E068
:10D70000089580912B348F77A1DFA0912934B091B7
:10D710002A348C9184FF0DC0E0912734F091283495
:10D7200012968D919C911397E05CFF4F808381E06E
:10D73000089580E0089580912B348F7787DFE09102
:10D740002934F0912A3480818D788083E0912934C6
:10D75000F0912A34808181608083E0912734F091B8
:10D760002834EF5BFF4F108280912B3480686EDF8E
:10D77000E0912934F0912A34808181608083E091A6
:10D780002734F0912834EF5BFF4F10820895E09129
:10D790002934F0912A34818184608183E091293495
:10D7A000F0912A348181807C803459F480912B342B
:10D7B00080584CDFE0912934F0912A3481818460D3
:10D7C000818308951F93CF93DF931F921F92CDB74C
:10D7D000DEB7182F4A83698339DFE0912934F0914D
:10D7E0002A341182E0912934F0912A34812F881F44
:10D7F0008827881F880F8083E0912934F0912A348C
:10D8000069816183E0912934F0912A341282138274
:10D81000209127343091283424833583110F110B44
:10D820004A814123F901E05CFF4F40833196108229
:10D8300081E00F900F90DF91CF911F910895AF92EB
:10D84000BF92CF92DF92EF92FF920F931F93CF93ED
:10D85000DF93A62E8C017C0184E0E80EF11CB12C34
:10D86000BA1409F443C0F801D081DD23C1F1C180AD
:10D87000D280F70131978081F7019081923010F4C6
:10D8800098E001C098E128E030E0C0E02C153D05AB
:10D8900020F4CF5F220F331FF9CFC92B9D2F9F702C
:10D8A000963010F080E023C0CF7EF1E4CF16D10493
:10D8B000C8F7882321F0813021F4C06C0AC0C0640D
:10D8C00003C0C068811105C04C2D6C2F80E88D0FFE
:10D8D00079DF4C2D6C2F8D2F75DF882319F3B394CE
:10D8E0000B5F1F4F85E0E80EF11CBACF81E0DF919E
:10D8F000CF911F910F91FF90EF90DF90CF90BF904D
:10D90000AF90089580E090E0E091C604F091C704E4
:10D910009C0144E0220F331F4A95E1F7E20FF31F09
:10D9200011864091C6045091C704FA01E20FF31F1B
:10D93000118201968630910539F7089580911F3440
:10D9400087FF0DC0C4DE811105C080911E34811196
:10D95000F9CF09C04CCE80911E34882321F0ABDE74
:10D960008823C9F32BCE08950F931F93CF93E09193
:10D97000C604F091C704E05AFF4F00811181C4E64C
:10D9800080912B3487FF0AC096DE811105C08091FB
:10D990001E34811105C021C080E024C098DEF5CF7F
:10D9A0008530E9F0E0912934F0912A34818182FDBB
:10D9B00018C0E091C604F091C704E05AFF4F80817F
:10D9C000918180179107E1F22FEF2C0FCC2319F0F2
:10D9D0008C01C22FD5CF84E005C082E003C083E074
:10D9E00001C081E0CF911F910F91089563D069D05C
:10D9F000E0ECF4E081818E7F818380818F7780836A
:10DA000010921D340895CF93DF93E0E4F0E0148288
:10DA10008481836084834ED054D0C0ECD4E088816C
:10DA20008F77888388818068888310921E34109253
:10DA30001A3410921C3410921B34888180648883BD
:10DA400048E068E480E8BEDE48E068E480E0BADEF2
:10DA5000888580648887898181608983DF91CF91FF
:10DA60000895CF93DF933FB7F894C0ECD1E022E064
:10DA70002A87EAE1F0E0E491A0ECB4E0DA96EC93D6
:10DA8000DA97EBE1F0E0E491DB96EC93DB971A8612
:10DA900085E497E38E7F16968D939C93179785E187
:10DAA0008C9318962C933FBF81E080931D34DF91B7
:10DAB000CF91A9CFE0ECF4E0808583708087118658
:10DAC0000895E0ECF4E08FEF8287848708951F9239
:10DAD0000F920FB60F92112408B60F9218BE09B616
:10DAE0000F9219BE0BB60F921BBE2F933F934F930D
:10DAF0005F936F937F938F939F93AF93BF93EF93B6
:10DB0000FF938091CA0487FF08C08091C80487FFF3
:10DB100004C080E88093CA04F8DB8091CA0486FFC1
:10DB200007C080E48093CA0410921E340E94621CD5
:10DB30008091CA0485FF14C080E28093CA0480915A
:10DB40001A34882311F084E007C08091C304811146
:10DB500002C081E001C083E080931E340E94511C0A
:10DB60008091CA0484FF14C080E18093CA0482E0DB
:10DB700080931E3410921A341092C304C3DE48E01E
:10DB800068E480E81FDE48E068E480E01BDEBDDB7F
:10DB9000FF91EF91BF91AF919F918F917F916F9185
:10DBA0005F914F913F912F910F900BBE0F9009BE47
:10DBB0000F9008BE0F900FBE0F901F901895CF9337
:10DBC000DF93EC01FC0170968BE0DF011D928A95DA
:10DBD000E9F782E08C83898783E08E8761E0CE015C
:10DBE00001962DDE882361F061E0CE01069627DEE6
:10DBF000882331F061E0CE010B96DF91CF911FCEEB
:10DC000080E0DF91CF9108950F931F93CF93DF931F
:10DC100020911E342430E1F4FC0104891589268901
:10DC20003789012B022B032B99F0EB0181810EDD4B
:10DC3000FE0101900020E9F73197BF016C1B7D0BBD
:10DC400040E050E0CE01DF91CF911F910F916FCB5B
:10DC500082E0DF91CF911F910F9108950F931F9351
:10DC6000CF93DF93FC0180911E348430A9F4848922
:10DC70009589A689B789892B8A2B8B2B69F08A0114
:10DC8000EB018181E3DC40E050E0B801CE01DF919F
:10DC9000CF911F910F914BCB82E0DF91CF911F91DC
:10DCA0000F910895CF93FC0180911E34843001F5CB
:10DCB00084899589A689B789892B8A2B8B2BC1F0FA
:10DCC000C62F8181C3DC2091273430912834F9019B
:10DCD000EF5BFF4F908131978081981720F48C2F54
:10DCE000A5DC80E006C06ADC3FDE8823C1F301C00A
:10DCF00082E0CF910895CF93DF9320911E3424309A
:10DD000091F5FC014489558966897789452B462B15
:10DD1000472B49F181819ADC80912B342091273463
:10DD200030912834F90187FF05C0EF5BFF4F8081F8
:10DD300090E008C0E05CFF4F80813196408190E028
:10DD4000841B9109892B69F0F901EF5BFF4FD081AA
:10DD50003197C08133DCDC1720F006DE811104C06E
:10DD60002DDC80E001C082E0DF91CF910895CF9358
:10DD7000DF9320911E34243099F4FC0144895589A5
:10DD800066897789452B462B472B51F0EC01818121
:10DD90005DDC91DC882321F0CE01DF91CF91ABCF08
:10DDA000DF91CF910895CF93DF9320911E342430DB
:10DDB00019F08FEF9FEF46C0FC01448955896689B1
:10DDC0007789452B462B472BA1F386813FDC7FDCEF
:10DDD000882379F380912B34209127343091283493
:10DDE000F90187FF05C0EF5BFF4F808190E008C01D
:10DDF000E05CFF4F80813196208190E0821B910989
:10DE0000892B21F003DCC82FD0E002C0CFEFDFEF79
:10DE100020912B348091273490912834FC0127FFE6
:10DE200005C0EF5BFF4F208130E008C0E05CFF4F92
:10DE300020813196808130E0281B3109232B09F4A1
:10DE4000D6DBCE01DF91CF9108950895FF920F9315
:10DE50001F93CF93DF93EC0154DC882309F48EC029
:10DE6000888190E020912334309124342817390799
:10DE700009F084C080912034813259F018F4803246
:10DE800049F17CC0823209F457C0833209F467C07B
:10DE900075C080911F34813A09F070C04CDC0BDCF6
:10DEA0008823E9F38C89FD880E891F89BFDB8F2DBC
:10DEB000BDDB802FBBDB812FB9DB888DB7DB898D84
:10DEC000B5DB8A8DB3DB7ADBDF91CF911F910F91A8
:10DED000FF9034CD80911F34813209F04FC02BDC8C
:10DEE000F6DB811105C080911E348111F9CF46C047
:10DEF0008DDB082F8BDB182F89DBF82E87DB4F2D6E
:10DF000050E060E070E0BA0155274427782B402BA1
:10DF1000512B4C8B5D8B6E8B7F8B78DB888F76DB08
:10DF2000898F74DB8A8F63DB09DDCE01DF91CF91AE
:10DF30001F910F91FF9089CF80911F348132F1F4AE
:10DF4000FADBFCDC8091213490912234888B998B10
:10DF5000CE01DF91CF911F910F91FF9076CF8091ED
:10DF60001F34813259F4E7DBE9DC60912134CE01C2
:10DF7000DF91CF911F910F91FF9067CFDF91CF91EC
:10DF80001F910F91FF900895AA1BBB1B51E107C081
:10DF9000AA1FBB1FA617B70710F0A61BB70B881F39
:10DFA000991F5A95A9F780959095BC01CD010895C8
:10DFB000B7FF04C003D0821B930B089509D0A59F1F
:10DFC000900DB49F900DA49F800D911D1124089574
:10DFD000A29FB001B39FC001A39F700D811D1124AA
:10DFE000911DB29F700D811D1124911D08958F9276
:10DFF0009F92AF92BF92CF92DF92EF92FF92CF9318
:10E00000DF93EC01688179818A819B8161157105BB
:10E010008105910521F464E279ED8BE597E02DE12E
:10E0200033EF41E050E022D749015A019B01AC0196
:10E03000A7EAB1E4C3DF6B017C01ACEEB4EFA5014C
:10E040009401B8DFDC01CB018C0D9D1DAE1DBF1D01
:10E05000B7FF03C00197A109B04888839983AA83B9
:10E06000BB839F77DF91CF91FF90EF90DF90CF90B0
:10E07000BF90AF909F908F900895B9CF82E290E2C9
:10E08000B6CFA0E0B0E08093222090932320A0930D
:10E090002420B09325200895FB01DC0102C00590E7
:10E0A0000D9241505040D8F70895FB01DC018D914D
:10E0B000059080190110D9F3990B0895FB01DC013B
:10E0C0004150504048F005900D920020C9F701C022
:10E0D0001D9241505040E0F70895FB01DC0104C05F
:10E0E0008D910190801921F441505040C8F7881B50
:10E0F000990B0895FB01DC0102C001900D92415083
:10E100005040D8F708956817790768F4FB01DC01DF
:10E11000E40FF51FA40FB51F02C002900E924150EC
:10E120005040D8F70895E6CFDC0101C06D9341500F
:10E130005040E0F70895FC018191861721F0882373
:10E14000D9F7992708953197CF010895FB01DC0194
:10E1500001900D920020E1F708950F931F93CF9344
:10E16000DF93CDB7DEB72E97CDBFDEBF0E891F89F7
:10E17000888D998D26E02C8309831A8397FF02C02E
:10E1800080E090E801978D839E83AE01445E5F4FEF
:10E190006A8D7B8DCE01019667D04D815E8157FDE2
:10E1A0000AC02F813885421753070CF49A01F801F1
:10E1B000E20FF31F10822E96CDBFDEBFDF91CF910D
:10E1C0001F910F9108950F931F93CF93DF93CDB7B6
:10E1D000DEB72E97CDBFDEBF0E891F89888D998D42
:10E1E0002EE02C8309831A8397FF02C080E090E819
:10E1F00001978D839E83AE01445E5F4F6A8D7B8D58
:10E20000CE01019631D04D815E8157FD0AC02F812C
:10E210003885421753070CF49A01F801E20FF31FF7
:10E2200010822E96CDBFDEBFDF91CF911F910F914F
:10E230000895CF93DF93CDB7DEB72E97CDBFDEBF66
:10E240008DE08C838C899D8989839A83AE01485E99
:10E250005F4F6E897F89CE0101968FD32E96CDBFF9
:10E26000DEBFDF91CF9108952F923F924F925F9240
:10E270006F927F928F929F92AF92BF92CF92DF92D6
:10E28000EF92FF920F931F93CF93DF93CDB7DEB73B
:10E290002C97CDBFDEBF7C016B018A01FC01168289
:10E2A0001782838181FFB0C1CE0101964C01F70135
:10E2B0009381F60193FD859193FF81916F018823EE
:10E2C00009F49EC1853239F493FD859193FF8191C4
:10E2D0006F01853221F4B70190E0D6D4E8CF512CFC
:10E2E000312C20E02032A0F48B3269F030F48032FF
:10E2F00059F0833269F420612CC08D3239F08033BB
:10E3000039F4216026C02260246023C0286021C027
:10E3100027FD27C030ED380F3A3078F426FF06C0CD
:10E32000FAE05F9E300D1124532E13C08AE0389E10
:10E33000300D1124332E20620CC08E3221F426FDC4
:10E340005FC1206406C08C3611F4206802C0883694
:10E3500041F4F60193FD859193FF81916F01811145
:10E36000C1CF982F9F7D9554933028F40C5F1F4F99
:10E37000FFE3F9830DC0833631F0833771F08335C5
:10E3800009F057C021C0F801808189830E5F1F4FBB
:10E3900044244394512C540114C03801F2E06F0E10
:10E3A000711CF801A080B18026FF03C0652D70E0CC
:10E3B00002C06FEF7FEFC5012C871DD42C018301B4
:10E3C0002C852F77222E16C03801F2E06F0E711CBB
:10E3D000F801A080B18026FF03C0652D70E002C067
:10E3E0006FEF7FEFC5012C87FBD32C012C852068B4
:10E3F000222E830123FC19C0832D90E04816590674
:10E40000A0F4B70180E290E03FD43A94F5CFF50153
:10E4100027FC859127FE81915F01B70190E034D4FC
:10E4200031103A94F1E04F1A51084114510479F730
:10E43000DEC0843611F0893631F5F80127FF07C0B8
:10E4400060817181828193810C5F1F4F08C0608160
:10E450007181072E000C880B990B0E5F1F4F2F76D2
:10E46000722E97FF09C090958095709561957F4FAA
:10E470008F4F9F4F2068722E2AE030E0A40155D4C0
:10E48000A82EA81843C0853729F42F7EB22E2AE083
:10E4900030E025C0F22FF97FBF2E8F36C1F018F47F
:10E4A000883579F0ADC0803719F0883721F0A8C0E1
:10E4B0002F2F2061B22EB4FE0DC08B2D8460B82E9C
:10E4C00009C024FF0AC09F2F9660B92E06C028E01D
:10E4D00030E005C020E130E002C020E132E0F80188
:10E4E000B7FE07C060817181828193810C5F1F4FED
:10E4F00006C06081718180E090E00E5F1F4FA40133
:10E5000014D4A82EA818FB2DFF777F2E76FE0BC003
:10E51000372D3E7FA51450F474FE0AC072FC08C06B
:10E52000372D3E7E05C0BA2C372D03C0BA2C01C052
:10E53000B52C34FF0DC0FE01EA0DF11D8081803342
:10E5400011F4397E09C032FF06C0B394B39404C0FD
:10E55000832F867809F0B39433FD12C030FF06C0D4
:10E560005A2CB31418F4530C5B18B32CB31460F486
:10E57000B70180E290E03C8787D3B3943C85F6CF27
:10E58000B31410F43B1801C0312C34FF11C0B70193
:10E5900080E390E03C8778D33C8532FF16C031FDA4
:10E5A00003C088E790E002C088E590E0B7010CC0A6
:10E5B000832F867851F031FF02C08BE201C080E2E8
:10E5C00037FD8DE2B70190E05FD3A51430F4B701B9
:10E5D00080E390E059D35A94F8CFAA94F401EA0D5D
:10E5E000F11D8081B70190E04FD3A110F6CF332009
:10E5F00009F45DCEB70180E290E046D33A94F7CFBC
:10E60000F7018681978102C08FEF9FEF2C96CDBFD7
:10E61000DEBFDF91CF911F910F91FF90EF90DF90C0
:10E62000CF90BF90AF909F908F907F906F905F90B2
:10E630004F903F902F90089520FD09C0FC0123FDCD
:10E6400005C022FF02C07383628351834083089513
:10E6500044FD10C046FD10C0DB01FC01AA0FBB1F2A
:10E66000EE1FFF1F1094D1F76A0F7B1F8E1F9F1F95
:10E6700031E003C033E001C034E0660F771F881F2C
:10E68000991F3150D1F7620F711D811D911D0895A1
:10E690000F931F93CF93DF938C01C801B7D2EC0186
:10E6A00097FD06C08AD2892BC1F7B801CE0124D3C9
:10E6B000CE01DF91CF911F910F9108958F929F927C
:10E6C000AF92BF92CF92DF92EF92FF920F931F9380
:10E6D000CF93DF931F92CDB7DEB78C01C62E7A01A0
:10E6E000298394D2AC01552729814B32510521F061
:10E6F0004D32510561F42068CA94C11002C080E017
:10E700006FC0C801298382D2298197FDF8CF322FAB
:10E710003D7FD32E322F307339F5803329F5BB245A
:10E72000BA94BC0C09F449C0C80129836FD229816D
:10E7300097FD43C0382F3F7D383561F48D2D8264BD
:10E74000D82ECA94CA94CC20C1F1C8015FD297FFD9
:10E750000BC033C026FF04C02D2D2260D22E03C073
:10E760003D2D3261D32ECB2C812C912C540120EDE8
:10E77000280F283078F0D4FE03C0B801BDD21AC0EB
:10E780002A3040F0D6FEF9CF2F7D3FEE320F3630E3
:10E79000A0F727504D2DC501B4015ADF4B015C0194
:10E7A0008D2D8260D82ECA94CC2051F0C8012ED273
:10E7B00097FFDDCFD1FC04C0A2CF812C912C540156
:10E7C000D7FE08C0B094A09490948094811C911CB2
:10E7D000A11CB11C2D2DB501A401C7012DDF81E0C5
:10E7E0000F90DF91CF911F910F91FF90EF90DF90ED
:10E7F000CF90BF90AF909F908F9008956F927F922F
:10E800008F929F92AF92BF92CF92DF92EF92FF9240
:10E810000F931F93CF93DF93CDB7DEB7A197CDBFF3
:10E82000DEBF5C017A01CE0101966C0180E2F60147
:10E8300011928A95E9F7F501838040E050E0912C30
:10E84000712C70E0A1E0B0E0F90183FC859183FEBA
:10E8500081918F01982F9F01811103C080E090E08A
:10E860007AC08E3519F44115510549F1E72FF0E0D2
:10E87000E417F5073CF48D3559F18D3219F4772002
:10E8800001F103C0711001C0982E892F86958695DD
:10E8900086958601080F111D892F87703D0101C0E3
:10E8A000660C8A95EAF7F80180818629808399159C
:10E8B00059F0991510F49F5FE8CF9150E6CF71E0C1
:10E8C00004C07724739401C0712C4F5F5F4FBCCF9D
:10E8D000772019F08E8180628E83711103C0992494
:10E8E000939416C0F6019E012F5D3F4F8081809565
:10E8F0008193E217F307D1F7F2CFE114F10429F085
:10E90000F7018083C70101967C016150912CE9F0E9
:10E91000C50169A37BD169A197FD15C0282F269554
:10E9200026952695F601E20FF11D208130E0AC011D
:10E930004770552702C0359527954A95E2F720FD87
:10E94000DCCFB501D9D1911089CFE114F10411F0D8
:10E95000F7011082C801A196CDBFDEBFDF91CF9134
:10E960001F910F91FF90EF90DF90CF90BF90AF90ED
:10E970009F908F907F906F9008954F925F927F92BB
:10E980008F929F92AF92BF92CF92DF92EF92FF92BF
:10E990000F931F93CF93DF931F92CDB7DEB76C0118
:10E9A0002B015A01FC0116821782712CF601F380AB
:10E9B000F201F3FC8591F3FE8191382F2F0188231A
:10E9C00009F4E5C090E03983F8D03981892B19F03A
:10E9D000C6015EDEEBCF353241F4F201F3FC359136
:10E9E000F3FE31912F01353259F4C60139830ED12E
:10E9F000398197FDCAC03817C9F2B6017DD1C7C0A9
:10EA00003A3239F4F3FC3591F3FE31912F0151E0A4
:10EA100001C050E0420110E020ED230F2A3088F4BD
:10EA20005260612F70E080E090E040E2598310DE98
:10EA3000162FF401F3FC3591F3FE31914F0159810A
:10EA4000EBCF052F232F240151FF03C0111102C06A
:10EA50009EC01FEF383619F03C3659F011C0F40152
:10EA6000F3FC2591F3FE21912F01283649F4052F5F
:10EA700008600460F201F3FC2591F3FE21912F015F
:10EA8000222309F484C0622F70E083E299E1298394
:10EA90009CD02981892B09F47AC000FD07C0F501BB
:10EAA000E080F180C50102965C0102C0E12CF12CEE
:10EAB0002E3649F4F6014681578160E070E0202F40
:10EAC000C701BADD73CF233689F401FF11E0C60117
:10EAD0009DD097FD5AC0E114F10429F0F70180831D
:10EAE000C70101967C01115091F74BC02B3551F4B1
:10EAF0009201A701612FC60181DE2C01892B09F04B
:10EB000040C03AC0C6012983C3DD298197FD3DC0BD
:10EB10002F3641F128F4243619F1293631F124C079
:10EB2000233769F02537E1F01FC0E114F10429F023
:10EB3000F7018082C70101967C01115059F0C6018E
:10EB400065D04C0197FD06C038D0892B71F3B60112
:10EB5000C401D2D0E114F104A1F0F701108211C078
:10EB6000006203C0006101C00064202FA701612F73
:10EB7000C601A4DD811105C0F6018381807329F4EB
:10EB800006C000FD13CF739411CF772019F0872DA5
:10EB900090E002C08FEF9FEF0F90DF91CF911F9118
:10EBA0000F91FF90EF90DF90CF90BF90AF909F902C
:10EBB0008F907F905F904F900895911114C1803293
:10EBC00019F089508550D0F70895FC01059006167C
:10EBD00021F00020D9F7C00108953197CF010895A1
:10EBE000FC010590615070400110D8F78095909518
:10EBF0008E0F9F1F0895FC0161507040019001101D
:10EC0000D8F7809590958E0F9F1F0895CF93DF932F
:10EC1000EC012B8120FF33C026FF0AC02F7B2B8302
:10EC20008E819F8101968E839F838A8190E029C087
:10EC300022FF0FC0E881F9818081082E000C990B1A
:10EC4000009719F420622B831AC03196E883F98368
:10EC50000EC0EA85FB85199597FF09C02B810196A7
:10EC600011F080E201C080E1822B8B8308C02E81ED
:10EC70003F812F5F3F4F2E833F83992702C08FEF45
:10EC80009FEFDF91CF9108950F931F93CF93DF9361
:10EC9000FB01238121FD03C08FEF9FEF28C022FFDE
:10ECA00016C046815781248135814217530744F4A9
:10ECB000A081B1819D012F5F3F4F208331838C93D1
:10ECC000268137812F5F3F4F2683378310C0EB01AA
:10ECD000092F182F0084F185E02D1995892BE1F675
:10ECE0008E819F8101968E839F83812F902FDF914C
:10ECF000CF911F910F910895FB01238120FF12C036
:10ED000026FD10C08F3F3FEF930761F082832F7D78
:10ED1000206423832681378121503109268337835C
:10ED2000992708958FEF9FEF0895FA01AA272830B9
:10ED300051F1203181F1E8946F936E7F6E5F7F4FC8
:10ED40008F4F9F4FAF4FB1E03ED0B4E03CD0670F44
:10ED5000781F891F9A1FA11D680F791F8A1F911D97
:10ED6000A11D6A0F711D811D911DA11D20D009F4E7
:10ED700068943F912AE0269F11243019305D319329
:10ED8000DEF6CF010895462F4770405D4193B3E012
:10ED90000FD0C9F7F6CF462F4F70405D4A3318F0B9
:10EDA000495D31FD4052419302D0A9F7EACFB4E06A
:10EDB000A6959795879577956795BA95C9F7009722
:10EDC0006105710508959B01AC010A2E06945795C3
:10EDD000479537952795BA95C9F7620F731F841F1A
:10EDE000951FA01D089599278827089503D0808135
:10EDF00099270895E0ECF1E0378537FDFDCF3485A4
:10EE000038603487FC01E050F04F0895262FF2DF80
:10EE10000080021611F008D001970197089501961D
:10EE2000272FF5DFF3CF262FE0ECF1E0378537FD14
:10EE3000FDCF3485377F3487378531FF09C036E30E
:10EE4000328738ED34BF31E03387378537FDFDCF6A
:10EE500033E33287808391831282248325E32287E0
:10EE600028ED31E024BF338701960895052E97FBE6
:10EE700016F400940FD057FD05D014D007FC02D033
:10EE800046F408C050954095309521953F4F4F4F1F
:10EE90005F4F089590958095709561957F4F8F4F46
:10EEA0009F4F0895A1E21A2EAA1BBB1BFD010DC0A6
:10EEB000AA1FBB1FEE1FFF1FA217B307E407F5072A
:10EEC00020F0A21BB30BE40BF50B661F771F881F06
:10EED000991F1A9469F760957095809590959B019C
:0CEEE000AC01BD01CF010895F894FFCFF4
:10EEEC0002400F0083100000010410000001820892
:10EEFC000000010000000000000000000000040001
:10EF0C0080000100000000000000D727DE27DE276C
:10EF1C00EA27F62700281D282B28542857285B2879
:10EF2C003E000426140004043E00042E040C0404C9
:10EF3C000008000800000000000000080008080895
:10EF4C000808080008000800000008080008080865
:10EF5C0000800080000000000000008000808080A5
:10EF6C008080800080008000000080800080808095
:10EF7C00000100010000000000000001000101017F
:10EF8C00010101000100010000000101000101016B
:10EF9C000000000000000000000000000000000065
:10EFAC000101010101010101010101010101010145
:10EFBC000101010101010101010101010101010135
:10EFCC000101010101010101010101010101010125
:10EFDC000000000000000000000000000000000025
:10EFEC000000000000000000000000000000000015
:10EFFC000000000000000000000000000000000005
:10F00C0001010101010101010101010101010101E4
:10F01C0000000000000000000000000000000000E4
:10F02C0000000000000000000000000000000000D4
:10F03C0001010101010101010101010101010101B4
:10F04C0000000000000000000000000000000000B4
:10F05C000101010101010101010101010101010194
:10F06C000101010101010101010101010101010184
:10F07C000000000000000000000000000000000084
:10F08C000101010101010101010101010101010164
:10F09C000000000202000002000202020200000254
:10F0AC000000000202000002000202020200000244
:10F0BC000000000202000002000202020200000234
:10F0CC0004040406060404060406060606040406E4
:10F0DC0004040406060404060406060606040406D4
:10F0EC000000000202000002000202020200000204
:10F0FC0000000002020000020002020202000002F4
:10F10C0004040406060404060406060606040406A3
:10F11C0000000002020000020002020202000002D3
:10F12C000404040606040406040606060604040683
:10F13C000404040606040406040606060604040673
:10F14C000404040606040406040606060604040663
:10F15C000404040606040406040606060604040653
:10F16C000000000202000002000202020200000283
:10F17C000000000202000002000202020200000273
:10F18C000404040606040406040606060604040623
:10F19C000008080800000008000008000808000823
:10F1AC000008080800000008000008000808000813
:10F1BC000008080800000008000008000808000803
:10F1CC0010181818101010181010181018181018F3
:10F1DC0010181818101010181010181018181018E3
:10F1EC0000080808000000080000080008080008D3
:10F1FC0000080808000000080000080008080008C3
:10F20C0010181818101010181010181018181018B2
:10F21C0000080808000000080000080008080008A2
:10F22C001018181810101018101018101818101892
:10F23C001018181810101018101018101818101882
:10F24C001018181810101018101018101818101872
:10F25C001018181810101018101018101818101862
:10F26C000008080800000008000008000808000852
:10F27C000008080800000008000008000808000842
:10F28C001018181810101018101018101818101832
:10F29C000000C05AC55AE35AEC5A115B2B5B345B25
:10F2AC00675B875BCD5B005C434C4F4E4500434C2A
:10F2BC004F4E455F4D465500546F6F206D616E7912
:10F2CC0020646174612E000D0A000D0A50415249F0
:10F2DC005459204552524F52000D0A504152495434
:10F2EC0059204F4B002534753A20002533750043C7
:10F2FC0061726420436C6F6E656420746F20536C74
:10F30C006F7400556E6B6E6F776E20636172642044
:10F31C00747970652E002573206F7220004D756C0A
:10F32C007469706C6520706F73736962696C697451
:10F33C006965732C206E6F7420636C6F6E61626CE8
:10F34C00652100436C6F6E6564204F4B2100436C4C
:10F35C006F6E6520756E737570706F727465642155
:0AF36C00004E4F20444154410000C0
:020000021000EC
:1000000000000000000000000000000000000000F0
:1000100000000000000000000000000000000000E0
:1000200000000000000000000000000000000000D0
:1000300000000000000000000000000000000000C0
:00000001FF
